:100000002E6A040000000000FFFFFF00FFFFFF005A
:10001000FFFFFF00FFFFFF00FFFFFF00FFFFFF00EC
:10002000FFFFFF00FFFFFF00FFFFFF001E030000B8
:10003000FFFFFF00FFFFFF00D8020000FFFFFF00EF
:10004000FFFFFF00FFFFFF00FFFFFF00BC010000FC
:10005000FFFFFF0072030000FFFFFF00FFFFFF0034
:10006000FFFFFF00FFFFFF00FFFFFF008402000013
:1000700030020000FFFFFF00FFFFFF00FFFFFF0057
:10008000FFFFFF00FFFFFF0000010000FFFFFF0078
:10009000FFFFFF00FFFFFF00FFFFFF00FFFFFF006C
:1000A000FFFFFF00FFFFFF00FFFFFF00FFFFFF005C
:1000B000FFFFFF00FFFFFF00FFFFFF00FFFFFF004C
:1000C000FFFFFF00FFFFFF00FFFFFF00FFFFFF003C
:1000D000FFFFFF00FFFFFF00FFFFFF00FFFFFF002C
:1000E000FFFFFF00FFFFFF00FFFFFF00FFFFFF001C
:1000F000FFFFFF00FFFFFF00FFFFFF00FFFFFF000C
:10010000FFFFFF00FFFFFF00FFFFFF00FFFFFF00FB
:10011000FFFFFF00FFFFFF00FFFFFF00FFFFFF00EB
:10012000FFFFFF00FFFFFF00FFFFFF00FFFFFF00DB
:10013000FFFFFF00FFFFFF00FFFFFF00FFFFFF00CB
:10014000FFFFFF00FFFFFF00FFFFFF00FFFFFF00BB
:10015000FFFFFF00FFFFFF00FFFFFF00FFFFFF00AB
:10016000FFFFFF00FFFFFF00FFFFFF00FFFFFF009B
:10017000FFFFFF00FFFFFF00FFFFFF00FFFFFF008B
:10018000FFFFFF00FFFFFF00FFFFFF00FFFFFF007B
:10019000FFFFFF00FFFFFF00FFFFFF00FFFFFF006B
:1001A000FFFFFF00FFFFFF00FFFFFF00FFFFFF005B
:1001B000FFFFFF00FFFFFF00FFFFFF00FFFFFF004B
:1001C000FFFFFF00FFFFFF00FFFFFF00FFFFFF003B
:1001D000FFFFFF00FFFFFF00FFFFFF00FFFFFF002B
:1001E000FFFFFF00FFFFFF00FFFFFF00FFFFFF001B
:1001F000FFFFFF00FFFFFF00FFFFFF00FFFFFF000B
:100200000200FA003600F800801F7800200020006D
:100210000C000900B01F780032048000001020009C
:10022000000061004801DE000200E0004B003200E7
:10023000C0108000620060004101DE0060005100DB
:1002400040003A00C0108000610160003B003200B5
:10025000E0108000000F7800020F200060004700CF
:100260001002610002092000020052001A0036004C
:10027000E0024700150078004500DE0065005000F0
:100280004101DD0060F720000202400004608800A8
:1002900005007800100078006F0160004006200023
:1002A0000010B800000A78000500780010007800FF
:1002B0007001600004003200F0FF2F001060880021
:1002C0006801040000000000100020001060880099
:1002D0009A0104000000000060024700140078004A
:1002E0004400DE006F016000A00020000011B80093
:1002F00004007800100078006F00600000014100E9
:10030000006080001008410000608000100178004B
:1003100020C020001091B900006080000208780021
:10032000B27B800040C0200060081100C07B8000CC
:10033000306088002201040000000000A8010400D1
:1003400000000000D2FF2F00802120001008610073
:10035000F2EF2F006008200010086100A0012000CB
:100360000C0009004F1078004F0078003600F900AB
:100370000080FA00004006003600F800801F780078
:10038000200020000C000900B01F7800210480002C
:100390000020200000806000C900DE000100E000B5
:1003A000290032007010800062006000C100DE0091
:1003B000608050001E003A0070108000E100600074
:1003C0001900320081C02000A0D0200090804000A1
:1003D000901080008048780050688000E100400064
:1003E00051688800F00F200000806000506888008D
:1003F000E1004000F00F20000081600081D020006B
:100400001100510006003A001000200060688800CA
:10041000000020004068880000002000506888002C
:10042000DC010400000000001E02040000000000C7
:10043000D1FF2F00E020200010886000F1DF2F00A6
:100440004008200010886000A00120000C00090076
:100450004F1078004F0078003600F9000040060089
:100460003600F800801F7800200020000C000900F2
:10047000B01F78008640AE00780204000000000043
:100480005E61AE004E02040000000000E00A800041
:1004900001002000400204000000000061F0200084
:1004A000C8A2AE005E0204000000000080087800D0
:1004B000910098007602040000000000000178001E
:1004C00011005100706888008000EB00816888008E
:1004D000916880000100E00004003A00A1688000FB
:1004E0000100E00001003200C00E88008640A90033
:1004F000A00120000C0009004F1078004F00780088
:100500003600F900004006003600F800801F780031
:10051000200020000C000900B01F78008620AE00EB
:10052000CC020400000000005A61AE00A2020400E8
:1005300000000000C00A80000100200094020400B6
:100540000000000021F02000C882AE00B2020400CA
:10055000000000008008780091009800CA020400A2
:10056000000000000001780011005100B068880010
:100570008000EB00C1688800916880000100E00005
:1005800004003A00A16880000100E0000100320090
:10059000B00E88008620A900A00120000C000900F0
:1005A0004F1078004F0078003600F9000040060038
:1005B0003600F800801F7800200020000C000900A1
:1005C000B01F78008480AE00120304000000000019
:1005D0004661AE00F602040000000000200A800020
:1005E00001002000E802040000000000A1F020004B
:1005F000D422AE000603040000000000800878004A
:100600009100980010030400000000000001780031
:1006100011005100D06888000000EB00E0688800FD
:100620008480A900A00120000C0009004F10780070
:100630004F0078003600F900004006003600F80050
:10064000801F7800200020000C000900B01F7800F7
:100650008420AE0066030400000000004261AE008A
:100660003C03040000000000000A8000010020009C
:100670002E03040000000000E1F02000D402AE00D0
:100680004C030400000000008008780091009800EE
:100690006403040000000000000178001100510014
:1006A000F06888008000EB00016988009168800094
:1006B0000100E00004003A00A16880000100E000B1
:1006C00001003200D00E88008420A900A001200083
:1006D0000C0009004F1078004F0078003600F90038
:1006E000004006003600F800801F7800200020003F
:1006F0000C000900B01F7800220480000080200058
:10070000000061004B01DE000200E0003F0032000B
:100710001215800000082000000061004701DE0083
:100720000200E00008003200101480001069880008
:10073000201480002069880000148000306988003F
:10074000B0030400000000009014800010698800CD
:10075000A01480002069880080148000306988001F
:1007600032698000CF91DE0080D220001018410055
:10077000109049006469800012002000C0D220005F
:1007800010084100923E2000020052001C0035007B
:10079000A23E2000CF91DE004069800051698000B8
:1007A0000002EB00E51F07007069880002002000CE
:1007B000CF91DE0042698800536988000200200062
:1007C0006269880002D3200012015000726988001B
:1007D0006000510002003D000000200070698800A8
:1007E00072698000CF91DE0020D3200010184100F4
:1007F000109049001200200060D3200010484100F2
:10080000F27F2F004008200010086100A0012000A6
:100810000C0009004F1078004F0078003600F900F6
:100820000040060001002800C02020001088700051
:1008300001402000E0202000108870000000060029
:100840000000FA007110800000102000008060009D
:10085000C800DE000100E00002003A0022040400AB
:100860000000000068005700104078000080FB0086
:10087000801088000080FA000000060000000000E0
:100880000000000090108000000006007010800042
:100890006100600000000600711080000010200060
:1008A00000806000C800DE000100E00003003A00A4
:1008B000000000004C0404000000000000000600DE
:1008C0000C00FA0000422000C0698800E0432000CC
:1008D000D069880060442000E0698800C04420009E
:1008E000F069880020412000006A880040582000FC
:1008F000106A8800000020006010880000002800B6
:100900007010880048000700000F78001107980059
:10091000823E2000CF91DE00C732070020079800FA
:1009200031079800000F780011079800660020003A
:10093000CFB3DE006A02570034017800A4017800CA
:100940000603E900030035000201D0008381D200D4
:10095000FBFF370042079800530798000002EB00A6
:100960004A1F07002E029000BE0290004E01900028
:10097000DE019000200798003107980004007800FD
:10098000850078000002EB006C1F0700000F780064
:100990001107980012002000CF91DE004E00900059
:1009A000DE00900000027800810278000201E90078
:1009B000030035008502D1000482D300FBFF37001D
:1009C0002E019000BE0190000400510005805900E6
:1009D0000500360012002000CF91DE0060004700C5
:1009E0001018410010904900600147003200780063
:1009F000A200780061005000E0805800000F7800ED
:100A000011079800A0108800D2FF2F00E0202000DE
:100A10001008610083FF07000D0007000C000700AD
:100A20000080FA000000060000882300110020006A
:100A300000000600010028006021200010887000DE
:100A40000140200080212000108870000000060076
:100A5000E0462000801F7800A0072000801F78005B
:100A6000AB2F07004F00B100000006000000FA00A5
:100A7000C11080000010200000806000C800DE006F
:100A80000100E00002003A00380504000000000008
:100A900068005700104078000080FB00D0108800EC
:100AA0000080FA00000006000000000000000000C6
:100AB000E010800000000600C010800061006000AF
:100AC00000000600C11080000010200000806000BF
:100AD000C800DE000100E00003003A000000000052
:100AE000620504000000000000000600F1FF27007E
:100AF0006021200010886000F1BF2F0080212000BD
:100B00001088600000000600F1FF2700C0202000D0
:100B100010886000F1BF2F00E020200010886000E6
:100B2000000006000C00FA0060532000C069880035
:100B300040552000D0698800C0552000E069880039
:100B400020562000F0698800A0512000006A88002B
:100B500060572000106A880000002000B010880054
:100B600000002800C0108800AFFF0700000F7800C9
:100B700011079800823E2000CF91DE002E32070040
:100B80002007980031079800000F7800110798009F
:100B900066002000CFB3DE006A02570034017800FF
:100BA000A40178000603E900030035000201D0002B
:100BB0008381D200FBFF370042079800530798005B
:100BC0000002EB00B11E07002E029000BE02900052
:100BD0004E019000DE019000200798003107980038
:100BE00004007800850078000002EB00D31E0700A7
:100BF000000F78001107980012002000CF91DE004E
:100C00004E009000DE009000000278008102780023
:100C10000201E900030035008502D1000482D300FF
:100C2000FBFF37002E019000BE0190000400510030
:100C3000058059000500360012002000CF91DE002B
:100C40006000470010184100109049006001470003
:100C500032007800A200780061005000E080580067
:100C6000000F780011079800F0108800D2FF2F00C5
:100C700080212000100861006EFF070074FF07004C
:100C800073FF07000080FA00000006004003200008
:100C9000401588003030200030158800C004200046
:100CA000001588002020200010158800700020000A
:100CB00020158800B0FF2F003016880000002000AB
:100CC000A0168800F0FF2F0090168800000020007A
:100CD000C016880000002000F01688000000060002
:100CE000F1F32F00E02020001088600001022000B6
:100CF000800920009080680000072000808060004C
:100D00008009200010886800F1DF2F0040082000D3
:100D10001088600001202000C008200010887000AA
:100D2000F1F32F00802120001088600011002000C6
:100D3000000A200010806800E7006000000A200020
:100D4000108868000000200030088800000128009A
:100D500080088800E004200070088800000020005F
:100D60005008880000012800900888000100280031
:100D7000002A200010887000F17F2F00400820001A
:100D80001088600001802000C008200010887000DA
:100D900001082000A015200010887000110020001C
:100DA000A015200010806800E7006000A01520005A
:100DB0001088680001022000C009200090806800AF
:100DC0000007200080806000C009200010886800B3
:100DD000D1FF2F0060082000108860002100200053
:100DE000E00820001088700001082000E0152000B5
:100DF0001088700011002000E015200010806800AD
:100E0000E7006000E0152000108868000120200045
:100E1000C009200090806800007020008080600081
:100E2000C009200010886800B1FF2F006008200072
:100E30001088600041002000E00820001088700049
:100E400001082000201420001088700011002000EC
:100E50002014200010806800E700600020142000AB
:100E6000108868000102200040092000908068007E
:100E70000007200080806000400920001088680082
:100E8000D1FF2F00400820001088600021002000C2
:100E9000C0082000108870000108200060142000A5
:100EA000108870001100200060142000108068007D
:100EB000E700600060142000108868002100200016
:100EC0006009200010806800E700600060092000D1
:100ED00010886800F1FE2F00400820001088600094
:100EE00001012000C00820001088700000000600EA
:100EF0000000FA00F1FB2F000022200010886000A3
:100F00000011800062006000C100DE000100E0000E
:100F10000200320080070400000000006800570053
:100F2000100078002011880000118000E1006000AE
:100F300002003A0094070400000000002011800025
:100F40000080FA00000006000000FA0001002800FE
:100F500000222000108870000080FA0000000600C7
:100F60000000FA00F1FF2700002220001088600036
:100F70000080FA00000006000000FA0080772000E0
:100F8000206A8800407A2000306A8800007B2000B8
:100F9000406A880068005700900078006A00570097
:100FA000908070006C005700908070006E005700B9
:100FB00090807000700057009080700072005700A1
:100FC000908070007400570010817000F600570088
:100FD0002022200011087100F1FB2F0000222000C8
:100FE0001088600001002800002220001088700096
:100FF0000080FA00000006000C00FA0060004700C4
:1010000041642F000A00090031587800E0222000D6
:10101000801F7800D0032000801F78003C2E07003E
:101020004F00B10060004700801F7800F11A0700F0
:101030002F00B100E0462000801F7800A0072000AC
:10104000801F7800322E07004F00B1006800570063
:1010500010007800A01088000080FA000000060050
:101060000200FA00F0FF2F00000F780054688000A3
:1010700083D02000130052000E00320083C02000F5
:1010800080D0200090814100134078000080FB0058
:10109000000F780040688000E1014000436888004C
:1010A00002102000110009008281D80001007800A0
:1010B000406888001E0078000080FA0000000600EA
:1010C0005168800080D020001080500002003A005B
:1010D0000000200001003700100020000000060082
:1010E0000000FA006C0157009240780010002000C8
:1010F000124910000104E0001D0032004EB89700B4
:101100009040780060C05000070032003EB9970060
:101110004EB897009040780012C0500002003A008C
:10112000A808040000000000CEB897003EB8970061
:101130001041780001007800904078008180FB0029
:101140000281FB0002007800008050000900370097
:101150001100200068005700108840001100200096
:101160006A00570010884000720804000000000068
:10117000000020000080FA00000006000400FA00D1
:101180006800570010007800100798000000200049
:10119000000F7800620047009000780060805000E7
:1011A0001100360011002000620047001088100076
:1011B0001E017800110020006000470010884000E8
:1011C0006A0057001000410010417800C102200061
:1011D0000140510002003200D80804000000000065
:1011E000CA080400000000001E0078000080FA0019
:1011F000000006002A00FA0070004700F1642F008A
:1012000013000900315878000000200030079800D2
:1012100000002000010020004007980051079800BE
:10122000D0CC2C00C1DC2300600798007107980027
:10123000000020002017980000002000000F780018
:101240006000470010017800730051001C003D0051
:10125000680057001001780060004700100041004E
:1012600010427800D20220000240520014003900DF
:10127000680057001001780060004700100041002E
:101280001042780092032000024052000C003E0001
:1012900070004700E0024700150240006800570058
:1012A000100178000500780010004100104A780015
:1012B00010002000950A40002009040000000000F2
:1012C000F002470060024700148142000000200045
:1012D000004978000400780010007800100798009A
:1012E00004007800100078002007980005007800BE
:1012F00010427800D20220000240520002003A0060
:1013000010002000300798006600470010007800A9
:10131000000F78006000470010027800620147006B
:101320001200520018003D007001470060004700A5
:101330001000410010427800E202200002405200FA
:101340000C003A0060014700120078002007980066
:101350000200780010027800660147001200520077
:1013600002003A00F0FF2F0020079800C409040093
:10137000000000001200200060004700100841003B
:101380008A09040000000000F4FF2F0064014700F8
:10139000120012002A003200640047001001780099
:1013A00060004700610851006000470010027800AB
:1013B0006601470012005200210035006E009000C7
:1013C000FE0090000200200003122400F42D07000C
:1013D000301798004117980060079800710798002F
:1013E0007001470060004700100041001041780084
:1013F0000281FB000003200000005100CF80DE00CE
:101400000081EB008B2D07003E119000CE11900063
:10141000E32D07006802470034017800A40178003A
:10142000B42E0700400798005107980012002000D2
:101430006000470010081100D409040000000000FB
:101440000000200001F82300600798007107980051
:1014500062004700100078006102500064014700FC
:10146000120012003D003200F4FF2F00640147001B
:101470001200120003003A006600470010007800D6
:101480002007980000002000201798006600470001
:10149000100178006000510002003A0010002000A6
:1014A000201798006400470010017800660047008C
:1014B0001002410042022000020147006000470084
:1014C00012084200600047001002780062014700E5
:1014D0001200520021003D000200200003122400EF
:1014E0006E009000FE009000382F07003017980023
:1014F0004117980060079800710798007001470035
:101500006000470010004100104178000281FB009C
:101510000003200000005100CF80DE000081EB00BE
:10152000442D07003E119000CE1190009C2D070025
:101530006802470034017800A40178006D2E07008E
:1015400040079800510798001200200060004700F3
:1015500010084100620A0400000000006600470015
:10156000100178006100510007003A004E00900021
:10157000DE0090000200200003F82B00882D0700F9
:1015800040079800510798004E009000DE00900040
:101590000080FA00000006000600FA00CEB89700AE
:1015A000114078000080FB00000F7800020220004C
:1015B000E000470011001100060032006000470003
:1015C000900078006980500002003200F40A0400A4
:1015D0000000000011002000680057001088400043
:1015E000CE0A040000000000000020001007980050
:1015F0000000200020079800D2022000E0004700F1
:101600001100110008003A0011002000640047009A
:10161000108840001100200068005700108840002A
:10162000220B040000000000B2022000E00047008E
:101630001100110003003A0011002000680057005B
:1016400010884000CEB89700114078000080FB0061
:10165000000F780060004700901F7800611A0700B3
:101660002F00B1000000E0000D00320062024700D0
:1016700094007800A00020000089B9000103200038
:101680006000470010801000000A41001100200097
:101690006800570010884000220B04000000000082
:1016A0002E0090000000E0000400320062004700BD
:1016B0001000780060001000010037001E0090004C
:1016C0000080FA00000006000800FA004EB99700FA
:1016D000124078000080FB00000F78000402200018
:1016E000600147001200120006003200600047004F
:1016F0001001780069005100020032008C0B0400D8
:10170000000000001200200068005700100841008F
:10171000660B04000000000000002000CF80DE0007
:10172000100798002107980000002000300798005B
:101730004EB8970010427800D202200002405200BA
:1017400008003A001200200066004700100841001F
:10175000120020006800570010084100C20B04006E
:10176000000000004EB8970010427800B20220003E
:101770000240520003003A001200200068005700A7
:10178000100841004EB99700124078000080FB001D
:10179000000F780060004700901F7800111A0700C2
:1017A0002F00B1000000E000120032001E00900087
:1017B000AE009000A2002000030020001E2F0700B2
:1017C00004032000600147001201120002027800A9
:1017D000CFA2DE00620147000419400005914800D5
:1017E000120020006800570010084100C20B0400DE
:1017F000000000003E0090000000E0000600320003
:101800006200470030017800A001780060001100FC
:10181000E0801900020037001E009000AE0090002A
:101820000080FA00000006000000FA006A0157007C
:1018300062004100904078002003200001487800B9
:1018400012007800C00088009C05BA00B00080003B
:101850000080FA00000006000A00FA006A00570043
:1018600010007800100798004EB9970032007800F9
:10187000A20078002007980031079800000020009F
:10188000000F780060004700100278006C015700DC
:101890001200520015003D00640047004007980008
:1018A000B01F7800A01F7800DFFF07004F00B100D5
:1018B0001E0190000009780022002000620047000D
:1018C0001008410022002000CF91DE004E00900061
:1018D00010184100109049001200200060004700DD
:1018E00010084100420C0400000000006C0057008A
:1018F000100078004100DD004EB99700CF80DE0077
:1019000012194000129148000080FA000000060001
:101910004E00FA0060004700D1672F000500090063
:10192000315878006600470031682F000500090033
:10193000315878006C00470091682F0005000900BD
:101940003158780072004700F1682F000400090048
:10195000315878007700470041692F0005000900E1
:10196000315878007D004700A1692F00060009006A
:10197000315878004002200000004700116A2F0013
:10198000020009003158780000002000101F980064
:1019900068005700901F7800862507002F00B100CF
:1019A0006200500040179800610150006800570025
:1019B0001000410010427800A202200002405200B4
:1019C0000200320000002000D5023700860220000D
:1019D00006034700160078006100500068025700B7
:1019E0001401400000002000004978000400780045
:1019F00010017800060078001000410010417800C6
:101A00000281FB00000320000001510052179800E2
:101A1000690051000400340072002000A002200080
:101A20000000470010081100A0022000000047003D
:101A3000100078004400DD00101F98008002200094
:101A40000000470010007800610140006800570066
:101A500010004100104178000281FB0000032000CB
:101A60000001510052179800690051000400340031
:101A700072002000A00220000000470010081100A2
:101A8000A002200000004700100178002003200081
:101A9000000047001008410000002000506A880044
:101AA0000000200050179800000020004017980008
:101AB00068005700100178008002200000004700F5
:101AC0001000410010417800604051000E003200CB
:101AD00068005700100078008402200004024700CC
:101AE00014004000104178000281FB00A002200099
:101AF000000047001008690010002000140A400090
:101B0000580D0400000000002003200000004700E2
:101B100010027800A20220000201470012005200C9
:101B20000400320010002000506A880000002000ED
:101B30007B02370050002000801F780068005700AB
:101B4000901F780060004700801F780064FD070048
:101B50006F00B10060015000D6003A0068025700E3
:101B6000542798001400780071004000104178005C
:101B700070D320000248780004007800901F78009D
:101B800010002000801F78007CFD07004F00B1008E
:101B9000401798006601400068005700100141009E
:101BA00000002000004978005E20900010017800BD
:101BB00080022000000047004027980010004100EC
:101BC00064004000801F78008AFD07002F00B100EC
:101BD000606A8800716A8800800220000000470067
:101BE00010007800640140006800570010014100B7
:101BF00000002000004978005E209000100178006D
:101C00004E2090001000410062004000801F7800CC
:101C100061FE07002F00B100806A8800800220006A
:101C20000000470010007800620140006800570083
:101C30001001410000002000004978005E20900063
:101C4000100178004E20900010004100801F7800A5
:101C500051FE07002F00B100906A8800680057000D
:101C6000901F780030002000801F780043FD07009F
:101C70004F00B10040179800680157001200400063
:101C800062004000801F78005AFD07002F00B1005D
:101C9000201F9800311F980080022000000047009C
:101CA00010007800620140006800570010014100F8
:101CB00000002000004978005E20900010017800AC
:101CC0004E20900010004100801F780049FD070061
:101CD0002F00B10020279800312798000200200033
:101CE000032724002E189000BE189000372D0700FF
:101CF0002E219000BE2190007E2C0700A06A880053
:101D0000B16A880068005700901F780040002000EA
:101D1000801F780019FD07004F00B10068015700CF
:101D2000120040001041780080D520000248780061
:101D30005E209000901F780050002000801F7800E7
:101D40000EFD07004F00B1004017980068015700D2
:101D50001200400063004000801F780025FD07004E
:101D60002F00B100201F9800311F98008002200032
:101D70000000470010007800630140006800570031
:101D80001001410000002000004978005E20900012
:101D9000100178004E20900010004100801F780054
:101DA00014FD07002F00B10020279800312798006C
:101DB00002002000032724002E189000BE18900077
:101DC000022D07002E219000BE219000492C070013
:101DD000D06A8800E16A880068005700901F780088
:101DE00060002000801F7800E4FC07004F00B10075
:101DF00068015700120040001041780090D5200083
:101E0000024878005E209000901F7800700020004B
:101E1000801F7800D9FC07004F00B100680157000F
:101E200012004000801F7800F2FC07002F00B10074
:101E300062E52000D3FE2300592B0700F06A8800DA
:101E4000016B880068005700901F78008000200018
:101E5000801F7800C9FC07004F00B10068015700DF
:101E600012004000801F7800E2FC07002F00B10044
:101E7000106B8800216B880068005700901F780065
:101E800090002000801F7800BCFC07004F00B100CC
:101E90006801570012004000801F78000AFE07000A
:101EA0002F00B100306B8800416B880010002000CB
:101EB0009B01370050002000801F78006800570009
:101EC000901F780066004700801F780084FC0700A0
:101ED0006F00B1006001500028003A006800570010
:101EE000901F780070002000801F7800A3FC07007E
:101EF0004F00B1006801570012004000801F7800B9
:101F0000A5FD07002F00B100506B88006800570046
:101F1000901F780080002000801F780097FC070049
:101F20004F00B1006801570012004000801F780088
:101F3000B0FC07002F00B100606B8800716B880057
:101F400068005700901F780090002000801F7800E4
:101F50008AFC07004F00B1006801570012004000E2
:101F6000801F7800A3FC07002F00B100806B880061
:101F7000916B88001000200069013700500020009C
:101F8000801F780068005700901F78006C004700A1
:101F9000801F780052FC07006F00B1006001500004
:101FA000CF003A0010002000A06B880068005700A6
:101FB000901F780030002000801F78006FFC070021
:101FC0004F00B1006801570012004000801F7800E8
:101FD00071FD07002F00B1005017980060015000FC
:101FE00004003D0000002000501798000810040075
:101FF00000000000A002200000004700100178004F
:102000006C00510002003400C000200050179800FE
:10201000A002200000004700100078004017980040
:10202000A002200000004700100178006C00510061
:1020300016003D00A40220000402470014007800AE
:102040004201DD0060D720000201400000002000B6
:102050000009780004007800100078004201DD00DB
:1020600060D7200002004000620140000000200014
:102070000009780012002000A002200000004700A4
:102080001008410010100400000000006800570014
:10209000901F780020002000801F780037FC070088
:1020A0004F00B1006801570012004000801F780007
:1020B00039FD07002F00B100610150006217980040
:1020C0006300510084003D00C00220000000470072
:1020D000100078004201DD0080022000000047006F
:1020E00010011100421798006400510002003400F2
:1020F0004000200040179800000020005017980072
:10210000A002200000004700100278008202200098
:1021100002014700120052006F003D0068005700A6
:10212000901F7800A00220000000470010007800F7
:102130004200DD0064004000801F78000FFC0700B3
:102140004F00B100101F98006801570012004000B6
:10215000104178006040510059003200680057007B
:10216000100178002003200000004700100041000B
:1021700010427800C202200002405200500032009B
:10218000C00220000000470060279800100078007F
:102190004201DD00A0022000000047005027980007
:1021A000100041004201DD0060D720000200400025
:1021B00040279800680057002027980010017800F9
:1021C000200320000000470010004100801F78001D
:1021D000F1FC07002F00B1004E21900000097800AB
:1021E0002E209000901F78005E2090001000780054
:1021F0004200DD006400400063004000801F780062
:10220000DEFB07004F00B100101F9800C202200043
:1022100002014700120178004212DD00A2022000F4
:1022200002014700120142004212DD0062D7200085
:102230000401410062014100222798006801570013
:1022400012004000801F7800D3FC07002F00B1006F
:102250004101DD002E209000020878006E209000E1
:10226000100078004201DD005E2090001000410067
:102270004201DD0060D72000020040006202400001
:1022800032062000140011000D003600C0022000AC
:1022900000004700100078004201DD00A00220008D
:1022A00000004700100041004201DD0060D720001F
:1022B0000200400062014000300620000009780062
:1022C00012002000A002200000004700100841007A
:1022D0008010040000000000100020009000370073
:1022E00050002000801F780068005700901F780081
:1022F00072004700801F780079FB07006F00B10073
:102300006001500006003A0077004700801F780007
:10231000191607002F00B1001000200080003700C0
:1023200050002000801F780068005700901F780040
:102330007D004700801F780069FB07006F00B10037
:102340006001500073003A0080C52F00F1072000A3
:10235000002798001127980010002000801F7800A7
:10236000A002200000004700801F78000004200029
:1023700000004700801F780037FD07006F00B100A4
:1023800020002000801F7800E002200000004700AD
:10239000801F78000004200000004700801F7800A4
:1023A0002DFD07006F00B100E00220000000470093
:1023B000B01F7800A01F780030662F00801F7800C3
:1023C00060DA2000801F7800E82207008F00B1004B
:1023D00060DA2000801F7800E71507002F00B100A9
:1023E0005E12900012002000A002200000004700B2
:1023F00010081100600052003F003400000420006B
:102400000000470030027800A002780042FF2F0051
:10241000F30720000200520003805A0036003E00FD
:1024200020002000801F780080032000000047006B
:10243000801F78000004200000004700801F780003
:1024400005FD07006F00B10020002000801F78000C
:10245000C003200000004700801F78000004200017
:1024600000004700801F7800FBFC07006F00B100F0
:1024700010002000801F780080022000000047002C
:10248000801F78000004200000004700801F7800B3
:10249000F1FC07006F00B10080022000000047003F
:1024A000901F7800C003200000004700B01F780094
:1024B000A01F78008003200000004700B01F7800B4
:1024C000A01F7800D0662F00801F780060DA2000FF
:1024D000801F7800A5220700EF00B10060DA20001D
:1024E000801F7800A41507002F00B1000060FE00D7
:1024F000F01104000000000040022000000047002E
:10250000801F78009C1507002F00B10010002000EC
:102510000300370020002000506A880000002000DF
:102520000080FA00000006000000FA00106F800032
:102530000000E0001100320068005700901F780092
:102540009C2207002F00B100810220000080500073
:10255000C180DE00206F800068004000801F78008E
:10256000811F7800600A07004F00B1006800570023
:10257000901F7800A22207002F00B1000080FA000F
:10258000000006001000FA0060004700616B2F0099
:102590000C00090031587800606B8000716B80007E
:1025A00002002000030020000A2A07000000E000CB
:1025B00002003C0000002000010037001000200055
:1025C0000000E00058003200626B8000736B8000F6
:1025D000306F8000416F8000FE2907000000E0009E
:1025E00002003D0000002000010037001000200024
:1025F0000000E0004C003200606B8000716B8000D6
:10260000306F8800416F8800526F80006000510079
:1026100035003C00106F80000000E0000100320037
:10262000B4120700D06A8000E16A8000606F880001
:10263000716F8800A06A8000B16A8000806F880096
:10264000916F8800806B8000916B8000A06F880084
:10265000B16F880080D5200010427800320520003C
:102660000240520005003A0002002000030028004A
:1026700000DF2000101869001090690090D520003C
:1026800010427800720520000240520005003A0016
:102690000200200003002800C0DE2000101869009E
:1026A00010906900906A800020708800806A800025
:1026B00030708800606A8000716A8000A12807007D
:1026C000407088001000200050708800000020003A
:1026D000801F7800901507002F00B10072220700BC
:1026E0009013040000000000506F80006100500053
:1026F000506F8800801F7800406A2F00801F78008C
:1027000060DA2000801F7800182207006F00B100F7
:1027100060DA2000801F780083FF07002F00B100DF
:10272000E213040000000000546F8000C2E02000AB
:10273000120052001F0032000000200070079800B5
:102740006E00470010017800760051000A003D003D
:1027500062DA20006E0047001001410000022000F4
:1027600000497800120020006E0047001008410068
:10277000A01304000000000062DA20006E00470091
:1027800010014100000020000049780060DA2000BC
:10279000801F780064FF07002F00B1006070800088
:1027A000506F880060004700801F78005EFF0700C0
:1027B0002F00B1007070800081708000306F880041
:1027C000416F88000080FA00000006000800FA004F
:1027D0006A005700B01F7800A01F78008F02070022
:1027E0004F00B10000017800810178000000200056
:1027F00001F82300BA2907000000E00002003500BC
:102800000000200001003700100020000000E00060
:102810000300320000002000010020006D0037009E
:102820003EB89700CEB897003EB99700CEB9970052
:10283000DB280700200798003107980000002000DF
:1028400001F82300821F7800831F78002E0190007A
:10285000BE019000642907004F01BE00801F780070
:10286000811F78005D0007004F00B100000F780065
:10287000110798006A005700B01F7800A01F780069
:10288000660207004F00B100000178008101780066
:10289000F0282C0051F323004E2907000000E0002F
:1028A00002003C0000002000010037001000200062
:1028B0000000E0000A0032001E0178009E01900036
:1028C0003EB89700CEB89700402A0700801F7800D6
:1028D000811F78006B0207004F00B1003D003700F8
:1028E0006A01570032007800A20078000200200040
:1028F000030020007A2907000000E00002003500F4
:102900000000200001003700100020000000E0005F
:102910001D0032006000470030017800A0017800FF
:10292000000020000100280000006900818069008B
:102930003EB99700CEB99700242A0700801F78007F
:10294000811F78004F0207004F00B1002007980058
:1029500031079800B0FD200091FC2300821F780011
:10296000831F78002E019000BE0190001E290700F1
:102970004F01BE0002002000030028000200680092
:1029800083806800130037003EB99700CEB99700E6
:102990001E0078009E0090000C2A0700801F78001F
:1029A000811F7800370207004F00B1002007980010
:1029B00031079800B0FD200091FC2300821F7800B1
:1029C000831F78002E019000BE01900006290700A9
:1029D0004F01BE000080FA00000006000E00FA0061
:1029E0006A01570032007800A2007800020020003F
:1029F000030020003A2907000000E0000200340034
:102A00000000200001003700100020000000E0005E
:102A10000300320000002000010020006F0037009A
:102A20006A01570032007800A2007800000F780099
:102A3000110798000200780030017800A0017800AA
:102A40000000200001F82300E22807000000E00059
:102A500002003C00000020000100370010002000B0
:102A60000000E000070032001E0178009E01900087
:102A70000000200001F82300D4290700000F78008F
:102A8000110798006A004700801F78006000470027
:102A9000B01F7800A01F7800520007006F00B1003F
:102AA000000F7800110798006A01470012017800B2
:102AB0004191DE00821F7800801F7800811F78001E
:102AC0009C0007006F00B100000F7800110798000C
:102AD0006A00570030017800A00178000000200053
:102AE00001F82300BB2807000000E00002003C00C2
:102AF0000000200001003700100020000000E0006E
:102B0000070032001E0178009E01900000002000A6
:102B100001F82300AD290700000F78001107980085
:102B200040012000400798001E0178009E0190009F
:102B30003EB89700CEB89700A4290700600247006E
:102B40006407980034017800A4017800E9280700A0
:102B500002002000030024009C29070020079800A1
:102B60003107980000027800810278006E00900022
:102B70000001780032007800A2007800040178009B
:102B800085017800D62807000000E000020032002E
:102B90000000200001003700100020000000E000CD
:102BA00002003200EA150400000000006401470042
:102BB00032007800A2007800000F7800110798001A
:102BC000680047001000780061015000420798003B
:102BD000D5FF3A001E0078009E0090000080FA00A9
:102BE000000006000400FA00600247006A01570076
:102BF00032007800A2007800001A780001127800F4
:102C0000620042001001780000F827000000610017
:102C1000C701DE00E20720002EB8970002885100AD
:102C2000E201420000F023001301680000F82700D1
:102C3000000061009309680034007800A400780067
:102C40000080FA00000006000600FA006A01570042
:102C500032007800A200780002002000030020006B
:102C60009F2807000000E000020034000000200060
:102C700001003700100020000000E00003003200D7
:102C800000002000010020002800370060004700FD
:102C9000801F78006A005700B01F7800A01F7800DE
:102CA000D0FF07006F00B1000200200003002400E5
:102CB000BB2707000200200003F823004A28070072
:102CC00030BF9F0041BF9F001400200060014700FB
:102CD0001209120082002000821F7800426C2F002F
:102CE000821F7800801F7800811F78006B06070024
:102CF0008F00B100100798002107980030BF9F0097
:102D000041BF9F001E007800CF80DE000081EB00F5
:102D1000482707008221270013F32300A02707007C
:102D20001E019000AE019000722807000080FA009A
:102D3000000006000400FA00E00147006A015700A5
:102D400032007800A20078008019780081117800A4
:102D5000628041001001780000F827000000610047
:102D60004701DE006C0057001001410022BF9F00A8
:102D70006000510003003D00000020000100200021
:102D800023003700F30F20006C0157001280110060
:102D9000130034006A01570032007800A200780066
:102DA00002002000030020004D2807000000E00082
:102DB0000200350000002000010037001000200054
:102DC0000000E00003003200F0FF2F00F1F72F00B9
:102DD0000F003700F0FF2F00F1F727000C0037003D
:102DE00060004700E20140006C00570010007800CE
:102DF0004700DD001301680000F8270000006100B3
:102E0000930968006001470032007800A200780052
:102E10000080FA00000006000800FA006A0157006E
:102E200032007800A2007800020020000300200099
:102E30002B2807000000E000020032000000200004
:102E400001003700100020000000E0000300320005
:102E50000000200001F823007B0037006A005700C3
:102E600030017800A0017800E04F2D00212B2400D4
:102E70001B2807000000E0000200350000002000D1
:102E800001003700100020000000E00003003200C5
:102E9000F0FF2F00F1F727006B0037006A005700A2
:102EA00030017800A001780000C52A00E12A2C003A
:102EB000C82707000000E00002003C0000002000DE
:102EC00001003700100020000000E0000300320085
:102ED00000002000010020005B0037006A0157005D
:102EE00032007800A20078000200200003002000D9
:102EF000FB2707000000E000020035000000200072
:102F00000100370010002000000F78000000E000F2
:102F10000500320002002000030028006A0057006C
:102F200010186900109069003EB89700CEB897005D
:102F3000B2A32A0083FB23001927070030BF9F009C
:102F400041BF9F00801F7800811F78008305070024
:102F50004F00B1007B26070030079800CF80DE00CD
:102F60000081EB00B32607001007980021079800A6
:102F70006A01570032007800A2007800821F7800B2
:102F8000831F78001E019000AE0190009627070075
:102F90004F01BE0030BF9F0041BF9F003E01900027
:102FA000821F780092002000821F7800826E2F001E
:102FB000821F7800801F7800811F7800B705070006
:102FC0008F00B100801F7800811F780059FF070033
:102FD0006F00B10030BF9F0041BF9F001E0078000E
:102FE0000000E000160032006A005700300178004F
:102FF000A0017800F0FF2F00F1F72700B8270700A5
:103000000000E00002003200000020000100370054
:10301000100020000000E00003003200000020004B
:1030200001002000080037003EB99700CEB9970094
:103030000000200001F82300642807000200370088
:103040003EB89700CEB897000080FA000000060056
:103050000600FA0000002000000F78006A01570007
:1030600032007800A2007800020020000300200057
:103070009B2707000000E000020032000000200053
:1030800001003700100020000000E00003003200C3
:1030900000002000010020005E0037006E01570094
:1030A00032007800A2007800020020000300200017
:1030B0008B2707000000E000020032000000200023
:1030C00001003700100020000000E0000300320083
:1030D0000000200001F823004E0037006A0157006D
:1030E00032007800A20078000200200003002000D7
:1030F0007B2707000000E0000200350000002000F0
:1031000001003700100020000000E0002200320023
:103110001EB89700AEB89700261507001007980054
:10312000210798000001EB0042260700000278000A
:10313000810278006E01570032007800A20078000A
:103140000401780085017800652707000000E00091
:1031500002003A00000020000100370010002000AB
:103160000000E00003003200000020000100200009
:103170002800370062004700100178006000470017
:103180006108610002002000030028006A00570067
:1031900010186900109069006A005700B01F78008D
:1031A000A01F7800A8FE07004F00B10030BF9F00AD
:1031B00041BF9F001EB99700AEB99700782607005F
:1031C00030BF9F0041BF9F00801F7800811F7800A3
:1031D00011FF07004F00B10030BF9F0041BF9F00AB
:1031E0001E0078000000E000080032006A0057006E
:1031F00030017800A00178000000200001002800C4
:103200000000690081806900020037003EB8970025
:10321000CEB897000080FA00000006000000FA0017
:103220006A01570032007800A200780002002000F6
:10323000030020002A2707000000E00002003500FC
:103240000000200001003700100020000000E00016
:10325000080032006A00570030017800A0017800B1
:103260000000200001002800000069008180690042
:10327000020037003EB89700CEB897000080FA00F1
:10328000000006000A00FA006A005700B01F78002C
:10329000A01F7800E1FF07004F00B1001007980061
:1032A0002107980002002000030020000C270700DF
:1032B0000000E000020032000000200001003700A2
:1032C000100020000000E000030032000000200099
:1032D000010020006B0037006200470030027800D8
:1032E000A00278000000200001F82300040178000B
:1032F00085017800FA2607000000E0000200350092
:10330000000020000100370010002000000F7800AE
:103310000000E000070032001E019000AE019000A6
:103320000000200001F82300A827070010079800DC
:10333000210798001E009000AE0090001E01900032
:10334000AE0190001626070030079800410798004C
:1033500054002000841F780004712F00841F78001F
:10336000801F7800811F7800CC0407008F00B10017
:103370001E019000AE01900009260700100798007A
:103380002107980040002000801F780080722F00E5
:10339000801F780066004700B01F7800A01F7800EB
:1033A000BE0407008F00B1000001780081017800A1
:1033B0001E009000AE0090008427070010079800C0
:1033C000210798001E0078000000E0000A0032008B
:1033D000B6FD200097FC230062024700340178000C
:1033E000A401780006007800870078007E26070098
:1033F00010079800210798006A02570034007800EF
:10340000A40078000200200003002000B42607007A
:103410000000E0000200350000002000010037003D
:10342000100020000000E0000B00320062004700A6
:1034300030027800A002780000002000010028007F
:1034400000006A0081806A00000378008103780030
:10345000361A0400000000006202470034007800C1
:10346000A40078000003780081037800060078004B
:103470008700780010079800210798001E00900030
:10348000AE0090000080FA00000006000000FA0084
:103490006E01570032007800A20078000200200080
:1034A000030020004B2607000000E00002003C0063
:1034B0000000200001003700100020000000E000A4
:1034C0000A0032001EB99700AEB997003EB89700C7
:1034D000CEB897003D270700801F7800811F780035
:1034E00068FF07004F00B1007D0037006A015700F8
:1034F00032007800A20078000200200003002000C3
:10350000342607000000E00002003D00000020001B
:1035100001003700100020000000E0001A00320017
:103520006E01570032007800A200780002002000EF
:10353000030020006A2607000000E00002003500BA
:103540000000200001003700100020000000E00013
:103550000D0032001EB99700AEB997003EB8970033
:10356000CEB8970019270700801F7800811F7800C8
:1035700044FF07004F00B100B2FD20009304240077
:103580005C260700560037006A01570032007800B9
:10359000A20078000200200003002000502607004F
:1035A0000000E000020035000000200001003700AC
:1035B000100020000000E0002A0032006E015700D9
:1035C00032007800A20078000200200003002000F2
:1035D000432607000000E000020035000000200044
:1035E00001003700100020000000E0000D00320054
:1035F0001EB99700AEB997003EB89700CEB89700B5
:10360000F2260700801F7800811F78001DFF070049
:103610004F00B100B2FD200093042C0035260700B6
:103620002F0037006E01570032007800A2007800AA
:103630000200200003002000292607000000E0000F
:1036400002003200000020000100370010002000BE
:103650000000E00003003200B0FD200091FC2B00D0
:103660001F0037006E01570032007800A20078007A
:103670000200200003002000192607000000E000DF
:10368000020032000000200001003700100020007E
:103690000000E000100032006A015700320078009C
:1036A000A20078000200200003002000C9250700C6
:1036B0000000E00002003C00000020000100370094
:1036C000100020000000E00003003200B0FD2000E8
:1036D00091FC2300020037000000200001002000C0
:1036E0000080FA00000006001800FA00D06A80008E
:1036F000E16A8000B2FD2000930424002825070021
:103700000200200043332400B0260700000F780099
:1037100011079800A06A8000B16A8000B2FD200005
:10372000930424001E2507000200200043332400D8
:10373000A6260700400798005107980090D5200062
:1037400010437800740520000440530005003A003F
:1037500004002000050028006000470010186A00DF
:1037600010906A0080D520001043780034052000B6
:103770000440530005003A00040020000500280022
:103780006800470010186A0010906A00C40020000A
:10379000680057001022B800C0DE2000040240007C
:1037A000040F980034007800A4007800B2FD2000D7
:1037B00093042400FA24070002002000433324006D
:1037C0008226070020079800310798000E08900015
:1037D0006402400034007800A4007800B2FD2000AC
:1037E00093042400EE240700020020004333240049
:1037F00076260700600798007107980004002000F3
:1038000005002400841F7800851F780068034700A6
:1038100036027800A602780004017800850178005D
:10382000712507000200200003002400672607001E
:10383000801F7800811F7800BC0307004F00B10093
:10384000801F7800811F780001FE07008F00B10003
:10385000200F9800310F980068004700B01F7800D3
:10386000A01F78004E0407004F00B100000F980021
:10387000110F98006C004700B01F7800A01F78005F
:10388000470407004F00B1000E0A90009E0A900006
:103890000401780085017800C1240700000F98001A
:1038A000110F98000000200001002400801F780004
:1038B000811F78006400470030037800A00378007F
:1038C0006002470034017800A40178000600780007
:1038D0008700780044250700020020000300240030
:1038E0003A260700801F7800811F78008F030700A9
:1038F0004F00B100801F7800811F7800D4FD0700C1
:103900008F00B1000E0A90009E0A9000040178001A
:1039100085017800A22407002E0A9000BE0A9000BC
:10392000040178008501780072250700801F780067
:10393000811F780029FC07004F00B100801F78002C
:10394000811F7800A1FB07004F00B100020020009A
:1039500003002400922407000200200043332400C7
:103960008F240700B2FD20009304240017260700CF
:1039700002002600A37624008924070062E52000C7
:10398000D3FE23008624070090708800A170880071
:103990000400200005002400841F7800851F7800A3
:1039A000801F7800811F7800A9FD07008F00B100FB
:1039B000000F9800110F9800000020000100240063
:1039C000801F7800811F78001A0EF8001C0EF80086
:1039D0009FFD07008F00B1000E0A90009E0A900024
:1039E000040178008501780042250700801F7800D7
:1039F000811F7800F9FB07004F00B100B07088000C
:103A0000C170880068004700B01F7800A01F7800D0
:103A1000E30307004F00B100000F9800110F98005A
:103A20006C004700B01F7800A01F78003F0307001C
:103A30004F00B1000E0A90009E0A90000401780029
:103A40008501780056240700200F9800310F980058
:103A500068004700B01F7800A01F780033030700FC
:103A60004F00B100000F9800110F98006C00470044
:103A7000B01F7800A01F7800C90307004F00B100F5
:103A80000E0A90009E0A90000401780085017800DB
:103A900043240700000F9800110F980064004700AE
:103AA00030037800A00378006002470034017800FA
:103AB000A40178000600780087007800CA24070077
:103AC000801F7800811F7800B50307004F00B10008
:103AD0000E0A90009E0A900004017800850178008B
:103AE0002F240700000F9800110F98002E08900057
:103AF000BE089000821F7800831F78000E09900096
:103B00009E099000B82407004F01BE00801F780076
:103B1000811F78006400470030037800A00378001C
:103B20006002470034017800A401780006007800A4
:103B300087007800AC240700801F7800811F780080
:103B4000FA0207004F00B100000F9800110F980013
:103B50006C004700B01F7800A01F7800900307009A
:103B60004F00B1000E0A90009E0A900004017800F8
:103B7000850178000A240700801F7800811F7800E3
:103B800042FE07008F00B1000200200043332400F2
:103B900003240700B2FD2000930424008B250700B6
:103BA000F0708800017188000200200003002000EE
:103BB000CB2407000000E0000200350000002000D8
:103BC00001003700100020000000E0000900320072
:103BD00004002000453B2400F0708000017180004B
:103BE0000401780085017800C2240700F070880085
:103BF00001718800546B800063005200360034006D
:103C0000F46A8000056B80001071800021718000D3
:103C10000401780085017800B12407000000E0006D
:103C200002003500000020000100370010002000D5
:103C30000000E00004003200F06A8000016B8000A8
:103C40001071880021718800B4708000C5708000F8
:103C50003071800041718000040178008501780096
:103C60009F2407000000E000020035000000200053
:103C700001003700100020000000E00004003200C6
:103C8000B0708000C1708000307188004171880080
:103C9000D4708000E57080005071800061718000F8
:103CA00004017800850178008D2407000000E00001
:103CB0000200350000002000010037001000200045
:103CC0000000E00004003200D0708000E17080004D
:103CD00050718800617188000080FA0000000600C1
:103CE0002A00FA0060004700C1732F000400090099
:103CF000315878006500470011742F000E0009004C
:103D00003158780026032000E4E2200074004700C8
:103D10001408430068005700100278006000520049
:103D200015003A00807180000000E00010003200B1
:103D300000002000A0718800000020009071880021
:103D4000000020008071880074004700901F7800F8
:103D5000700B2000801F7800DE0107004F00B100CB
:103D600060004700801F7800A51C07002F00B100ED
:103D7000CC2104000000000084718000600052002B
:103D80000C003A0010002000807188007400470089
:103D9000901F7800700B2000801F7800CD01070075
:103DA0004F00B10065004700801F7800941C070099
:103DB0002F00B1003EB897000000E0005001320033
:103DC000B4718000C5718000D2708000E370800003
:103DD000040078008500780003240700300F980065
:103DE000410F98000002780081027800D0718000B5
:103DF000E171800004017800850178003824070013
:103E00000000E00002003500000020000100370043
:103E1000100020000000E00006003200D071800099
:103E2000E1718000300F9800410F9800521F04008C
:103E300000000000D4718000E571800000002000C7
:103E40000100280000036A0081836A0076004700B1
:103E500030027800A0027800060078008700780021
:103E60000401780085017800DA2307000000E000F3
:103E700002003C000000200001003700100020007C
:103E80000000E00007003200D6718000E77180007A
:103E900004002000050028007600470004186B008D
:103EA00005906B003E089000CE089000F2718000F3
:103EB000037280003A230700700F980001179800E2
:103EC0000002780081027800107280002172800068
:103ED0000401780085017800012407000000E0005B
:103EE0000200350000002000010037001000200013
:103EF0000000E00006003200107280002172800095
:103F0000700F980001179800C01F04000000000007
:103F1000147280002572800000002000010028003B
:103F200000036A0081836A007E0047003002780047
:103F3000A00278000600780087007800040178006D
:103F400085017800A32307000000E00002003C0088
:103F50000000200001003700100020000000E000F9
:103F600007003200167280002772800004002000D3
:103F7000050028007E00470004186B0005906B00C8
:103F8000F46A8000056B800030728000417280000E
:103F900004017800850178008E2307000000E0000E
:103FA00002003C000000200001003700100020004B
:103FB0000000E0000A00320032728000437280008C
:103FC000F06A8000016B8000802407007E09900069
:103FD0008E119000F2220700700F980001179800D0
:103FE000F470800005718000126B8000236B8000EC
:103FF00004007800850078007B230700500F9800AC
:10400000610F980000027800810278000000200013
:10401000413324000401780085017800B0230700B3
:104020000000E00002003500000020000100370021
:10403000100020000000E0000C0032007A00470071
:1040400030027800A002780002002000433B2400E8
:10405000040078008500780063230700500F980063
:10406000610F980068200400000000007A004700FB
:1040700030027800A00278000000200041332C00BC
:104080000401780085017800522307000000E00059
:1040900002003C000000200001003700100020005A
:1040A0000000E0000A0032007A0047003002780089
:1040B000A002780000002000413B240004017800A9
:1040C000850178008B230700500F9800610F98003E
:1040D0007A00470030027800A0027800000020003B
:1040E0004123240004017800850178007C23070027
:1040F0000000E00002003500000020000100370051
:10410000100020000000E000060032000000200047
:1041100041232400500F9800610F9800B82004003C
:10412000000000007A00470030027800A00278000A
:104130000000200041232C00040178008501780054
:10414000242307000000E00002003C0000002000E3
:1041500001003700100020000000E00004003200E1
:104160000000200041232C00500F9800610F9800A0
:1041700002002000433324005E089000EE08900007
:1041800012240700527280006372800084220700AC
:10419000101798002117980000027800810278001B
:1041A0000000200001172400040178008501780038
:1041B0004B2307000000E000020035000000200053
:1041C00001003700100020000000E000060032006F
:1041D00000002000011724001017980021179800F4
:1041E0001C21040000000000200220000000470005
:1041F00030027800A00278000000200001172C0097
:104200000401780085017800F22207000000E00038
:1042100002003C00000020000100370010002000D8
:104220000000E000040032000000200001172C0014
:1042300010179800211798007E0047003002780080
:10424000A0027800827280009372800004007800DF
:1042500085007800E4220700BA2107007072880008
:10426000C61220000602500004003400C0122000D4
:10427000707288004A2104000000000076728000FD
:1042800044ED2F000400530002003D0040ED2F00DC
:104290007072880020022000000047003002780081
:1042A000A0027800B2728000C3728000040078001F
:1042B00085007800CC2207000200200003102400B3
:1042C000372207009F210700A0728800C612200035
:1042D0000602500004003400C0122000A0728800C2
:1042E0008021040000000000A672800044ED2F0031
:1042F0000400530002003D0040ED2F00A072880032
:104300007472800020E320003017980010025200E1
:1043100032002000110009000202D8003E12900075
:10432000140040004017980090718800A47280002B
:1043300040E32000301798001002520032002000A5
:10434000110009000202D8003E1290001403400040
:10435000A6718800C4E520004E1090001484B900B6
:10436000D872880000E6200010B3B900F672880009
:104370001673880064D12000601D2000140814000A
:10438000E4D02000801D200014084300E4D1200068
:10439000A01D2000140813000080FA000000060091
:1043A0000E00FA0080C52F00F1072000400798009A
:1043B00051079800D06A8000E16A8000000F780001
:1043C00011079800A06A8000B16A80002007980059
:1043D0003107980080D52000104278003205200077
:1043E0000240520005003A000200200003002800AD
:1043F00064004700101869001090690090D52000F3
:1044000010427800720520000240520005003A0078
:104410000200200003002800600047001018690017
:1044200010906900D2708000E3708000A06F80005F
:10443000B16F8000AF22070042210700600798009B
:1044400020002000801F780060004700801F780057
:1044500068005700901F7800AC0E07006F00B10095
:1044600020002000801F780064004700801F780033
:1044700068005700901F7800A40E07006F00B1007D
:1044800010002000801F78006C004700801F78001B
:1044900068005700901F78009C0E07006F00B10065
:1044A0006A00570010007800600798001000200094
:1044B000801F78006C004700801F7800680047006C
:1044C000801F7800910E07006F00B1000080FA0095
:1044D000000006000000FA006A005700901F7800F4
:1044E00068005700901F780000752F00801F78002B
:1044F00040E62000801F78009C1A07008F00B10062
:1045000040E62000801F7800BD1A07002F00B10090
:104510000080FA00000006000000FA006A00570060
:10452000901F780068005700901F7800D0752F000A
:10453000801F780040E62000801F78008B1A07005B
:104540008F00B10040E62000801F7800AC1A070001
:104550002F00B1000080FA00000006000600FA00FB
:104560006A03570070012000CF80DE003602780019
:10457000A60278000000E900030035008502D100A2
:104580000482D300FBFF3700F00F2000000262001E
:1045900024079800F007200000025200240798002A
:1045A0006000520013003D006A025700340078009A
:1045B000A400780002002000030020004822070029
:1045C0000000E0000200350000002000010037007C
:1045D000100020000000E000030032000000200076
:1045E00001F82B002B003700000020000100200004
:1045F000280037006400470010027800780052005D
:10460000030036003EB89700CEB89700210037006F
:104610003EB89700CEB89700CA2007000081EB0093
:1046200004210700000F78001107980000037800AC
:10463000810378006A02570034007800A4007800F3
:104640000601780087017800252207000000E000BD
:10465000020035000000200001003700100020009B
:104660000000E000090032006000470030027800DE
:10467000A00278000200200003F823000400780064
:1046800085007800D8210700020037001E0078005E
:104690009E0090000080FA00000006000400FA006E
:1046A0006E005700100078004201DD006C005700DA
:1046B0001001410032007800A2007800000F78005D
:1046C000110798001EB897000000E00013003200A8
:1046D0003EB89700CEB897001E0178009E0190006A
:1046E0002F2107006E01570012017800610151006F
:1046F00012BF9F004212DD006C01570012024200FF
:1047000034017800A4017800FA210700000F780036
:104710001107980062230400000000001E007800CA
:104720009E0090000080FA00000006000A00FA00D7
:1047300000002000200798006A025700340078002B
:10474000A40078000200200003002000E4210700FC
:104750000000E000020035000000200001003700EA
:10476000100020000000E0000700320004002000DC
:10477000050028006A00570010186A0010906A00AF
:1047800010002000200798003EB89700CEB8970090
:1047900032982F0023E223000121070030BF9F0041
:1047A00041BF9F00801F7800811F78006BFF0700CA
:1047B0004F00B10030079800410798006A02570087
:1047C00034007800A4007800821F7800831F7800EE
:1047D0003E019000CE019000832107004F01BE00F2
:1047E0000200200003082400ED20070030BF9F00D6
:1047F00041BF9F0000027800810278000000200085
:10480000010024000401780085017800B42107002C
:104810000000E00002003500000020000100370029
:10482000100020000000E000110032006A00570074
:1048300030027800A002780002002000030024006B
:1048400004007800850078006721070030BF9F00D2
:1048500041BF9F002E0090000000E00002003200E7
:104860000000200001003700100020002007980001
:104870006A00570030027800A00278000000200093
:1048800001F82300040178008501780094210700D5
:104890000000E000020035000000200001003700A9
:1048A000100020000000E0000A0032000600200096
:1048B000070024006A02570034017800A401780040
:1048C00006007800870078004721070030BF9F006E
:1048D00041BF9F003EB89700CEB897003EB9970001
:1048E000CEB99700AE200700000F7800110798009E
:1048F00044002000841F7800A4762F00841F7800D5
:10490000801F7800811F780064FF07008F00B100CE
:104910003EB99700CEB99700A120070030BF9F0095
:1049200041BF9F0030002000801F7800E0772F00FB
:10493000801F780060004700B01F7800A01F78003B
:1049400056FF07008F00B100000178008101780058
:104950003EB89700CEB897001C22070030BF9F00DA
:1049600041BF9F002E0090000000E00008003200D0
:104970006A00570030027800A00278000000200092
:104980000100280000006A0081806A0002003700F0
:104990003EB89700CEB897000080FA0000000600ED
:1049A0000000FA006A00570030027800A002780088
:1049B000B0FD2000910424000401780085017800F6
:1049C000472107000000E000020035000000200041
:1049D00001003700100020000000E0000D00320050
:1049E0006A00570030027800A002780042BE2C0016
:1049F000630924000400780085007800FA2007008D
:104A0000801F7800811F780048FF07004F00B10029
:104A10000C0037006A00570030027800A0027800CE
:104A2000B0FD200091FC230004017800850178008E
:104A300030210700801F7800811F78003BFF0700AE
:104A40004F00B1000080FA00000006000600FA00E6
:104A500060004700E1782F00050009003158780018
:104A60006E005700901F78006C005700901F780070
:104A70006A005700901F780068005700901F780068
:104A8000070007008F00B10060004700801F78001A
:104A90005B1907002F00B1000080FA00000006003B
:104AA0000000FA00010920006A0057001080400051
:104AB000801F7800010F2000680057001080400020
:104AC000801F780040792F00801F780040E620008A
:104AD000801F7800251907008F00B10040E62000F4
:104AE000801F7800461907002F00B100010920003F
:104AF0006E00570010804000801F7800010F2000DA
:104B00006C00570010804000801F7800E0792F0073
:104B1000801F780040E62000801F780013190700EE
:104B20008F00B10040E62000801F78003419070094
:104B30002F00B1000080FA00000006000600FA0015
:104B400060004700817A2F00040009003158780086
:104B50006E005700901F78006C005700901F78007F
:104B60006A005700901F780068005700901F780077
:104B7000CBFF07008F00B10060004700801F780066
:104B80001F1907002F00B1000080FA000000060086
:104B90001C00FA0060004700717B2F000F00090025
:104BA0003158780030608000CF80DE000081EB005B
:104BB000A01F0700B2FD200093042400F81F070087
:104BC000020020004333240080210700801F78006A
:104BD000811F7800D5FE07004F00B10002002000C1
:104BE00023352C00EE1F0700200F9800310F98008E
:104BF00020608000CF80DE000081EB008D1F070069
:104C000002002000432B2400BA200700B2FD200040
:104C100093042400E21F0700020020004333240015
:104C20006A210700801F7800811F7800BFFE0700FF
:104C30004F00B1002E099000BE099000D81F070058
:104C4000401F0700100F98002E089000BE0890002B
:104C50000200200003042400D11F070002002000EE
:104C60000300240059210700400F9800510F9800BD
:104C700020608000CF80DE000081EB006D1F070008
:104C800002002000432B24009A200700B2FD2000E0
:104C900093042400C21F07000200200043332400B5
:104CA0004A210700801F7800811F78003CFF070021
:104CB0004F00B1004E099000DE099000B81F0700B8
:104CC000201F0700000F980004EA20001401500084
:104CD00007003A00720047001002780022EA200024
:104CE0001200520002003A00A82604000000000052
:104CF000A20EF800A00EF80000002000801F78002F
:104D000000002000801F780050FF07008F00B100D6
:104D10007002470014007800007588007201470097
:104D2000120078001075880002007800901F78004B
:104D300004007800901F780000002000801F780099
:104D400000002000801F78007CFF07008F00B1006A
:104D500020608000CF80DE000081EB00351F07005F
:104D6000B2FD2000930424008D1F070002002000E4
:104D70004333240015210700801F7800811F78002D
:104D80006AFE07004F00B10002002000032A240041
:104D9000831F0700EB1E0700100F980020608000A3
:104DA000CF80DE000081EB00221F0700B2FD200053
:104DB000930424007A1F07000200200043332400DC
:104DC00002210700801F7800811F7800F4FE070091
:104DD0004F00B10002002000032F2400701F0700C5
:104DE000D81E0700000F980044EA2000140150006C
:104DF00007003A00720047001002780062EA2000C3
:104E00001200520002003A004C270400000000008B
:104E1000AA0EF800A80EF800A60EF800A40EF800DE
:104E20000AFF07008F00B1007201470012007800EE
:104E300024EA20001404400038758800F00347007D
:104E40001700780006EA20009602400025758800C9
:104E50000200780010007800600110000400780063
:104E60001002410054758800070078001000780097
:104E700060011000060078001000410040758800B5
:104E8000841F7800801F7800881F7800851F7800B5
:104E90002AFF07008F00B10000092000801F780062
:104EA000400F2000801F7800D07A2F00801F7800EC
:104EB00040E62000801F78002C1807008F00B1000A
:104EC00040E62000801F78004D1807002F00B10039
:104ED00060004700801F7800491807002F00B100CC
:104EE0000080FA00000006000000FA006800570089
:104EF000901F78006A005700901F7800707C2F0088
:104F0000801F780040E62000801F780017180700F7
:104F10008F00B10040E62000801F7800381807009D
:104F20002F00B1000080FA00000006009600FA0091
:104F30006000470061A22F0004000900315878008A
:104F400065004700B1A22F00040009003158780025
:104F50006A00470001A32F000400090031587800BF
:104F60006F00470051A32F0004000900315878005A
:104F700074004700A1A32F000C00090031587800ED
:104F8000100220000000470071A42F000B00090050
:104F900031587800D00220000000470031A52F00D2
:104FA0000500090031587800300320000000470058
:104FB00091A52F00050009003158780090032000CA
:104FC00000004700F1A52F000500090031587800C6
:104FD000F00320000000470051A62F000500090043
:104FE000315878005004200000004700B1A62F007F
:104FF0000500090031587800B00420000000470087
:1050000011A72F0004000900315878000005200086
:105010000000470061A72F00040009003158780004
:105020005005200000004700B1A72F00050009002F
:1050300031587800B00520000000470011A82F006B
:1050400005000900315878001006200000004700D4
:1050500071A82F0004000900315878006006200074
:1050600000004700C1A82F00020009003158780055
:105070009006200000004700F1A82F000200090060
:1050800031587800C00620000000470021A92F00F9
:105090000200090031587800F006200000004700A7
:1050A00051A92F0002000900315878002007200084
:1050B0000000470081A92F00020009003158780044
:1050C0005007200000004700B1A92F00020009008E
:1050D000315878008007200000004700E1A92F0028
:1050E0000200090031587800B00720000000470096
:1050F00011AA2F000200090031587800E0072000B3
:105100000000470041AA2F00040009003158780030
:10511000300820000000470091AA2F00030009007A
:1051200031587800707180006B004000801F78005B
:105130006075800061004000801F7800E5FC07007A
:105140004F00B100547080006000520012003A001D
:10515000606A8000716A8000FA1D0700801F780075
:10516000500DF800520DF800407D2F00801F780090
:1051700040E62000801F78007C170700AF00B100D8
:1051800040E62000801F78009D1707002F00B10027
:105190005229040000000000606A8000716A8000EB
:1051A000E81D070084E020001402500044879800A6
:1051B000806A800050879800906A8000608798001D
:1051C0006000520008003D00C40320008008200059
:1051D000000047001008420014002000A008200032
:1051E0000000470010081200A0082000000047003F
:1051F0001002780060E020001002520054879800EE
:105200006000520008003D00C4032000A0082000F8
:10521000000047001008420014002000C0082000D1
:105220000000470010081200C008200000004700DE
:105230001002780040E020001002520064879800BD
:105240006000520004003D0084012000C0082000DE
:1052500000004700100842008008200000004700BE
:10526000901F7800A008200000004700901F7800E1
:10527000C008200000004700901F7800A07E2F008B
:10528000801F780040E62000801F78003717070055
:10529000AF00B10040E62000801F780058170700DB
:1052A0002F00B100707180006B004000801F7800FB
:1052B00074172000C0EA200010005200801F780000
:1052C00084FC07004F00B100707580000000E00012
:1052D0000A0032005E0DF800600DF800C07F2F005C
:1052E000801F780040E62000801F78001F1707000D
:1052F0008F00B1009829040000000000F06A8000CF
:10530000016B8000A2212100F3F12300241E07007D
:10531000801F7800811F7800A0802F00801F7800F8
:1053200040E62000801F7800101707008F00B100B2
:1053300040E62000801F7800311707002F00B100E1
:105340008472800095728000D0CC2C00C1E42B00C8
:105350000401780085017800E11E07000000E000EC
:10536000020035000000200001003700100020007E
:105370000000E00018003200847280009572800006
:10538000D0CC2C00C1E42300040178008501780012
:10539000901E07000000E00002003C00000020001A
:1053A00001003700100020000000E0000A00320079
:1053B0002409200004024700000A2000004A780067
:1053C0003409200004024700000C2000004A780045
:1053D000202A0400000000003409200004024700D5
:1053E000400C2000004A780080728000917280009A
:1053F0000200200003002000761E07000000E000ED
:1054000002003C00000020000100370010002000D6
:105410000000E000060032002409200004024700DA
:1054200020082000004A7800202A04000000000024
:10543000240920000402470010082000004A7800D8
:10544000807580009175800092708000A37080004C
:10545000D31D0700D4708000E5708000040178003F
:10546000850178005B1E07000000E00002003C00A0
:105470000000200001003700100020000000E000C4
:105480000600320010042000801F7800F716070085
:105490002F00B100502A040000000000021707008E
:1054A0007071800078004000801F78007417200021
:1054B000C0EA200010005200801F780005FC0700A1
:1054C0004F00B100707580000000E0000A0032005B
:1054D0001A0EF8001C0EF80080812F00801F780043
:1054E00040E62000801F7800A01607008F00B10062
:1054F000962A040000000000D0708000E170800057
:1055000082942F0013052400A51D0700801F78003A
:10551000811F780040822F00801F780040E6200025
:10552000801F7800911607008F00B10040E6200030
:10553000801F7800B21607002F00B100200920005C
:1055400000004700104078000080FB00801F7800BA
:105550003009200000004700104078000080FB0068
:10556000801F780010832F00801F780040E6200005
:10557000801F78007D1607008F00B10040E62000F4
:10558000801F78009E1607002F00B100C616070086
:10559000A07580000000E00014003A00B47580009F
:1055A000C5758000D0758000E17580000401780029
:1055B00085017800071E07000000E00002003C00A3
:1055C0000000200001003700100020000000E00073
:1055D0000600320010042000801F7800A316070088
:1055E0002F00B100F82A040000000000AE160700EA
:1055F0007071800078004000801F78006075800026
:1056000061004000801F7800B2FB07004F00B1002E
:10561000B60EF800B80EF800A0832F00801F7800A7
:1056200040E62000801F7800501607008F00B10070
:1056300040E62000801F7800711607002F00B1009F
:10564000991607000403200040DE200010A2B900D4
:10565000000D200004034000E4E22000E0082000E8
:105660000000470014085300647580000009200002
:105670000000470061084200F47580000576800054
:105680000000200001F82300040178008501780063
:10569000131E07000000E00002003500000020009B
:1056A00001003700100020000000E0006D00320013
:1056B000E008200000004700901F7800000920004B
:1056C00000004700901F780082FB07004F00B100E8
:1056D000F4758000057680001076800021768000C9
:1056E0000401780085017800BA1D07000000E00081
:1056F00002003C00000020000100370010002000E4
:105700000000E0000600320010042000801F780036
:10571000561607002F00B100922B04000000000075
:1057200061160700BE0EF800C00EF80060842F005E
:10573000801F780040E62000801F78000B160700CD
:105740008F00B10040E62000801F78002C16070073
:105750002F00B100E0082000000047001000780092
:105760006D004000801F7800000920000000470005
:10577000901F780057FB07004F00B100C60EF800DD
:10578000C80EF800F0852F00801F780040E620004A
:10579000801F7800F51507008F00B10040E620005B
:1057A000801F7800161607002F00B100E0082000C7
:1057B00000004700100078007A004000801F780049
:1057C0000009200000004700901F780041FB0700FF
:1057D0004F00B100547680006576800070768000BE
:1057E000817680000401780085017800BC1D0700E7
:1057F0000000E0000200350000002000010037003A
:10580000100020000000E00006003200100420001C
:10581000801F7800151607002F00B100142C04001B
:105820000000000020160700CA0EF800CC0EF80099
:10583000B0862F00801F780040E62000801F78008F
:10584000CA1507008F00B10040E62000801F7800D5
:10585000EB1507002F00B10013160700822C04007F
:1058600000000000E008200000004700901F7800C2
:105870000009200000004700901F780015FB07007A
:105880004F00B10060004700801F7800DC15070062
:105890002F00B100E0082000000047001000780051
:1058A0006D004000801F78000009200000004700C4
:1058B000901F780007FB07004F00B100650047000C
:1058C000801F7800CE1507002F00B100E0082000EF
:1058D00000004700100078007A004000801F780028
:1058E0000009200000004700901F7800F9FA070027
:1058F0004F00B1006A004700801F7800C015070004
:105900002F00B10054708000600052000E0232007F
:105910000403200040DE200010A2B900D00D2000BA
:1059200004024000E0E2200010005200708798005E
:10593000801F7800F4182000C0EA200010005200F8
:10594000801F7800E3FA07004F00B10094708000D8
:10595000A570800090768000A17680000401780018
:10596000850178001B1D07000000E00002003C00DC
:105970000000200001003700100020000000E000BF
:1059800048003200707580000000E0000A0032001C
:10599000120EF800140EF80080872F00801F780088
:1059A00040E62000801F7800701507008F00B100CE
:1059B000462D04000000000090708000A17080005F
:1059C000A2212100F3F12300751C0700020024002E
:1059D000C3612400FD1D07000002780081027800E9
:1059E0000000200001F82300040178008501780000
:1059F0003B1D07000000E000020035000000200011
:105A000001003700100020000000E000120032000A
:105A100090708000A1708000A2212100F3F123008A
:105A20005F1C070002002000A3472400E71D0700B9
:105A3000801F7800811F780030882F00801F780039
:105A400040E62000801F7800481507008F00B10055
:105A5000462D04000000000090708000A1708000BE
:105A600082942F00130524004D1C0700801F78002E
:105A7000811F780000892F00801F780040E62000F9
:105A8000801F7800391507008F00B10040E6200024
:105A9000801F78005A1507002F00B1005A2D04000E
:105AA000000000006F004700801F780054150700B9
:105AB0002F00B100E008200000004700100078002F
:105AC0006D004000801F7800B4162000C0EA20005E
:105AD00010005200801F78007EFA07004F00B100CE
:105AE00074004700801F7800451507002F00B100A3
:105AF000B4708000C5708000B0768000C1768000F0
:105B00000401780085017800F51C07000000E00022
:105B100002003500000020000100370010002000C6
:105B20000000E0000600320010042000801F780012
:105B30004E1507002F00B100A22D04000000000048
:105B400059150700707580000000E0000A0032005F
:105B5000160EF800180EF800C0892F00801F78007C
:105B600040E62000801F7800001507008F00B1007C
:105B7000262E040000000000B0708000C17080007C
:105B8000A2212100F3F12300051C070002002400DC
:105B9000C36124008D1D0700000278008102780097
:105BA0000000200001F8230004017800850178003E
:105BB000CB1C07000000E0000200350000002000C0
:105BC00001003700100020000000E0001200320049
:105BD000B0708000C1708000A2212100F3F1230089
:105BE000EF1B070002002000A3472400771D0700D9
:105BF000801F7800811F7800708A2F00801F780036
:105C000040E62000801F7800D81407008F00B10004
:105C1000262E040000000000B0708000C1708000DB
:105C200082942F0013052400DD1B0700801F7800DD
:105C3000811F7800408B2F00801F780040E62000F5
:105C4000801F7800C91407008F00B10040E62000D3
:105C5000801F7800EA1407002F00B100121507001A
:105C60000403200040DE200010A2B900F00820004C
:105C700004034000E4E22000E008200000004700A8
:105C80001408530036152000C4EA20000009200043
:105C90000000470014085300F46A8000056B800080
:105CA0000000200001F02300040178008501780045
:105CB000481C07000000E00002003C00000020003B
:105CC00001003700100020000000E000CE0032008C
:105CD000E008200000004700901F780084022000A8
:105CE000000920000000470010004200801F7800DB
:105CF00009FA07004F00B100100220000000470021
:105D0000801F7800BE1407002F00B100707580005E
:105D10000000E00040003200E008200000004700E2
:105D2000100078006D004000801F780000092000FE
:105D300000004700901F7800E6F907004F00B1000F
:105D4000220EF800240EF800008C2F00801F78002F
:105D500040E62000801F7800841407008F00B10007
:105D600040E62000801F7800A51407002F00B10036
:105D7000E008200000004700100078007A00400092
:105D8000801F78000009200000004700901F780065
:105D9000D0F907004F00B1002A0EF8002C0EF800D1
:105DA000C08D2F00801F780040E62000801F780003
:105DB0006E1407008F00B10040E62000801F7800BD
:105DC0008F1407002F00B10074022000E0082000AB
:105DD0000000470010004200801F780000092000EA
:105DE00000004700901F7800BAF907004F00B1008B
:105DF000260EF800280EF800608F2F00801F780014
:105E000040E62000801F7800581407008F00B10082
:105E1000AC2F040000000000E00820000000470054
:105E2000100078006D004000801F780000092000FD
:105E300000004700901F7800A6F907004F00B1004E
:105E40001071800021718000A2212100F3F1230054
:105E5000531B0700801F7800811F7800F0902F00EF
:105E6000801F780040E62000801F78003F14070064
:105E70008F00B10040E62000801F7800601407000A
:105E80002F00B100E008200000004700100078005B
:105E90007A004000801F78000009200000004700C1
:105EA000901F78008BF907004F00B10050718000FF
:105EB0006171800082942F0013052400381B0700B5
:105EC000801F7800811F7800B0922F00801F78001B
:105ED00040E62000801F7800241407008F00B100E6
:105EE00040E62000801F7800451407002F00B10015
:105EF00074022000E008200000004700100042006B
:105F0000801F78000009200000004700901F7800E3
:105F100070F907004F00B1003071800041718000BE
:105F2000A2212100F3F123001D1B07000200200025
:105F3000A3472400A51C0700801F7800811F78005C
:105F400060942F00801F780040E62000801F7800BA
:105F5000061407008F00B10040E62000801F780083
:105F6000271407002F00B100F4758000057680002B
:105F70000000200001F8230004017800850178006A
:105F8000D71B07000000E0000200350000002000E1
:105F900001003700100020000000E0001600320071
:105FA00044032000E00820000000470010004200E9
:105FB000801F78000009200000004700901F780033
:105FC00044F907004F00B100DA0EF800DC0EF800CB
:105FD00010962F00801F780040E62000801F780078
:105FE000E21307008F00B10040E62000801F780018
:105FF000031407002F00B10010002000F076880085
:10600000A430040000000000F4768000610052001B
:106010004D003A00E008200000004700901F780083
:106020008402200000092000000047001000420008
:10603000801F780038F907004F00B100D00220001F
:1060400000004700801F7800ED1307002F00B1000B
:10605000E008200000004700100078006D004000BC
:10606000801F78000009200000004700901F780082
:1060700018F907004F00B10030032000000047006E
:10608000801F7800DE1307002F00B100E008200019
:1060900000004700100078007A004000801F780060
:1060A0000009200000004700901F780009F9070050
:1060B0004F00B1009003200000004700801F7800CF
:1060C000CF1307002F00B10074022000E008200069
:1060D0000000470010004200801F780000092000E7
:1060E00000004700901F7800FAF807004F00B10049
:1060F000F003200000004700801F7800C013070055
:106100002F00B10044032000E008200000004700F9
:1061100010004200801F78000009200000004700A6
:10612000901F7800EBF807004F00B10050042000EA
:1061300000004700801F7800B11307002F00B10056
:1061400000002000F076880054708000600052004B
:10615000160032008075800091758000927080007A
:10616000A37080008E1A0700D4708000E570800054
:106170000401780085017800161B07000000E0008C
:1061800002003C0000002000010037001000200049
:106190000000E00005003A00A468800060005200A2
:1061A00002003200C8310400000000009468800042
:1061B0006000520076003A00707180006B00400071
:1061C000801F780080072000801F7800C1F807003A
:1061D0004F00B100546B80006300520009003D0085
:1061E0006A0DF800B0972F00801F780040E620006D
:1061F000801F78005D1307006F00B10010310400AC
:10620000000000006A0DF80020992F00801F780020
:1062100040E62000801F7800541307006F00B10093
:1062200040E62000801F7800751307002F00B100A2
:10623000707180006B004000801F7800600E2000AD
:10624000801F7800A3F807004F00B10080D5200020
:10625000104078000080FB00801F7800540DF8008B
:10626000560DF800F0992F00801F780040E62000BE
:10627000801F78003D130700AF00B10040E620000A
:10628000801F78005E1307002F00B100707180003E
:1062900078004000801F7800600E2000801F78008A
:1062A0008CF807004F00B10090D520001040780016
:1062B0000080FB00801F78005A0DF8005C0DF8008C
:1062C000D09A2F00801F780040E62000801F7800C1
:1062D00026130700AF00B10040E62000801F7800C1
:1062E000471307002F00B100707180007800400054
:1062F000801F7800E0062000801F780075F80700F6
:106300004F00B100606B8000716B800002002000C4
:1063100003002000AF1A07000000E00002003C006C
:106320000000200001003700100020000000E00005
:106330000E0032006C0DF8006E0DF800B09B2F00BF
:10634000801F780040E62000801F780007130700B8
:106350008F00B10040E62000801F7800281307005E
:106360002F00B100C031040000000000B004200084
:1063700000004700801F7800211307002F00B100A4
:106380001000200000778800323204000000000076
:10639000047780006100520032003A007071800082
:1063A0006B004000801F780080072000801F78006D
:1063B00048F807004F00B10000052000000047002A
:1063C000801F78000E1307002F00B100707180004D
:1063D0006B004000801F7800600E2000801F780056
:1063E0003CF807004F00B1005005200000004700B6
:1063F000801F7800021307002F00B1007071800029
:1064000078004000801F7800600E2000801F780018
:1064100030F807004F00B100B00520000000470031
:10642000801F7800F61207002F00B1007071800005
:1064300078004000801F7800E0062000801F780070
:1064400024F807004F00B1001006200000004700AC
:10645000801F7800EA1207002F00B1000000200022
:106460000077880000002000408798000403200087
:1064700040DE200010A2B900900D2000040340006F
:10648000E4E22000E0082000000047001408530068
:10649000C0082000008F9800106B8000216B8000E6
:1064A0002819070060879800C406200004025000E5
:1064B000648798006000520004003D0084162000AC
:1064C000C00820000000470010084200C00820005B
:1064D000000047001002780062002000110009004F
:1064E0000202D80060879800640020000480B90090
:1064F000608798007602200084082000040247008C
:106500001400130090003D00C00820000000470068
:10651000100078006603400066879800841620000B
:10652000040053000400350084162000C008200039
:106530000000470010081200C008200000004700BB
:1065400010027800E2012000110009000202D800C8
:1065500001007800600250000A00320060DA20007A
:10656000860820000603470016024000D0022000E3
:10657000004A780010002000160B4000A0330400F1
:1065800000000000A4052000C00820000000470013
:1065900010007800110009000400D8000100780004
:1065A0006002500012003200C008200000004700C6
:1065B000901F7800009D2F00801F780064DA200073
:1065C000800820000000470010004200801F780073
:1065D000661207006F00B100340020008008200020
:1065E000000047001008420098330400000000003B
:1065F00060DA2000860820000603470016024000EB
:10660000D0022000004A780010002000160B400045
:106610004833040000000000240920000402470061
:10662000E0042000004A78007633040000000000F7
:10663000240920000402470050042000004A78008A
:106640007633040000000000240920000402470003
:1066500030052000004A7800763304000000000076
:10666000240920000402470070052000004A780039
:1066700076330400000000002409200004024700D3
:10668000F0032000004A7800763304000000000088
:10669000C00820000000470010027800600052008F
:1066A000DDFF3200A6052000C408200004024700D8
:1066B00014001300DEFF3200460B2000C408200047
:1066C0000402470014001300DFFF3200C00820005E
:1066D0000000470010037800E4102000040053007D
:1066E000DFFF32003C3304000000000060DA2000CD
:1066F00086082000060347001602400020092000FB
:1067000000004700104A780006007800100078006A
:10671000610240004487980060DA200004024000D3
:10672000D0022000004A780010002000160B400024
:10673000C4002000C00820000000470010084200EC
:106740007A3204000000000064DA20008008200093
:10675000000047001002420000002000004A7800BC
:10676000106B8000216B800076180700408798002E
:1067700064002000110009000400D8000100780026
:10678000408798006002500005003A0084DC200039
:1067900000002000004A7800D6330400000000000A
:1067A00094DC200000002000004A7800000920004E
:1067B0000000470010027800800820000000470019
:1067C000100352004687980094DC2000000020004F
:1067D000004A7800E0082000000047001000780020
:1067E0006A004000801F7800861F78004AF7070083
:1067F0004F00B10090DA2000801F7800509D2F00DC
:10680000801F780040E62000801F7800D711070025
:106810006F00B10040E62000801F7800F8110700EB
:106820002F00B100F470800005718000126B8000B1
:10683000236B800004007800850078006A19070047
:106840004018070060879800E0082000000047001B
:10685000901F7800A40520000009200000004700D8
:1068600010004200801F78002BF707004F00B10096
:10687000C0082000000047001002780060005200AD
:106880000D003A00507080000000E0000A00320065
:10689000620DF800640DF800A09D2F00801F7800A5
:1068A00040E62000801F7800B01107008F00B10083
:1068B0006C34040000000000620DF800640DF80064
:1068C000609E2F00801F780040E62000801F780027
:1068D000A61107008F00B10040E62000801F78005D
:1068E000C71107002F00B100EF11070050708000A2
:1068F0000000E0002B013200107780000000E00073
:1069000001003200A2F80700C00820000000470084
:10691000100278006000520004003D008416200040
:10692000C00820000000470010084200460B20006D
:10693000C4082000040247001400130004003400BF
:1069400084162000C0082000000047001008120034
:106950000000200050879800A00820000000470099
:10696000100278007F0052000C003D0064DA200025
:10697000A008200000004700100242000002200092
:10698000004A780014002000A00820000000470002
:1069900010084200AC3404000000000064DA20005B
:1069A000A008200000004700100242000000200064
:1069B000004A780006FA2F00C408200004024700AD
:1069C000140013002400340006062000C408200030
:1069D00004024700140013001F003D00A40520001E
:1069E000C00820000000470010024200248F9800D9
:1069F0005487980062002000110009000202D800AC
:106A00000100780040879800640020002E889000E4
:106A1000110009000400D80050879800600250005F
:106A20000B003500A008200000004700100278008D
:106A30007F00520006003D0064DA2000A00820001C
:106A4000000047001002420080042000004A780045
:106A5000303504000000000000002000408798004E
:106A60008008200000004700100278000009200084
:106A7000000047001002420044879800E008200010
:106A8000000047001000780074004000801F78006C
:106A9000841F7800A0F607004F00B100C008200056
:106AA0000000470010027800600052000A003A001F
:106AB00060DA2000801F7800D09E2F00801F7800B1
:106AC00040E62000801F7800281107006F00B10009
:106AD000A835040000000000C008200000004700A6
:106AE00010027800670052000700350096FF2F0063
:106AF000C4082000040247001400130002003C00F8
:106B0000983504000000000060DA2000801F780043
:106B1000C09F2F00801F780040E62000801F780073
:106B2000121107006F00B100A8350400000000003A
:106B300060DA2000801F780010A02F00801F7800EE
:106B400040E62000801F7800081107006F00B100A8
:106B500040E62000801F7800291107002F00B100B7
:106B6000C0082000000047001002780060005200BA
:106B700024003A00E00820000000470010007800E0
:106B80006A004000801F78000009200000004700D4
:106B90001000780067005000801F78004DF6070055
:106BA0004F00B1006006200000004700801F780001
:106BB000131107002F00B100E0082000000047007B
:106BC000100078006A004000801F7800F40B20005D
:106BD000000920000000470010004200801F7800DC
:106BE0003CF607004F00B10090062000000047006F
:106BF000801F7800021107002F00B100CE3604007C
:106C000000000000C00820000000470010027800CB
:106C1000600052002E003D00E00820000000470008
:106C2000100078006A004000801F780000092000F2
:106C3000000047001000780067005000801F7800B7
:106C400024F607004F00B10066FA2F00C4082000A8
:106C5000040247001400130007003D00C006200096
:106C600000004700801F7800E51007002F00B100EA
:106C70004636040000000000F00620000000470037
:106C8000801F7800DE1007002F00B100E008200010
:106C900000004700100078006A004000801F780064
:106CA000F40B200000092000000047001000420003
:106CB000801F780007F607004F00B1002007200072
:106CC00000004700801F7800CD1007002F00B100A2
:106CD000C008200000004700100278006000520049
:106CE0002E003400E008200000004700100078006B
:106CF0006A004000801F7800F40B2000000920008B
:106D00000000470010004200801F7800F1F50700E6
:106D10004F00B100A6052000C4082000040247006F
:106D20001400130007003400500720000000470043
:106D3000801F7800B21007002F00B100AC360400AD
:106D4000000000008007200000004700801F78003E
:106D5000AB1007002F00B100E00820000000470042
:106D6000100078006A004000801F780000092000B1
:106D7000000047001000780067005000801F780076
:106D8000D4F507004F00B100B00720000000470015
:106D9000801F78009A1007002F00B1007638040099
:106DA00000000000A06B80000000E000CF00320077
:106DB000206F80006B024000748798000000200064
:106DC000A06B8800841F7800B0002000801F78002E
:106DD00045F807004F00B1000000200040879800F0
:106DE0008008200000004700100278006C0052006C
:106DF0003E003D00800820000000470010007800A1
:106E00004202DD0060D72000040040006203400021
:106E1000240320001600120006003100340920006F
:106E20000402470000092000004A78004C370400A3
:106E300000000000800820000000470010007800DB
:106E40004202DD0060D720000400400062024000E2
:106E5000100320001402100072002000110009002D
:106E60000282D800040920000002420030092000FC
:106E700000004700044878000443780064092000BB
:106E80000440530004003600340920000402470087
:106E900060092000004A7800300920000000470007
:106EA000104078000080FB00801F780060A02F0059
:106EB000801F780040E62000801F78002B1007001C
:106EC0006F00B10040E62000801F78004C100700E2
:106ED0002F00B100140020008008200000004700AF
:106EE00010084200F036040000000000E008200016
:106EF000000047001000780061004000801F78000B
:106F0000B0002000801F7800F7F707004F00B100A5
:106F10000000200040879800800820000000470003
:106F2000100278006C00520034003D008008200000
:106F300000004700100078004202DD0060D720000A
:106F400004004000620340001403200016001200F9
:106F500006003900340920000402470060092000BF
:106F6000004A7800D43704000000000080082000A8
:106F700000004700100078004202DD0060D72000CA
:106F800004004000620040001002780072002000FF
:106F9000110009000282D8000609200034092000EF
:106FA00004024700004A4300300920000000470067
:106FB000104078000080FB00801F780030A12F0077
:106FC000801F780040E62000801F7800E70F070050
:106FD0006F00B10040E62000801F78000810070015
:106FE0002F00B1001400200080082000000047009E
:106FF000100842008C37040000000000E008200068
:10700000000047001000780062004000801F7800F8
:10701000B0002000801F7800B3F707004F00B100D8
:10702000E007200000004700801F7800F40F0700F1
:107030002F00B10000002000408798008008200049
:1070400000004700100278006C00520027003D004D
:107050008008200000004700100078004202DD0098
:1070600060D7200004004000100278006000520049
:107070001300320080082000000047001000780054
:107080004202DD0060D7200004004000901F78001D
:1070900000A22F00801F780040E62000801F7800AB
:1070A000B20F07006F00B10040E62000801F78009B
:1070B000D30F07002F00B1006A3804000000000061
:1070C0003008200000004700801F7800CC0F070028
:1070D0002F00B100140020008008200000004700AD
:1070E000100842001E380400000000000080FA0072
:1070F000000006000600FA0060004700D1AA2F0039
:10710000040009003158780060004700801F7800B3
:10711000BB0F07002F00B1000080FA00000006003E
:107120000600FA0080012000000F7800226F800026
:10713000300020000090B900F001400023079800C3
:1071400068015700120078001007980012801100A3
:1071500007003400C00D2000000F780064004700D5
:107160001000780061014000620047001008110023
:107170006200470010017800D00020000090B900A4
:10718000100798007A00400010079800801F7800D0
:1071900060004700901F780020AB2F00801F780010
:1071A00040E62000801F7800700F07008F00B100BC
:1071B00040E62000801F7800910F07002F00B100EB
:1071C0000080FA00000006004A00FA006000470054
:1071D00041D52F00030009003158780064004700B2
:1071E00081D52F000300090031587800680047005E
:1071F000C1D52F0003000900315878006C0047000A
:1072000001D62F00030009003158780070004700B4
:1072100041D62F000600090031587800770047005A
:10722000B1D62F0008000900315878000002200074
:107230000000470041D72F000300090031587800B3
:10724000400220000000470081D72F000400090001
:10725000315878009002200000004700D1D72F005D
:107260000300090031587800D002200000004700D8
:1072700011D82F0005000900315878003003200094
:107280000000470071D82F00030009003158780032
:107290007003200000004700B1D82F000300090050
:1072A00031587800B003200000004700F1D82F00CB
:1072B0000200090031587800E00320000000470078
:1072C00021D92F0004000900315878003004200033
:1072D0000000470071D92F000100090031587800E3
:1072E000500420000000470091D92F00040009003D
:1072F0003158780068005700901F780088FF070019
:107300002F00B100680057001001780041EE200006
:107310001100510006003A00A0042000801F7800F0
:10732000520F07002F00B1009A390400000000003E
:107330005D0F0700823C040000000000D60EF8003C
:10734000D80EF800F0AB2F00801F780040E6200038
:10735000801F7800050F07008F00B1006E3D04000C
:1073600000000000B00EF800B20EF80070AD2F0063
:10737000801F780040E62000801F7800FB0E070089
:107380008F00B1006E3D0400000000000E0EF800FA
:10739000100EF800F0AE2F00801F780040E62000AD
:1073A000801F7800F10E07008F00B1006E3D0400D1
:1073B000000000000C0EF80070B02F00801F780055
:1073C00040E62000801F7800E80E07006F00B10043
:1073D0006E3D040000000000D20EF800D40EF8004C
:1073E000D0B12F00801F780040E62000801F780079
:1073F000DE0E07008F00B1006E3D040000000000AB
:10740000420EF800440EF80050B32F00801F7800A1
:1074100040E62000801F7800D40E07008F00B100E6
:107420006E3D040000000000E60EF800E80EF800D3
:10743000D0B42F00801F780040E62000801F780025
:10744000CA0E07008F00B1006E3D0400000000006E
:107450003E0EF800400EF80050B62F00801F780056
:1074600040E62000801F7800C00E07008F00B100AA
:107470006E3D040000000000EA0EF800EC0EF8007B
:10748000D0B72F00801F780040E62000801F7800D2
:10749000B60E07008F00B1006E3D04000000000032
:1074A000EE0EF800F00EF80050B92F00801F7800A3
:1074B00040E62000801F7800AC0E07008F00B1006E
:1074C0006E3D0400000000004A0EF8004C0EF8006B
:1074D000D0BA2F00801F780040E62000801F78007F
:1074E000A20E07008F00B1006E3D040000000000F6
:1074F000460EF800480EF80050BC2F00801F7800A0
:1075000040E62000801F7800980E07008F00B10031
:107510006E3D040000000000360EF800380EF80042
:10752000D0BD2F00801F780040E62000801F78002B
:107530008E0E07008F00B1006E3D040000000000B9
:107540003A0EF8003C0EF80050BF2F00801F780064
:1075500040E62000801F7800840E07008F00B100F5
:107560006E3D040000000000F20EF800F40EF8007A
:10757000D0C02F00801F780040E62000801F7800D8
:107580007A0E07008F00B1006E3D0400000000007D
:10759000CE0EF800D00EF80050C22F00801F7800E9
:1075A00040E62000801F7800700E07008F00B100B9
:1075B0006E3D040000000000E17280006180500018
:1075C00004003A006000470080007800EE3A0400B2
:1075D000000000006400470080007800010078008F
:1075E000801F7800D0C32F00801F780040E6200065
:1075F000801F78005D0E07006F00B1006E3D040033
:1076000000000000017380006180500004003A0017
:107610006800470080007800143B04000000000070
:107620006C0047008000780001007800801F78001F
:1076300030C52F00801F780040E62000801F7800B2
:107640004A0E07006F00B1006E3D0400000000000C
:10765000707580000000E0000400320070004700F8
:10766000800078003A3B04000000000077004700EB
:107670008000780001007800801F780090C62F00FD
:10768000801F780040E62000801F7800370E07003A
:107690006F00B1006E3D040000000000300DF800E6
:1076A000C0C72F00801F780040E62000801F7800B0
:1076B0002E0E07006F00B1006E3D040000000000B8
:1076C000206F80000000E000050032000002200072
:1076D0000000470080007800763B040000000000B6
:1076E0004002200000004700800078000100780080
:1076F000801F780020C92F00801F780040E62000FE
:10770000801F7800190E07006F00B1006E3D040065
:1077100000000000F60EF80050CA2F00801F78000D
:1077200040E62000801F7800100E07006F00B100B7
:107730006E3D040000000000507080000000E0007A
:107740000500320090022000000047008000780011
:10775000B23B040000000000D002200000004700FF
:107760008000780001007800801F7800B0CB2F00E7
:10777000801F780040E62000801F7800FB0D070086
:107780006F00B1006E3D040000000000F80EF8002C
:10779000FA0EF800E0CC2F00801F780040E62000B1
:1077A000801F7800F10D07008F00B1006E3D0400CE
:1077B00000000000FC0EF800FE0EF80040CE2F0086
:1077C000801F780040E62000801F7800E70D07004A
:1077D0008F00B1006E3D040000000000AC0EF80008
:1077E000C0CF2F00801F780040E62000801F780067
:1077F000DE0D07006F00B1006E3D040000000000C8
:10780000A07580000000E000050032003003200079
:107810000000470080007800163C040000000000D3
:10782000700320000000470080007800010078000D
:10783000801F780020D12F00801F780040E62000B4
:10784000801F7800C90D07006F00B1006E3D040075
:1078500000000000107780000000E000050032000A
:10786000B00320000000470080007800403C040086
:1078700000000000E00320000000470080007800C6
:1078800001007800801F780080D22F00801F7800D0
:1078900040E62000801F7800B40D07006F00B100A3
:1078A0006E3D040000000000007880000000E00051
:1078B00005003200300420000000470080007800FE
:1078C0006A3C040000000000500420000000470053
:1078D0008000780001007800801F7800E0D32F003E
:1078E000801F780040E62000801F78009F0D070071
:1078F0006F00B1006E3D0400000000006E3D04000A
:107900000000000068005700900078006080500080
:107910008AFE3200680057009000780061805000B5
:1079200090FE32006800570090007800628050009E
:1079300096FE320068005700900078006380500087
:107940009CFE320068005700900078006480500070
:10795000A1FE32006800570090007800658050005A
:10796000A7FE320068005700900078006680500043
:10797000ADFE32006800570090007800678050002C
:10798000B3FE320068005700900078006880500015
:10799000B9FE3200680057009000780069805000FE
:1079A000BFFE320068005700900078006A805000E7
:1079B000C5FE320068005700900078006B805000D0
:1079C000CBFE320068005700900078006C805000B9
:1079D000D1FE320068005700900078006D805000A2
:1079E000D7FE320068005700900078006E8050008B
:1079F000DDFE320068005700900078006F80500074
:107A0000E3FE32006800570090007800708050005C
:107A1000E9FE320068005700900078007180500045
:107A2000F8FE320068005700900078007280500025
:107A300007FF320068005700900078007380500004
:107A400016FF3200680057009000780074805000E4
:107A50001BFF3200680057009000780075805000CE
:107A60002CFF3200680057009000780076805000AC
:107A700031FF320068005700900078007780500096
:107A800042FF320068005700900078007880500074
:107A900048FF32006800570090007800798050005D
:107AA0004EFF320068005700900078007A80500046
:107AB00053FF320068005700900078007B80500030
:107AC00064FF320068005700900078007C8050000E
:107AD00075FF32007E3C04000000000040E62000FC
:107AE000801F7800460D07002F00B1000080FA00CB
:107AF000000006000200FA0000002000000F7800DD
:107B000060004700900078007C80500009003C0035
:107B100060004700901F7800ABFD07002F00B10008
:107B2000110020006000470010884000803D0400E4
:107B3000000000000080FA00000006000000FA00CB
:107B4000A2072000E80057001100110007003E00C6
:107B500012062000E8005700110011000300390050
:107B6000F1FD2F0068005700108860004EB89700A4
:107B70000080FA00000006000200FA000000200069
:107B8000000F780068005700900078006000470000
:107B9000108040009040780060C050001300320018
:107BA000711080000020200000806000C900DE000D
:107BB0000100E00002003200D03D0400000000009F
:107BC00068005700100078006001470092004000F4
:107BD000114078000080FB00801088001000200019
:107BE00012094000C23D0400000000000080FA00BD
:107BF000000006000C00FA0020002000000F7800B2
:107C000000002000300798006800570090007800BE
:107C100066004700108040009040780060C050002F
:107C20000C00320068005700100078006601470021
:107C300012004000904078008180FB006000470007
:107C4000108868001000200012094000043E040063
:107C50000000000060004700901F7800E0D92F006E
:107C6000801F780062004700801F7800BF0C07006B
:107C70006F00B1000000200030079800E2004700CC
:107C800066004700108040009040780060C05000BF
:107C900011003200E20047006600470050079800DC
:107CA0001080400040079800104078000080FB00E2
:107CB000801F7800A1FF07002F00B100CE009000C8
:107CC00080487800110020005E009000108840007D
:107CD0003E3E04000000000062004700801F780064
:107CE00068005700901F780030DA2F00801F78005E
:107CF00060DA2000801F78009C0C07008F00B10024
:107D000060DA2000801F78009BFF07002F00B10081
:107D10000080FA00000006002A00FA006000470018
:107D200001DB2F000E000900315878006F0047007A
:107D3000F1DB2F0001000900315878007100470085
:107D400011DC2F0001000900315878007300470052
:107D500031DC2F0016000900315878006000470020
:107D6000801F7800A3FF07002F00B1004EB89700D6
:107D70000000E000060032006F004700801F78001E
:107D80009CFF07002F00B100D03E0400000000005F
:107D900071004700801F780096FF07002F00B10098
:107DA00073004700801F780092FF07002F00B1008A
:107DB0000080FA00000006000000FA00F1EF2F003A
:107DC00060082000108860004EB89700C800DD00F1
:107DD000E008200090806800001020008080600093
:107DE000E008200010886800D1FF2F0080212000CB
:107DF000108860000080FA00000006000000FA0011
:107E0000EA00570011007800103B880062804000B3
:107E10009040780020032000014878006C00570053
:107E200010007800003B88000C0007000080FA007A
:107E3000000006000000FA0040042400801F7800C3
:107E40006A005700B01F7800A01F7800EBFF070002
:107E50006F00B1000080FA00000006000000FA0088
:107E60000500FC005C0520003C3B8800AC0A2000BB
:107E70003C3B880061E7A800000000000000000013
:107E80000080FA00000006000000FA006A005700B7
:107E9000B01F7800A01F7800E6FF07004F00B10078
:107EA000013B80000000280000806000CF00DE0061
:107EB0000100E00002003200503F0400000000001A
:107EC000EA00570011007800C0008800628040007E
:107ED0009040780020032000014878006C00570093
:107EE00010007800B00088000B0EBB00400024009A
:107EF000003B8800D9FF0700F1FF2B00007620002F
:107F0000108860000080FA00000006000A00FA00F5
:107F10006A00570010007800100798004EB99700CB
:107F200032007800A20078002007980031079800FE
:107F300000002000000F7800600047001002780069
:107F40006C015700120052001D003D001E00900001
:107F5000901F78006400470040079800B01F780029
:107F6000A01F7800C8FF07006F00B10022002000AA
:107F7000620047001008410022002000CF91DE007F
:107F80004E0090001018410010904900023B800004
:107F900000002800000061004F01DE000200E00048
:107FA00002003200C63F0400000000001200200062
:107FB00060004700100841009C3F040000000000E2
:107FC0006C005700100078004100DD004EB99700AA
:107FD000CF80DE0012194000129148000080FA00A4
:107FE000000006000000FA0092032000E80057009D
:107FF0001100110008003E0002032000E8005700B5
:1080000011001100040039001000200080407800A9
:1080100010400400000000000000200080407800B4
:108020008180FB00010078000080FA00000006005B
:108030000600FA00680057001042780060405200C5
:1080400072003D0068025700144078000000FB00F9
:1080500060001000004A780000437800E406200029
:10806000044053003A00350068005700200798008C
:10807000104278000402FB00420620000402FB00CC
:10808000110009000202D800720040004202DD0027
:10809000A0DD2F000400400030027800A00278002C
:1080A0002E009000040798001507980010427800F1
:1080B0000402FB0042062000110009000202D80061
:1080C00001007800A4002000110009000400D8007D
:1080D000690040004202DD00A0DD2F0004004000E6
:1080E00030027800A00278000E0090009E00900000
:1080F0000401780085017800A91207002E02900083
:1081000000079800110798000400780010427800DA
:108110000402FB00A2002000110009000202D800A6
:10812000010078004202DD00A0DD2F0004004000C5
:1081300030027800A00278000E0090009E009000AF
:108140000401780085017800951207009C00370033
:1081500068005700104278006A4052002200340044
:108160006800570000079800104278000402FB00E6
:10817000A20020000402FB00110009000202D80046
:10818000690040004202DD00A0DD2F000400400035
:1081900030027800A00278000E00900004079800DA
:1081A00015079800104278000402FB00A20020008E
:1081B000110009000202D800010078004202DD002F
:1081C000A0DD2F000400400030027800A0027800FB
:1081D0000E0090009E009000040178008501780058
:1081E0006F120700760037006800570010407800D3
:1081F0000000FB004202DD00A0DD2F000402400071
:1082000034007800A40078006D0037006800570043
:1082100010437800E4062000044053003A00350083
:108220006800570020079800104278000402FB0005
:10823000420620000402FB00110009000202D800DF
:10824000720040004202DD00E0E02F000400400028
:1082500030027800A00278002E00900004079800F9
:1082600015079800104278000402FB004206200027
:10827000110009000202D80001007800A4002000CB
:10828000110009000400D800690040004202DD002E
:10829000E0E02F000400400030027800A0027800E7
:1082A0000E0090009E009000040178008501780087
:1082B0003B1207002E02900000079800110798005B
:1082C00004007800104278000402FB00A2002000A5
:1082D000110009000202D800010078004202DD000E
:1082E000E0E02F000400400030027800A002780097
:1082F0000E0090009E009000040178008501780037
:10830000271207002E00370068005700104278003F
:108310006A405200220034006800570000079800AD
:10832000104278000402FB00A20020000402FB00BF
:10833000110009000202D800690040004202DD007D
:10834000E0E02F000400400030027800A002780036
:108350000E0090000407980015079800104278005E
:108360000402FB00A2002000110009000202D80054
:10837000010078004202DD00E0E02F000400400030
:1083800030027800A00278000E0090009E0090005D
:108390000401780085017800011207000800370009
:1083A00068005700104078000000FB004202DD002A
:1083B000E0E02F000402400034007800A4007800C0
:1083C0000080FA00000006000600FA00680057006E
:1083D00010437800E4062000044053003E003900BA
:1083E0006800570020079800104278000482FB00C4
:1083F000420620000402FB00110009000202D8001E
:10840000720040004202DD00A0DD2F0004024000A7
:1084100034007800A40078000200200003F023005C
:10842000DF1107002E029000000798001107980046
:1084300004007800104278000482FB00420620000D
:10844000110009000202D80001007800A4002000F9
:10845000110009000400D800690040004202DD005C
:10846000A0DD2F000400400030027800A002780058
:108470000E0090009E0090000401780085017800B5
:10848000C71107002E0290000007980011079800FE
:1084900004007800104278000482FB00A200200053
:1084A000110009000202D800010078004202DD003C
:1084B000A0DD2F000400400030027800A002780008
:1084C0000E0090009E009000040178008501780065
:1084D000B3110700350037006800570010427800DC
:1084E0006A405200260036006800570000079800D6
:1084F000104278000482FB00A20020000402FB006E
:10850000110009000202D800690040004202DD00AB
:10851000A0DD2F000402400034007800A4007800A1
:108520000200200003F023009D1107000E029000BE
:1085300000079800110798000400780010427800A6
:108540000482FB00A2002000110009000202D800F2
:10855000010078004202DD00A0DD2F000400400091
:1085600030027800A00278000E0090009E0090007B
:108570000401780085017800891107000B0037009D
:1085800068005700104078000080FB004202DD00C8
:10859000A0DD2F000402400034007800A400780021
:1085A0000200200003F023007D1107000080FA0084
:1085B000000006000000FA00020007004243040029
:1085C000000000000001BE00190007000470A700B1
:1085D00003F0A10003F8A30013003A006509B100FD
:1085E00010003200090035006928E1000200350062
:1085F00001002800000005000000400081804800C4
:108600008502E900FCFF3A0000000600F88F4200F6
:10861000050035008100D1000080D3008502E8000C
:10862000FCFF3A00000006008000EB00000005009F
:10863000C70ADE00F107B200F50FB20008003200F1
:10864000E1CF4200020032000170A00024000500CA
:10865000810F70000100320004080500440005008D
:10866000810F700002003A00140005008502E90045
:108670000000400081C04800FCFF3B000170A000EA
:10868000240005000080FA00000006000000FA0047
:10869000020007009A430400000000000400E0000C
:1086A00002003A001000070000000600811F780059
:1086B0000100E00002003D0060001000E0801800B2
:1086C0000300E00002003D0060011100E08119009C
:1086D000050007004F00E00002003B0060001000B2
:1086E000E080180000000600020007000400BE0041
:1086F000000006006022B800060220000000D00042
:108700008180D2000482D2008582D2000000A000C5
:108710000202520083825A0003003B000202420020
:1087200083824A000000A1000603E900F3FF3A003B
:10873000000006000080FA00000006000000FA00B9
:1087400002000700EC430400000000000400E00009
:1087500002003A001000070000000600839F680036
:108760000100E00002003D0060001000E080180001
:108770000300E00002003D0060011100E0811900EB
:10878000050007004F00E00002003B006000100001
:10879000E0801800000006006022B80006022000F9
:1087A0000000D0008180D2000482D2008582D200F5
:1087B0000000A0000202520083825A0003003B0026
:1087C0000202420083824A000000A1000603E90081
:1087D000F3FF3A00000006000080FA0000000600E7
:1087E0002800FA0060004700C1ED2F0006000900D4
:1087F0003158780000002000000F98000000200091
:10880000700798003EBB9700140020006A005700D4
:1088100010084200164278006A00470004487800B9
:108820000404E000CE0932006A00470010437800DB
:1088300054022000044053000B0032006A0247003B
:108840004EB89700144878001400200068005700C4
:108850001008420014002000700047001008420079
:10886000024404000000000000002000600798009F
:1088700000002000700798009044040000000000F1
:10888000840020006E0047001008720014002000D1
:108890006A00570010084200C644040000000000AF
:1088A000140020006E004700100872001400200021
:1088B0006A00570010084200C6440400000000008F
:1088C000240020006E0047001008720014002000F1
:1088D0006A00570010084200C6440400000000006F
:1088E000048020006E004700100872001400200071
:1088F0006A00570010084200C6440400000000004F
:10890000440020006E004700100872001400200090
:108910006A00570010084200C6440400000000002E
:108920003EB8970010437800D40220000440530062
:10893000D3FF32003EB897001043780004022000B5
:1089400004405300D6FF32003EB897001043780031
:10895000B402200004405300D9FF32003EB8970013
:10896000104378003402200004405300DCFF320042
:108970003EB89700104378000403200004405300E1
:10898000DFFF3200CA440400000000003C44040041
:10899000000000006E0047001000780062026000D6
:1089A00003003200E4FF2F006E0047001008620051
:1089B0006E0047001000780068026000030032007B
:1089C000B4FF2F006E004700100862003EB8970009
:1089D000104078000080FB00801F780081FD0700B8
:1089E0002F00B1000000E00019003200000020005C
:1089F000600798006C03470016027800A000200072
:108A000000A2B9003EB89700104078000080FB003B
:108A10000002420000032000000B52006A005700D1
:108A2000100078006100400030BF9F0010407800C7
:108A30000080FB00801F78006AFD07002F00B10056
:108A40000000E000EBFF3A00464504000000000093
:108A50003EB8970010437800A40220000440530061
:108A60000A003A002EBB97002EBA97002000200083
:108A7000140A1000160278001400780060079800AD
:108A8000140020006A005700100842003EB897000A
:108A900010437800E4022000044053002F003A0005
:108AA0006A005700100078006100400030BF9F004E
:108AB00010437800A4022000044053000C003A0048
:108AC0002EBB97002EBA970020002000140A100039
:108AD0001602780014007800400798001400200067
:108AE0006A00570010084200AA4504000000000078
:108AF00000002000400798003EB897001040780022
:108B00000080FB00801F780036FD07002F00B100B9
:108B10000000E0000F0032006803470016027800F2
:108B2000A000200000A2B9003EB8970010407800D5
:108B30000080FB000002420000032000000B5200F6
:108B4000140020006A005700100842007C45040011
:108B500000000000B84504000000000000002000F4
:108B600040079800040021006E00470010087200C2
:108B70003EBB9700140020006A0057001008420016
:108B8000164278006A004700044878003E47040017
:108B9000000000000E089000F208370004012000D9
:108BA0006E00470010087200B84504000000000085
:108BB000044020006E00470010087200E0470400E7
:108BC00000000000040220006E0047001008720040
:108BD000041020006E00470010087200E0470400F7
:108BE00000000000042020006E0047001008720002
:108BF000E047040000000000040420006E0047006D
:108C000010087200E047040000000000E047040084
:108C100000000000040220006E00470010087200EF
:108C2000040820006E00470010087200E0470400AE
:108C300000000000F8044700090478002EBB9700EC
:108C40002EBA970020002000140A100016007800A9
:108C5000100C7800190278006000520003003A00FE
:108C60007802470060004700000A7800780047005B
:108C70006202400000002000000A780078034700EC
:108C80006202430016007800140240001404E00061
:108C900006003200780047006202400014007800AD
:108CA000610A40003E460400000000004E009000B3
:108CB0000000E0000B003200780047006203400033
:108CC00068004700100278001600520005003100CD
:108CD00078004700620240006800470010007800FA
:108CE000000A780078004700620340006C004700EB
:108CF0001002780016005200070036007800470086
:108D000062004000100278006C004700100812005A
:108D1000904604000000000000002000600798005A
:108D20006E004700100078006802600011003A00F1
:108D30006E039000140020006C0047001008120021
:108D40000600E0000B0032004EBA9700000220003F
:108D5000004A780014002000680057001008420004
:108D600014002000700047001008420098460400DC
:108D700000000000780047006203400016027800FF
:108D800016007800610B50000400E0000F00320074
:108D90007800470000037800100278004EB8970072
:108DA00014487800140020006800570010084200A2
:108DB00016007800610B400014002000700047008E
:108DC00010084200BA460400000000006E00470090
:108DD0001000780068026000110032006E039000FD
:108DE000140020006C004700100812000600E0008C
:108DF0000B0032004EBA970000022000004A7800B3
:108E000014002000680057001008420014002000E1
:108E10007000470010084200EE4604000000000009
:108E200002440400000000002EBB97002EBA9700F9
:108E300020002000140A100016007800104278006C
:108E40006A00470004487800780247006A0047003B
:108E5000000A78006202420010002000000A780038
:108E60005646040000000000040C20006E0047007D
:108E700010087200E0470400000000006A0047008C
:108E8000104278006040520042FF32006A00470002
:108E900010437800C4042000044053003FFF320018
:108EA0006A00470010437800C406200004405300C5
:108EB0003AFF32006A004700104378006406200041
:108EC000044053003AFF32006A0047001043780024
:108ED00054042000044053003AFF32006A00470067
:108EE00010437800540620000440530038FF32003D
:108EF0006A004700104378007406200004405300C5
:108F000038FF32006A00470010437800F406200062
:108F10000440530038FF32006A00470010437800D5
:108F2000440620000440530038FF32006A00470026
:108F300010437800940620000440530033FF3200B1
:108F40006A004700104378000407200004405300E3
:108F500030FF32006A00470010437800840520008B
:108F6000044053002BFF32006A0047001043780092
:108F7000840720000440530029FF32006A004700A4
:108F800010437800340720000440530029FF3200CA
:108F90006A00470010437800340620000440530064
:108FA000A1FF32006A0047001043780054072000F8
:108FB00004405300ACFF32002447040000000000CE
:108FC0006E0047001002780000702000000262006E
:108FD0005F0532006E00470010027800000021009B
:108FE000000262000200320060002000400798008A
:108FF0002EBB97002EBA970040002000140A1000E4
:109000001602780034007800A4007800100F980051
:10901000210F98000200200003002000B00F07007D
:109020000000E000020035000000200001003700D1
:10903000100020000000E0000800320004002000C2
:10904000050028007200470010186A0010906A009E
:10905000340020006E00470010087200000020005D
:10906000300F98007202470034007800A4007800A6
:109070000200200003002000990F07000000E0001C
:1090800002003A000000200001003700100020001C
:109090000000E000580032007604470072034700E9
:1090A00070012000CF80DE0036027800A602780032
:1090B0000000E900030035008502D1000482D300DE
:1090C000FBFF3700F00F200000026200E0072000E5
:1090D000000C520008007800100078006102500077
:1090E000340F98003000200000A2B900340F98001F
:1090F000A2002000110009000202D800300F9800E1
:109100006002500003003D0014002000760047007C
:10911000100812007800470000179800600F9800B0
:10912000760047001000780060001000801F780073
:10913000BFFB07002F00B1001E099000AE09900090
:10914000970E07006E0A9000001A7800011278004E
:109150000E12900034007800A4007800000278001D
:10916000810278000000200001F82300040178004B
:1091700085017800170F07000000E00002003C00A6
:109180000000200001003700100020000000E00077
:10919000050032001400200076004700100812007D
:1091A000FC4804000000000078024700340078000A
:1091B000A4007800000278008102780000002000FE
:1091C000011224000401780085017800440F070093
:1091D0000000E00002003400000020000100370021
:1091E000100020000000E000030032001400200006
:1091F0007600470010084200760047001002780011
:109200006000520005003C006A0247001000200088
:10921000004A780016490400000000006A02470076
:109220007600470010407800004A78006E00470042
:1092300010027800001020000002620014003A00C2
:109240006E0047001002780000202000000262003B
:109250000D003200C6FF2F007602470014001300F5
:1092600007003500760047001003780068024700C9
:109270001400530002003D004449040000000000B7
:109280004849040000000000EC4D0400000000000C
:109290004E0090000000E000080032006E00470021
:1092A000100278000020200000026200030032005B
:1092B00014002000680047001008120068004700F2
:1092C0001002780068005200050036006A0247006C
:1092D00080002000004A7800784904000000000067
:1092E0006A0247006800470010407800004A780092
:1092F0007202470034007800A400780002002000C9
:1093000003002000F60E07000000E00002003A0013
:109310000000200001003700100020000000E000E5
:10932000700032007600470010007800801F78003F
:109330003FFB07002F00B100000178008101780099
:109340001E089000AE089000A00F0700100F9800B4
:10935000210F98006A004700104078000080FB0051
:1093600060001000801F780031FB07002F00B10063
:1093700000017800810178001E089000AE0890007E
:10938000920F07000017980011179800100F98000F
:10939000210F980087FC07000001EB00A50D0700D6
:1093A000600F9800710F98000E1090009E109000B2
:1093B000821F7800831F78006E099000FE099000DC
:1093C000890E07004F01BE0000027800810278007C
:1093D0000000200001F023000401780085017800DE
:1093E000BF0E07000000E000020034000000200073
:1093F00001003700100020000000E0000A003200E9
:109400007200470030027800A002780000002000BF
:1094100001F023000401780085017800B50E0700F3
:10942000100F9800210F98001E089000AE089000C1
:1094300060FC07006A024700144278000482FB00C7
:10944000610242004223DD0024E42F0006034200B3
:1094500036025000268258000C0039001E08900089
:10946000AE089000D2CC2C00C3DC2300CC0D07004A
:10947000100F9800210F980014002000760047007C
:1094800010084200724A0400000000001E0890000C
:10949000AE08900047FC07006A02470014427800BB
:1094A0000482FB004223DD0024E42F000603420077
:1094B00036025000268258000A0031001E08900033
:1094C000AE0890000200200003122400B40D070033
:1094D000100F9800210F980014002000760047001C
:1094E000100812006E0047001002780000202000D3
:1094F000000262004C0032006E004700100278004B
:10950000008020000002620047003A006800470027
:10951000100278006A00520002003400A00020000F
:109520004007980078004700600F98001E089000E0
:10953000AE0890001FFC07006E0A9000001A780029
:10954000011278007802470034007800240070008F
:109550001C00320078024700A2002000CF91DE00FC
:1095600034007800A40078000002EB0047FC0700FC
:10957000600250006082580012003A00140020007F
:10958000680047001008120078004700600F98003C
:1095900030027800A0027800A200200004007800C9
:1095A00085007800CF91DE000002EB0063FC07002D
:1095B0006E0A9000001A780001127800A24A040096
:1095C000000000006A004700104378000683FB009B
:1095D000680247001400130013003D006A004700B2
:1095E000104278000482FB0068004700100052001F
:1095F000801F78008EFA07002F00B100000178006C
:10960000810178001E089000AE089000EF0E070060
:10961000100F9800210F98006A0247006800470069
:1096200010407800004A7800680047001000780079
:10963000650240006C004700100812004E009000C8
:109640000000E00007003A006E00470010027800BA
:10965000008020000002620002003A00384B040043
:1096600000000000140020006C00470010081200E9
:109670006E004700100078006302600003003200B3
:10968000140020006C004700100812006E00470014
:109690001000780064026000390032006E0047005C
:1096A0001000780062026000140032006E00470073
:1096B000100078006102600004003200D002200037
:1096C000004278006A4B040000000000B002200055
:1096D000004278004EB8970004487800140020003B
:1096E0006800570010084200140020007000470076
:1096F00010084200984B0400000000006E00470074
:109700001000780061026000090032004EBA970034
:1097100000022000004A7800140020006800570072
:10972000100842001400200070004700100842009A
:109730006C00470010027800600052000E003400F8
:109740004EBA970000032000004A78001400200061
:109750006800570010084200140020007000470005
:1097600010084200140020006C004700100812008E
:10977000984B040000000000364C0400000000007C
:109780006E004700100078006802600012003A0086
:109790006C00470010027800600052000E00340098
:1097A0004EBA970000022000004A78001400200002
:1097B00068005700100842001400200070004700A5
:1097C00010084200140020006C004700100812002E
:1097D000C84B0400000000006E0047001000780035
:1097E00062026000140032006E0047001000780032
:1097F0006102600004003200D002200000427800C4
:10980000084C040000000000B00220000042780074
:109810004EB89700044878001400200068005700F4
:109820001008420014002000700047001008420099
:10983000364C0400000000006E0047001000780065
:1098400061026000090032004EBA97000002200059
:10985000004A7800140020006800570010084200F9
:1098600014002000700047001008420078004700F4
:10987000600F98001E089000AE0890004DFB070096
:109880006E0A9000001A7800011278006E089000AD
:1098900030037800A00378006A0047001040780089
:1098A0000080FB004202DD0020E42F0004024000A3
:1098B00034017800A4017800060078008700780061
:1098C0000002EB009DFB0700060320004EBA970044
:1098D000064A4000140020006800570010084200AB
:1098E0001400200070004700100842004E00900055
:1098F0000000E00007003A006E0047001002780008
:10990000008020000002620002003A00104D0400B6
:10991000000000004EBA9700E0022000004A7800E4
:1099200014002000680057001008420014002000B6
:1099300070004700100842006A004700104278009B
:109940000482FB0068004700100812002E489000B7
:109950000004E00021003200780047003003780066
:10996000A00378006A02470014407800614050006C
:10997000004A78000080FB004202DD0020E42F0056
:109980000402400034017800A40178000600780049
:10999000870078000002EB0068FB0700A4002000AD
:1099A00004017800CF91DE000002EB0037FB0700D6
:1099B000060320004EBA9700004A4300140020001E
:1099C0006800570010084200140020007000470093
:1099D00010084200A64C0400000000004E00900059
:1099E0000000E0000E0032004EBA97000003200095
:1099F000004A780014002000680057001008420058
:109A000014002000700047001008420014002000DD
:109A10006800470010081200EE4C0400000000002F
:109A2000040220006E004700100262000B003200AA
:109A30004EBA970050042000004A7800140020001D
:109A40006800570010084200140020007000470012
:109A500010084200404D0400000000004EBA97007C
:109A600050062000004A78001400200068005700CB
:109A70001008420014002000700047001008420047
:109A80007600470010027800600052000E003D0092
:109A90007602470014007800600A10004EBA970062
:109AA000D0022000004A780014002000680057000F
:109AB0001008420014002000700047001008420007
:109AC000764D0400000000004EBA9700B00220005E
:109AD000004A780014002000680057001008420077
:109AE0001400200070004700100842007600470074
:109AF0003017980010027800A20020001100090021
:109B00000202D800060320004EBA9700064A400021
:109B1000680057002017980010007800610040008E
:109B20000017980040BF9F001400200070004700FD
:109B3000600F9800100842003E109000100278005C
:109B4000A2002000110009000202D80001007800E4
:109B5000060320000E129000064A40000E109000EE
:109B6000140020002E109000100842001400200065
:109B70006E089000100842006E0047001000780048
:109B800068026000120032006C004700100278008A
:109B9000600052000E0034004EBA97000002200010
:109BA000004A7800140020006800570010084200A6
:109BB0001400200070004700100842006C004700AD
:109BC000100078006102500064079800F2FF3A002C
:109BD00002440400000000006E00470010027800FC
:109BE000002020000002620077003200760047006B
:109BF000100278006000520005003D00760047002A
:109C00001000780061025000680047001008120040
:109C100078004700600F98001E089000AE08900082
:109C200064FA07006E0A9000001A780001127800AA
:109C30006A02470010002000004A78006A004700CE
:109C4000104278006A405200130032007804470046
:109C50006A004700104078000080FB004202DD00EF
:109C600020E42F000403400038027800A8027800A6
:109C70003600520026805A00020031004C4E04008B
:109C800000000000140020006A0047001048420055
:109C90001E4E0400000000006A00470010427800D9
:109CA0000482FB0068004700100012002017980093
:109CB00040079800780247000400780000179800D9
:109CC00034007800A40078000001EB00590B070075
:109CD000600F9800710F98007202470034007800FE
:109CE000A4007800821F7800831F78006E0990001E
:109CF000FE0990003C0C07004F01BE002E129000A0
:109D0000600F9800710F9800841F7800C8F8070052
:109D10002F00B1006E0A9000FE0A90000401780046
:109D2000850178009E0B07000400200005F0230049
:109D300004017800850178006E0C07001DFA070009
:109D40000E129000001A7800011278004E00900068
:109D50000000E0001C00320078024700A200200052
:109D6000CF91DE0034007800A40078000002EB0000
:109D700046FA0700600250006082580012003A0064
:109D800078004700600F980030027800A002780049
:109D9000A20020000400780085007800CF91DE004A
:109DA0000002EB0065FA07006E0A9000001A7800C6
:109DB000011278001400200068004700100812000B
:109DC000A64E040000000000680047001002780062
:109DD0006C0052000D003C00680047001000780045
:109DE000801F780078F907002F00B1007203470048
:109DF00036027800A6027800040178008501780018
:109E00003C0C0700100F9800210F980072024700C9
:109E100034007800A4007800020020000300200035
:109E20002F0C07000000E00002003A0000002000B4
:109E300001003700100020000000E0004000320068
:109E40001E089000AE089000DAF90700600250008A
:109E5000608258003A003A0076004700100278000D
:109E60006100520036003400760047001000780090
:109E7000801F78006EF807002F00B1000001780005
:109E8000810178001E089000AE089000CF0C0700FA
:109E90000002780081027800F00527009108240074
:109EA0000401780085017800CA0B07000000E0007B
:109EB00002003C00000020000100370010002000DC
:109EC0000000E0000500320094002000760047000A
:109ED00010081200744F04000000000084002000ED
:109EE000760047001008120078004700600F9800C5
:109EF0007600470010007800801F78004CF80700BB
:109F00002F00B10000017800810178001E08900048
:109F1000AE089000AD0C0700A6F907006E0A90008D
:109F2000001A7800011278000000200001002000D3
:109F3000100F9800210F9800DA4F04000000000075
:109F400078004700600F98001E089000AE0890004F
:109F500098F907006E0A9000001A78000112780044
:109F60006E0890000002780034007800A4007800A9
:109F70000001EB00AF0A0700600F9800710F980016
:109F80007202470034007800A4007800821F780035
:109F9000831F78006E099000FE099000920B070065
:109FA0004F01BE00100F9800210F98000000200004
:109FB000300F98006A02470010002000004A780025
:109FC0006A004700104278006A40520013003200D5
:109FD000780447006A004700104078000080FB00CA
:109FE0004202DD0020E42F00040340003802780024
:109FF000A80278003600520026805A000200310084
:10A000000E50040000000000140020006A00470009
:10A0100010484200E04F0400000000006A004700C2
:10A02000104278000482FB006800470010024200E2
:10A0300076004700100242006C0047001008120032
:10A040006E004700100278000080200000026200CD
:10A0500005003A004E0090000000E00002003A00C7
:10A060003A50040000000000140020006C0047007B
:10A07000100812006E0047001000780063026000B4
:10A0800003003200140020006C004700100812008A
:10A090006E00470010007800640260003900320052
:10A0A0006E00470010007800620260001400320069
:10A0B0006E0047001000780061026000040032006A
:10A0C000D0022000004278006C5004000000000024
:10A0D000B0022000004278004EB897000448780093
:10A0E00014002000680057001008420014002000EF
:10A0F00070004700100842009A5004000000000061
:10A100006E00470010007800610260000900320014
:10A110004EBA970000022000004A78001400200088
:10A12000680057001008420014002000700047002B
:10A13000100842006C0047001002780060005200D6
:10A140000E0034004EBA970000032000004A780049
:10A15000140020006800570010084200140020007E
:10A160007000470010084200140020006C004700F7
:10A17000100812009A50040000000000385104003A
:10A18000000000006E0047001000780068026000C8
:10A1900012003A006C004700100278006000520084
:10A1A0000E0034004EBA970000022000004A7800EA
:10A1B000140020006800570010084200140020001E
:10A1C0007000470010084200140020006C00470097
:10A1D00010081200CA500400000000006E00470082
:10A1E0001000780062026000140032006E00470028
:10A1F000100078006102600004003200D0022000EC
:10A20000004278000A51040000000000B002200063
:10A21000004278004EB897000448780014002000EF
:10A22000680057001008420014002000700047002A
:10A230001008420038510400000000006E00470082
:10A240001000780061026000090032004EBA9700E9
:10A2500000022000004A7800140020006800570027
:10A26000100842001400200070004700100842004F
:10A270006A0347001642780010002000164B1000B9
:10A280000404E0001F00320078004700300378002B
:10A29000A00378006A004700104078000080FB00AF
:10A2A0004202DD0020E42F00040240003401780067
:10A2B000A401780006007800870078000002EB0017
:10A2C0001EF90700A400200004017800CF91DE00F1
:10A2D0000002EB00EDF80700060320004EBA9700DD
:10A2E000004A430014002000680057001008420094
:10A2F000140020007000470010084200385104008C
:10A300000000000076004700100278006000520054
:10A310000E0034004EBA970000032000004A780077
:10A3200014002000680057001008420014002000AC
:10A33000700047001008420014002000760047001B
:10A34000100812008251040000000000680047005D
:10A350001002780068005200050034006A024700CD
:10A3600080002000004A7800C05104000000000076
:10A370006A0247006800470010407800004A7800F1
:10A380006A004700104278000482FB006800470022
:10A39000100812002E4890000004E00007003A0068
:10A3A0006E0047001002780000802000000262006A
:10A3B00002003A00F0510400000000004EBA97007D
:10A3C000E0022000004A78001400200068005700D6
:10A3D00010084200140020007000470010084200DE
:10A3E00078004700600F98006A004700104078002E
:10A3F0000080FB00801F78000DF707002F00B100E0
:10A400001E099000AE099000E50907004D090700FC
:10A410006E0A9000001A7800011278002E48900011
:10A420000004E0002100320078004700300378008B
:10A43000A00378006A024700144078006140500091
:10A44000004A78000080FB004202DD0020E42F007B
:10A450000402400034017800A4017800060078006E
:10A46000870078000002EB00B4F80700A400200089
:10A4700004017800CF91DE000002EB0083F80700B2
:10A48000060320004EBA9700004A43001400200043
:10A4900068005700100842001400200070004700B8
:10A4A000100842000E520400000000004E00900010
:10A4B0000000E0000E0032004EBA970000032000BA
:10A4C000004A78001400200068005700100842007D
:10A4D0001400200070004700100842001400200003
:10A4E00068004700100812005652040000000000E7
:10A4F0006E00470010007800680260001200320011
:10A500006C00470010027800600052000E0034001A
:10A510004EBA970000022000004A78001400200084
:10A520006800570010084200140020007000470027
:10A53000100842006C0047001000780061025000D3
:10A5400064079800F2FF3A00024404000000000093
:10A55000040C20006E0047001002620060005200F0
:10A560002A003A006E004700100078007002600078
:10A570000B00320078004700000478002EBB9700E3
:10A580002EBA970040002000140A10001600780030
:10A59000301C780020147800E6520400000000000F
:10A5A00078004700000478002EBB97002EBA970071
:10A5B00020002000140A1000160078001000780017
:10A5C000CF80DE00001C780001147800780047007E
:10A5D00030027800A00278006000520060805A00CB
:10A5E00008003D00340020006E0047001008720093
:10A5F0007802470034007800A4007800601A100048
:10A60000609218003A530400000000006E004700FA
:10A6100010007800700260000B00320078004700E4
:10A62000000478002EBB97002EBA9700400020004F
:10A63000140A100016007800301C780020147800EE
:10A640003A5304000000000078004700000478003E
:10A650002EBB97002EBA970020002000140A10008D
:10A6600016007800100078008000EB00001C7800D5
:10A670000114780068004700100278006000520062
:10A6800009003A007800470030027800A002780004
:10A690006000520060805A0003003A00140020005D
:10A6A0006800470010084200040C20006E004700BC
:10A6B000100062008044780008540400000000008C
:10A6C0006A02470010002000004A78006A00470034
:10A6D000104278006A4052001300320078044700AC
:10A6E0006A004700104078000080FB004202DD0055
:10A6F00020E42F000403400038027800A80278000C
:10A700003600520026805A000200310094530400A3
:10A7100000000000140020006A00470010484200BA
:10A7200066530400000000001E54040000000000F6
:10A730006A02470010002000004A78006A004700C3
:10A74000104278006840520013003200780447003D
:10A750006A004700104078000080FB004202DD00E4
:10A76000A0E62F000403400038027800A802780019
:10A770003600520026805A0002003100CC530400FB
:10A7800000000000140020006A004700104842004A
:10A790009E530400000000001E540400000000004E
:10A7A0006A02470010002000004A78006A00470053
:10A7B000104278006C4052001300320078044700C9
:10A7C0006A004700104078000080FB004202DD0074
:10A7D000A0E82F000403400038027800A8027800A7
:10A7E0003600520026805A00020031000454040052
:10A7F00000000000140020006A00470010484200DA
:10A80000D6530400000000001E54040000000000A5
:10A8100060C05400AAFF3200040C200004C05400A1
:10A82000A7FF32000408200004C05400C0FF32001B
:10A830000404200004C05400D9FF32006A0047001D
:10A84000104378000683FB006802470014005300A1
:10A8500006003D006A02470068004700104078008B
:10A86000004A78004A540400000000006A004700D3
:10A87000104378000683FB006802470014001300B1
:10A8800004003D006A004700104078000080FB0093
:10A89000400798006E0090000000E00007003200C2
:10A8A0006E00470010007800630260000300320071
:10A8B000140020006C004700100812006C004700D4
:10A8C00010037800680247001400530006003400AB
:10A8D00068004700100278006C0047001008120062
:10A8E0007854040000000000000020006007980079
:10A8F0006E00470010027800408C200000036200C8
:10A90000048420000400530008003A006E00900008
:10A910000000E00003003200140020006C0047003B
:10A9200010081200BA540400000000006E00470036
:10A9300010027800008C20000003620004882000D0
:10A94000040053000B003A006C004700100278002E
:10A950006200520005003400240020006C00470013
:10A9600010081200BA54040000000000000020008B
:10A97000600798006E0047001000780064026000D5
:10A980005C0032006E004700100078006202600038
:10A99000140032006E004700100078006102600071
:10A9A00004003200D002200000427800DE5404008F
:10A9B00000000000B0022000004278004EB897006E
:10A9C0000448780014002000680057001008420076
:10A9D0001400200070004700100842005455040085
:10A9E000000000006E004700100078006102600067
:10A9F0000B0032004EBA970000022000004A780097
:10AA000014002000680057001008420014002000C5
:10AA10007000470010084200545504000000000078
:10AA20006E00470010027800008C200000036200D6
:10AA300004882000040053001B003A004EBA97001F
:10AA400000032000004A780014002000680057002E
:10AA50001008420014002000700047001008420057
:10AA6000040220006E004700100262000400320061
:10AA700080052000004278004455040000000000DA
:10AA800080072000004278004EB897000448780004
:10AA90001400200068005700100842001400200035
:10AAA00070004700100842006E0090000000E000B7
:10AAB0000E0032004EBA970000032000004A7800D2
:10AAC0001400200068005700100842001400200005
:10AAD00070004700100842006C004700100078002A
:10AAE0006102500064079800F2FF3A0056560400D5
:10AAF000000000006E0090000000E0001200320034
:10AB00006E00470010007800680260000E003A00F6
:10AB10004EBA970000022000004A7800140020007E
:10AB20006800570010084200140020007000470021
:10AB3000100842006C0047001000780061025000CD
:10AB400064079800F2FF3A006E004700100078009A
:10AB500062026000140032006E00470010007800AE
:10AB60006102600004003200D00220000042780040
:10AB7000C055040000000000B00220000042780030
:10AB80004EB8970004487800140020006800570071
:10AB90001008420014002000700047001008420016
:10ABA000EE550400000000006E0047001000780021
:10ABB00061026000090032004EBA970000022000D6
:10ABC000004A780014002000680057001008420076
:10ABD0001400200070004700100842006E0047007B
:10ABE00010027800008C2000000362000484200022
:10ABF000040053000B003A004EBA970000032000F7
:10AC0000004A780014002000680057001008420035
:10AC1000140020007000470010084200565604003F
:10AC2000000000006E00470010027800008C200039
:10AC30000003620004882000040053001B003A0057
:10AC40004EBA970000032000004A7800140020004C
:10AC500068005700100842001400200070004700F0
:10AC600010084200040220006E004700100262003B
:10AC7000040032008005200000427800465604009F
:10AC80000000000080072000004278004EB89700C6
:10AC900004487800140020006800570010084200A3
:10ACA0001400200070004700100842006A004700AE
:10ACB000104378000683FB0068024700140013006D
:10ACC0000B0034004EBA970000032000004A7800C1
:10ACD00014002000680057001008420014002000F3
:10ACE00070004700100842005656040000000000A3
:10ACF0004E03900014002000680047001008120066
:10AD00000600E0007E003200040C20006E004700C8
:10AD100010006200405F98004C57040000000000E3
:10AD20007800470030037800A003780068004700EF
:10AD3000100078004202DD0020E42F0004024000F1
:10AD400034017800A40178000600780087007800BC
:10AD50000002EB0079F60700A4002000040178004F
:10AD6000CF91DE000002EB0048F60700060320004A
:10AD70006A024700064A40006A57040000000000CB
:10AD8000040220006E00470010026200170032002B
:10AD90007800470030037800A0037800680047007F
:10ADA000100078004202DD00A0E62F0004024000FF
:10ADB00034017800A401780006007800870078004C
:10ADC0000002EB005DF607006F026000E0826000A9
:10ADD000A0EB2F0004004000104278006A004700FA
:10ADE0000448780020570400000000007800470065
:10ADF00030037800A0037800680047001000780056
:10AE00004202DD00A0E62F00040240003401780079
:10AE1000A401780006007800870078000002EB00AB
:10AE200046F607006F026000E0826000B0EC2F0081
:10AE300004004000104278006A004700044878008F
:10AE40006A570400000000007800470030037800D3
:10AE5000A003780068004700100078004202DD007F
:10AE6000A0E82F000402400034017800A40178001B
:10AE700006007800870078000002EB002FF607003C
:10AE800067036000040320006A0047000448430091
:10AE90006A570400000000004E5A900060405200C3
:10AEA0009FFF3200060C20004E5A900006405200D0
:10AEB0009BFF3200060820004E5A900006405200C8
:10AEC000AFFF3200060420004E5A900006405200A8
:10AED000DDFF32006A0247004EB897001448780040
:10AEE00014002000680057001008420014002000E1
:10AEF000700047001008420078560400000000006F
:10AF00006E004700100078006802600012003200F6
:10AF10006C00470010027800600052000E00340000
:10AF20004EBA970000022000004A7800140020006A
:10AF3000680057001008420014002000700047000D
:10AF4000100842006C0047001000780061025000B9
:10AF500064079800F2FF3A00024404000000000079
:10AF60000E0890000080FA00000006000400FA00BD
:10AF7000E20047006A00570080087800811F7800CF
:10AF8000901F780068005700901F780014F60700A3
:10AF90006F00B100000F7800E800570091004000FA
:10AFA00000002000804878001E0078000080FA0031
:10AFB000000006000200FA00680057001000780048
:10AFC000000F78001E01780011002000600047008B
:10AFD000108840001204E00002003200E257040032
:10AFE00000000000600047009000780068005700F3
:10AFF00010805000610050000080FA000000060040
:10B000000200FA0068005700901F7800E9FF07006F
:10B010002F00B100000F78002006070060014700F4
:10B0200092001000020036000C58040000000000DE
:10B03000C822A900680057009000780031407800CD
:10B040000080FB00060032002022AF0024580400DC
:10B0500000000000201188001E58040000000000BD
:10B06000C822A8000080FA00000006000000FA00D4
:10B0700068005700901F780030EE2F00801F780086
:10B0800040E62000801F7800B8FF07006F00B10085
:10B0900040E62000801F7800D9FF07002F00B10094
:10B0A0000080FA000000060050042000801F780095
:10B0B000EEFF07002F00B100000006000800FA00B4
:10B0C0002077800010079800E4DD2000CFA2DE008A
:10B0D00062D120003200120022801A000F003D00D1
:10B0E00022778000C0E5200010014100227788000F
:10B0F0006000510002003D00000020002077880021
:10B10000227780007C00510002003400C001200042
:10B11000207788003064040000000000E4F620007E
:10B12000CFA2DE0062D120003200120022801A007D
:10B130000F00340022778000C0E52000100151008C
:10B14000227788006000510002003D0000002000CE
:10B1500020778800227780007C00510002003400B4
:10B16000C001200020778800306404000000000047
:10B1700000002000000F7800E4F62000CFA2DE00DF
:10B18000E2D020003200120022801A0004003400B5
:10B1900010002000000F7800E058040000000000BC
:10B1A000E4DD2000CFA2DE00E2D020003200120059
:10B1B00022801A0002003D00F0FF2F00000F7800EF
:10B1C000600047001001780000E620001091B900EF
:10B1D000020F780060005100A10532002277800044
:10B1E0007C0051000600320010002000007888002A
:10B1F000C0012000801F7800F3EF07002F00B1008E
:10B200007863040000000000B2768000C3768000FE
:10B210000000200001F82300310707000000E000D3
:10B220000200340000002000010037001000200060
:10B230000000E000060032006000470010017800C6
:10B240006000510002003D00505904000000000061
:10B25000B2768000C376800000C02300C161240064
:10B26000DC0607000000E00002003C0000002000B7
:10B2700001003700100020000000E000060032004E
:10B2800060004700100178006000510002003400A7
:10B290005059040000000000625904000000000042
:10B2A0001E007800CF80DE000081EB00E105070082
:10B2B000B2768000C37680000E070700B076880063
:10B2C000C17688002A6404000000000082758000B6
:10B2D00093758000A0702D0031C223000007070085
:10B2E0000000E000020034000000200001003700F0
:10B2F000100020000000E00006003200600047005F
:10B30000100178006000510002003D00B2590400B5
:10B31000000000008275800093758000000020000E
:10B3200001F82300AB0607000000E00002003C002B
:10B330000000200001003700100020000000E000A5
:10B3400006003200600047001001780060005100E4
:10B3500002003400B259040000000000CA59040081
:10B36000000000001E007800CF80DE000081EB00AE
:10B37000B0050700A2702D0033C2230008060700A5
:10B380008275800093758000DA060700807588005A
:10B39000917588002A64040000000000727080002B
:10B3A00083708000D0CC2C00C1E42300CC060700C1
:10B3B0000000E0000200340000002000010037001F
:10B3C000100020000000E00006003200600047008E
:10B3D000100178006000510002003D001A5A04007C
:10B3E0000000000072708000837080003033230002
:10B3F000F1192400770607000000E00002003C007D
:10B400000000200001003700100020000000E000D4
:10B410000600320060004700100178006000510013
:10B42000020034001A5A040000000000325A0400DE
:10B43000000000001E007800CF80DE000081EB00DD
:10B440007C050700D2CC2C00C3DC2300D405070008
:10B450007270800083708000A606070070708800FC
:10B46000817088002A64040000000000627080007F
:10B4700061005100060034006000470010017800B0
:10B480006000510002003D00605A0400000000000E
:10B4900054092000C2E020001200120006003D0006
:10B4A0006000470010017800600051000200340085
:10B4B000605A040000000000685A04000000000008
:10B4C0006000470010017800C0E020001008410033
:10B4D0002A6404000000000092768000A3768000B9
:10B4E0000000200001F823007D0607000000E000B6
:10B4F000020035000000200001003700100020008D
:10B500000000E000060032006000470010017800F3
:10B510006000510002003D00B85A04000000000025
:10B5200092768000A376800000C02300C1612400D1
:10B53000280607000000E00002003C000000200098
:10B5400001003700100020000000E000060032007B
:10B5500060004700100178006000510002003400D4
:10B56000B85A040000000000CA5A0400000000009D
:10B570001E007800CF80DE000081EB002D05070063
:10B5800092768000A37680005A06070090768800A5
:10B59000A17688002A640400000000001272800076
:10B5A00023728000D0CC2C00C1DC23004C060700A5
:10B5B0000000E0000200350000002000010037001C
:10B5C000100020000000E00006003200600047008C
:10B5D000100178006000510002003D001A5B040079
:10B5E000000000001272800023728000D0CC2C007A
:10B5F000712C2400F70507000000E00002003C0069
:10B600000000200001003700100020000000E000D2
:10B610000600320060004700100178006000510011
:10B62000020034001A5B040000000000325B0400DA
:10B63000000000001E007800CF80DE000081EB00DB
:10B64000FC040700D2CC2C00C3DC23005405070007
:10B650001272800023728000260607001072880094
:10B66000217288002A640400000000003077800006
:10B67000417780000200200003002000D50507006C
:10B680000000E00002003C00000020000100370044
:10B69000100020000000E0000600320060004700BB
:10B6A000100178006000510002003D00825B040040
:10B6B0000000000032778000437780000000200007
:10B6C00041242400C30507000000E00002003C0004
:10B6D0000000200001003700100020000000E00002
:10B6E0000600320060004700100178006000510041
:10B6F00002003400825B040000000000945B040040
:10B70000000000001E007800CF80DE000081EB000A
:10B71000C80407003277800043778000F5050700F2
:10B7200030778800417788002A6404000000000018
:10B73000F271800003728000D0CC2C00C1DC2300A9
:10B74000E70507000000E0000200350000002000CF
:10B7500001003700100020000000E0000600320069
:10B7600060004700100178006000510002003D00B9
:10B77000E45B040000000000F271800003728000AE
:10B78000D0CC2C00712C2400920507000000E000B2
:10B7900002003C00000020000100370010002000E3
:10B7A0000000E00006003200600047001001780051
:10B7B0006000510002003400E45B0400000000005F
:10B7C000FC5B0400000000001E007800CF80DE005B
:10B7D0000081EB0097040700D2CC2C00C3DC2300CF
:10B7E000EF040700F271800003728000C1050700BA
:10B7F000F0718800017288002A64040000000000D3
:10B800005277800063778000D0CC2C00C1DC23000D
:10B81000B30507000000E000020035000000200032
:10B8200001003700100020000000E0000600320098
:10B8300060004700100178006000510002003D00E8
:10B840004C5C0400000000005277800063778000A9
:10B85000D0CC2C00712C24005E0507000000E00015
:10B8600002003C0000002000010037001000200012
:10B870000000E00006003200600047001001780080
:10B8800060005100020034004C5C04000000000025
:10B89000645C0400000000001E007800CF80DE0021
:10B8A0000081EB0063040700D2CC2C00C3DC230032
:10B8B000BB04070052778000637780008D05070086
:10B8C00050778800617788002A6404000000000037
:10B8D0007077800081778000020020000300200044
:10B8E0003C0507000000E00002003C0000002000D2
:10B8F00001003700100020000000E00006003200C8
:10B9000060004700100178006000510002003D0017
:10B91000B45C040000000000727780008377800030
:10B9200000002000412424002A0507000000E00058
:10B9300002003C0000002000010037001000200041
:10B940000000E000060032006000470010017800AF
:10B950006000510002003400B45C040000000000EC
:10B96000C65C0400000000001E007800CF80DE00EE
:10B970000081EB002F04070072778000837780003E
:10B980005C05070070778800817788002A640400CE
:10B9900000000000527280006372800000002000EE
:10B9A00001F823004E0507000000E000020035000A
:10B9B0000000200001003700100020000000E0001F
:10B9C000060032006000470010017800600051005E
:10B9D00002003D00165D040000000000527280006D
:10B9E0006372800000002000612C2400F90407002D
:10B9F0000000E00002003C000000200001003700D1
:10BA0000100020000000E000060032006000470047
:10BA1000100178006000510002003400165D04003F
:10BA200000000000285D0400000000001E007800F7
:10BA3000CF80DE000081EB00FE0307005272800021
:10BA4000637280002B0507005072880061728800C5
:10BA50002A640400000000003272800043728000FB
:10BA6000D0CC2C00C1DC23001D0507000000E00045
:10BA70000200350000002000010037001000200007
:10BA80000000E0000600320060004700100178006E
:10BA90006000510002003D00785D040000000000DD
:10BAA0003272800043728000D0CC2C00712C2400B4
:10BAB000C80407000000E00002003C000000200075
:10BAC00001003700100020000000E00006003200F6
:10BAD000600047001001780060005100020034004F
:10BAE000785D040000000000905D0400000000008C
:10BAF0001E007800CF80DE000081EB00CD03070040
:10BB0000D2CC2C00C3DC2300250407003272800055
:10BB100043728000F7040700307288004172880089
:10BB20002A64040000000000B2718000C37180002C
:10BB30000000200001F82300E90407000000E000F5
:10BB40000200350000002000010037001000200036
:10BB50000000E0000600320060004700100178009D
:10BB60006000510002003D00E05D040000000000A4
:10BB7000B2718000C371800000002C009147240046
:10BB8000940407000000E00002003C0000002000D8
:10BB900001003700100020000000E0000600320025
:10BBA000600047001001780060005100020034007E
:10BBB000E05D040000000000F25D040000000000F1
:10BBC0001E007800CF80DE000081EB0099030700A3
:10BBD000B2718000C3718000C6040700B071880094
:10BBE000C17188002A64040000000000D271800046
:10BBF000E37180000000200001F82300B804070072
:10BC00000000E000020035000000200001003700C5
:10BC1000100020000000E000060032006000470035
:10BC2000100178006000510002003D00425E0400F7
:10BC300000000000D2718000E3718000000020004D
:10BC4000612C2400630407000000E00002003C00B7
:10BC50000000200001003700100020000000E0007C
:10BC600006003200600047001001780060005100BB
:10BC700002003400425E040000000000545E040034
:10BC8000000000001E007800CF80DE000081EB0085
:10BC900068030700D2718000E371800095040700FB
:10BCA000D0718800E17188002A640400000000005F
:10BCB00092778000A37780000000200001F8230025
:10BCC000870407000000E0000200350000002000AB
:10BCD00001003700100020000000E00006003200E4
:10BCE00060004700100178006000510002003D0034
:10BCF000A45E04000000000092778000A37780001B
:10BD00000000200031332400320407000000E0006E
:10BD100002003C000000200001003700100020005D
:10BD20000000E000060032006000470010017800CB
:10BD30006000510002003400A45E04000000000016
:10BD4000B65E0400000000001E007800CF80DE0018
:10BD50000081EB003703070092778000A377800013
:10BD60006404070090778800A17788002A640400A3
:10BD700000000000727680008376800000002000C2
:10BD800001122400560407000000E0000200350004
:10BD90000000200001003700100020000000E0003B
:10BDA000060032006000470010017800600051007A
:10BDB00002003D00065F0400000000007276800073
:10BDC0008376800000C02300C161240001040700C5
:10BDD0000000E00002003C000000200001003700ED
:10BDE000100020000000E000060032006000470064
:10BDF000100178006000510002003400065F04006A
:10BE0000000000001C5F040000000000A2002000F1
:10BE1000600047001090B900CF80DE000081EB0089
:10BE200004030700727680008376800031040700E7
:10BE300070768800817688002A6404000000000083
:10BE4000E27280006000510006003400600047008C
:10BE5000100178006000510002003D00485F0400BE
:10BE600000000000E27280006000510006003D000A
:10BE700060004700100178006000510002003400AB
:10BE8000485F0400000000004E5F04000000000056
:10BE90006000470010007800E07288002A64040007
:10BEA00000000000027380006000510006003400B2
:10BEB00060004700100178006000510002003D0062
:10BEC0007A5F0400000000000273800060005100EF
:10BED00006003D006000470010017800600051003E
:10BEE000020034007A5F040000000000805F04005C
:10BEF0000000000060004700100078000073880018
:10BF00002A64040000000000727580006000510087
:10BF10000600340060004700100178006000510006
:10BF200002003D00AC5F040000000000727580005C
:10BF30006000510006003C006000470010017800DE
:10BF40006000510002003400AC5F040000000000FB
:10BF5000B45F04000000000060004700100178009A
:10BF6000E0EA2000100841002A64040000000000FC
:10BF700082698000600051000600340060004700C4
:10BF8000100178006000510002003D00E25F0400F3
:10BF90000000000084698000823E20000200520000
:10BFA00006003D006000470010017800600051006D
:10BFB00002003400E25F040000000000EA5F0400B9
:10BFC00000000000600047001001780000D320004E
:10BFD000100841002A64040000000000226F800065
:10BFE0006000510006003400600047001001780036
:10BFF0006000510002003D001660040000000000D7
:10C00000226F80006000510006003C006000470085
:10C010001001780060005100020034001660040036
:10C0200000000000226004000000000060004700E3
:10C030001001780040DE2000100841002DEC0700C0
:10C04000ACEE07002A64040000000000B277800014
:10C0500065005100060034006000470010017800C0
:10C060006000510002003D0050600400000000002C
:10C07000B4778000C21220000200520006003D008A
:10C080006000470010017800600051000200340099
:10C090005060040000000000586004000000000030
:10C0A000600047001001780060EF20001008410098
:10C0B0002A640400000000006000470010017800BE
:10C0C000600051000600340000002000507088001D
:10C0D00010002000801F78000FEF07002F00B10034
:10C0E0002A64040000000000C2778000D37780003B
:10C0F000C05A2C0071722300790307000000E00091
:10C100000200350000002000010037001000200070
:10C110000000E000060032006000470010017800D7
:10C120006000510002003D00C060040000000000FB
:10C13000C2778000D37780000000200001F8230040
:10C14000240307000000E00002003C000000200083
:10C1500001003700100020000000E000060032005F
:10C1600060004700100178006000510002003400B8
:10C17000C060040000000000D8600400000000005F
:10C180001E007800CF80DE000081EB00290207004E
:10C19000C25A2C007372230081020700C27780000C
:10C1A000D377800053030700C0778800D1778800D9
:10C1B0002A64040000000000E2778000F37780002A
:10C1C000F026210031A82300450307000000E0000D
:10C1D00002003500000020000100370010002000A0
:10C1E0000000E00006003200600047001001780007
:10C1F0006000510002003D002861040000000000C2
:10C20000E2778000F37780000000200001F823002F
:10C21000F00207000000E00002003C0000002000E7
:10C2200001003700100020000000E000060032008E
:10C2300060004700100178006000510002003400E7
:10C2400028610400000000004061040000000000BC
:10C250001E007800CF80DE000081EB00F5010700B2
:10C26000F226210033A823004D020700E277800068
:10C27000F37780001F030700E0778800F1778800DC
:10C280002A64040000000000627580006000510014
:10C290000600340060004700100178006000510083
:10C2A00002003D006E6104000000000084022000D6
:10C2B000C2EA20001200120006003D0060004700A4
:10C2C0001001780060005100020034006E6104002B
:10C2D000000000007861040000000000627580002A
:10C2E0006000470010004100607588007071880090
:10C2F0002A6404000000000060004700100078007D
:10C3000061005000020032000000200001003700F0
:10C3100010002000A07588002A64040000000000BE
:10C3200060004700100078006100500002003200F9
:10C330000000200001003700100020001077880066
:10C34000801F78009CEE07002F00B1002A640400D3
:10C3500000000000600047001001780060005100FC
:10C36000DF00340000C02F00F107200020079800F4
:10C370003107980020002000801F780060ED200029
:10C38000801F780064004700801F7800DFEE070000
:10C390006F00B10020002000801F780000EB20001B
:10C3A000801F780064004700801F7800D7EE0700E8
:10C3B0006F00B10020002000801F7800E0E0200026
:10C3C000801F780064004700801F7800CFEE0700D0
:10C3D0006F00B10010002000801F7800C0E0200036
:10C3E000801F780064004700801F7800C7EE0700B8
:10C3F0006F00B10020002000801F780020ED200099
:10C40000801F780064004700801F7800BFEE07009F
:10C410006F00B10020002000801F780020E4200081
:10C42000801F780064004700801F7800B7EE070087
:10C430006F00B10020002000801F780060EE200017
:10C44000801F780064004700801F7800AFEE07006F
:10C450006F00B10020002000801F7800E0E3200082
:10C46000801F780064004700801F7800A7EE070057
:10C470006F00B10020002000801F7800A0EE200097
:10C48000801F780064004700801F78009FEE07003F
:10C490006F00B10020002000801F7800E0EE200037
:10C4A000801F780064004700801F780097EE070027
:10C4B0006F00B10020002000801F7800A0E4200061
:10C4C000801F780064004700801F78008FEE07000F
:10C4D0006F00B10020002000801F780060E4200081
:10C4E000801F780064004700801F780087EE0700F7
:10C4F0006F00B10020002000801F780060E3200062
:10C50000801F780064004700801F78007FEE0700DE
:10C510006F00B10020002000801F780020EF200075
:10C52000801F780064004700801F780077EE0700C6
:10C530006F00B10020002000801F7800A0E32000E1
:10C54000801F780064004700801F78006FEE0700AE
:10C550006F00B10020002000801F7800E0EC200078
:10C56000801F780064004700801F780067EE070096
:10C570006F00B10010002000801F7800C0E520008F
:10C58000801F780064004700801F78005FEE07007E
:10C590006F00B10010002000801F780000E620002E
:10C5A000801F780064004700801F780057EE070066
:10C5B0006F00B10010002000801F7800E0EA20002A
:10C5C000801F780064004700801F78004FEE07004E
:10C5D0006F00B10010002000801F780000D3200001
:10C5E000801F780064004700801F780047EE070036
:10C5F0006F00B10010002000801F780040DE200096
:10C60000801F780064004700801F78003FEE07001D
:10C610006F00B10010002000801F780060EF200044
:10C62000801F780064004700801F780037EE070005
:10C630006F00B10020002000801F780080EF2000F4
:10C64000801F780064004700801F78002FEE0700ED
:10C650006F00B10020002000801F7800C0EF200094
:10C66000801F780064004700801F780027EE0700D5
:10C670006F00B10010002000801F7800C0EA200089
:10C68000801F780064004700801F78001FEE0700BD
:10C690006F00B10010002000801F780020EE200005
:10C6A000801F780064004700801F780017EE0700A5
:10C6B0006F00B10010002000801F780040EB2000C8
:10C6C000801F780064004700801F78000FEE07008D
:10C6D0006F00B100000020000078880005ED070021
:10C6E0002A640400000000002A6404000000000026
:10C6F0002277800060005100C3FA32002277800068
:10C7000061005100F1FA320022778000620051008E
:10C7100022FB3200227780006300510053FB32007D
:10C7200022778000640051006BFB3200227780008A
:10C730006500510099FB32002277800066005100AD
:10C74000CAFB32002277800067005100F8FB3200FC
:10C75000227780006800510029FC32002277800097
:10C76000690051005AFC3200227780006A005100B3
:10C7700088FC3200227780006B005100B6FC32004A
:10C78000227780006C005100E7FC320022778000A5
:10C790006D00510015FD3200227780006E005100BF
:10C7A00043FD3200227780006F00510071FD32009E
:10C7B0002277800070005100A1FD320022778000B6
:10C7C00071005100B7FD32002277800072005100E5
:10C7D000CDFD32002277800073005100E4FD32006D
:10C7E0002277800074005100FCFD32002277800027
:10C7F0007500510015FE320022778000760051004E
:10C800002DFE3200227780007700510036FE320084
:10C81000227780007800510067FE32002277800086
:10C820007900510098FE3200227780007A00510092
:10C83000B1FE3200227780007B005100B8FE32004A
:10C84000227780007C005100C2FE32007463040035
:10C8500000000000E40EF8005BEA07002F00B100C2
:10C86000620047001002780042EE200012005200E1
:10C870000700320062004700901F780052EA07006C
:10C880002F00B100E40EF8004FEA07002F00B100BE
:10C8900005FA07000080FA0000000600C822A9007F
:10C8A00020C2A9002022AF00526404000000000052
:10C8B000F00F2000201188002002AE005C6404000C
:10C8C0000000000020118000F10F20000104E100B1
:10C8D000F3FF3A0020C2A9002022AF006C640400DC
:10C8E000000000000000EB00201188002002AE00D4
:10C8F000766404000000000020118000F000B20007
:10C90000110020000008DD00C822A8000000060079
:10C910000000FA004EB89700BEB897000000E00093
:10C9200004003200FA3F0900000000000000E900A6
:10C93000FAFF370001800900000000000080FA00C3
:10C94000000006000000FA0002000700166504005F
:10C95000000000000001BE001F0007000470A700D7
:10C9600003F0A1006509B100160032000D0035008A
:10C970006828E10006003500F0FF2F00F1FF2700D6
:10C980000300E00013003B00010028000000050048
:10C9900000004000818048008502E900FCFF3A0069
:10C9A00008003700F88F420002003C008000EB00D6
:10C9B000000005008100D1000080D3008502E8005E
:10C9C000FCFF3A000300E00002003B0060001000A2
:10C9D000E080180000000600C70ADE00F107B20080
:10C9E000F50FB20008003200E1CF42000200320031
:10C9F0000170A00024000500810F700001003200CA
:10CA00000408050044000500810F700002003A0090
:10CA1000140005008502E9000000400081C04800C4
:10CA2000FCFF3B000170A000240005000080FA001C
:10CA3000000006000000FA0002000700CC650400B8
:10CA4000000000000200E00006003A000005EB00D4
:10CA50000100E0000F003E000000E000270032006F
:10CA60000C003700010578000100E00004003500EB
:10CA700008003C000000E000200032000500370004
:10CA800060001000E080180002003B0001F02C0064
:10CA90001A0037000004BE006011B8006B092000C6
:10CAA0000982CF00020039000882CF000441B000A3
:10CAB000694252000E00320008003B008281710082
:10CAC000610164008904D1000884D3008B05E8006B
:10CAD0000442E800F9FF3A0005003700080444006A
:10CAE00089844C008B05E9000442E900FBFF3A0011
:10CAF000030007000AF0A70001F0A00000000600F4
:10CB000081002000618055000B003D000B002000DB
:10CB100061FE2F000100E1001D00340082817100E0
:10CB2000610164008904D1000884D3000000E8009A
:10CB3000FAFF3A00710020006100640003007000F9
:10CB4000020060000900320061044400E0844C00EF
:10CB50000988A500050032008B05E8006808E1009F
:10CB600002003A008904D1000884D300F20F2000AB
:10CB70000258E10005003D00C75DDD00F907B20085
:10CB80008980750008007800000006000BF8270077
:10CB90008B007800000005000080FA00000006000D
:10CBA0000000FA0002000700E66604000000000032
:10CBB000889FBE008A9FBE008C1F7800300007004F
:10CBC0003700330003866C006450E100240032001B
:10CBD0006420E100270032006150E10022003200B1
:10CBE0006120E100210032008B854200EB07B1009B
:10CBF0000134B800003AB8000804420089844A00B1
:10CC0000013AB8000030B8008880400009014A00AD
:10CC10000400330000004000818048000201490008
:10CC20008B05E900C909DD008301700001003200B5
:10CC300013002000C814DE004814DD004709DE00A0
:10CC40001200B200C808DE0008847000240007004B
:10CC500001F0A1000CF0A70001F0A00019003700BE
:10CC60006120E1001B0032000801BE000200BE008E
:10CC7000F7FF37006150E100FCFF3A001500370074
:10CC80000004BE003C0007000003BE000405BE0017
:10CC90000200BE0038000700844F75000000060047
:10CCA0000200BE006450E100050036006420E1008F
:10CCB000020036000968A30001003A000800BE0027
:10CCC0000160A0004F0678004F05BE004F04BE0073
:10CCD00000000600F0FF2F00F1FF2700F9FF3700EA
:10CCE00081002000618055000B003D000B002000FA
:10CCF00061FE2F000100E1001D00340082817100FF
:10CD0000610164008904D1000884D3000000E800B8
:10CD1000FAFF3A0071002000610064000300700017
:10CD2000020060000900320061044400E0844C000D
:10CD30000988A500050032008B05E8006808E100BD
:10CD400002003A008904D1000884D300F20F2000C9
:10CD50000258E10005003D00C75DDD00F907B200A3
:10CD60008980750008007800000006000BF8270095
:10CD70008B00780000000500C70ADE00F107B20052
:10CD8000F50FB20008003200E1CF4200020032008D
:10CD90000170A00024000500810F70000100320026
:10CDA0000408050044000500810F700002003A00ED
:10CDB000140005008502E9000000400081C0480021
:10CDC000FCFF3B000170A000240005000080FA0079
:10CDD000000006000000FA00F4FF2F000700070023
:10CDE0000080FA00000006000000FA0003F0A20034
:10CDF000400007000080FA00000006000000FA0072
:10CE0000020007006C67040000000000841F780027
:10CE1000140007004F00780011003300F0FF2F00CE
:10CE2000838F6C0006003B00040565000A00A70024
:10CE30000800370009F0A6001000200008003700A5
:10CE4000820F5400838F5C00030039001000200023
:10CE500001003E000000200009F0A7000000EA00E9
:10CE6000000006000004BE00060007000003BE002C
:10CE70000405BE000200BE0002000700844F7500DA
:10CE800000000600C70ADE00F107B200F50FB2008D
:10CE900008003200E1CF4200020032000170A00021
:10CEA00024000500810F7000010032000408050015
:10CEB00044000500810F700002003A0014000500D4
:10CEC0008502E9000000400081C04800FCFF3B00F3
:10CED0000170A000240005000080FA000000060098
:10CEE0000000FA0014002000C4FF07000080FA00D0
:10CEF000000006000000FA0002000700E2680400DB
:10CF000000000000889FBE008A9FBE008C1F780032
:10CF100059000700600033006450E1004F00320008
:10CF20006420E1005200320003826C0007003B00E5
:10CF30000905D0000306D000820F54000C065D00E6
:10CF400002003900020032008901780003067800EF
:10CF50008582550004003D000003FD008103FD00B3
:10CF60008502EA008B854200840F720002003B00BC
:10CF700060001000E08018006011B8000005EB00B0
:10CF80007A28E1000A00390006007800C75DDD005C
:10CF9000F707B200878075002D003700828171008D
:10CFA0000A017800610560008180D1000080D30013
:10CFB0008502E900F9FF3B00060440008784480031
:10CFC00002003B0060041400E0841C000988A300F8
:10CFD000070032008A817100828171006101640062
:10CFE0008904D1000884D3008B05E80017003700BE
:10CFF0000978A30013003A000B00E000130034008E
:10D000008B05E9000804440089844C000A4474003C
:10D010000978A3000D003A000B00E000070034007F
:10D020008B05E9000804440089844C0001003A00A3
:10D030000B0020000978A300F7FF32000001EB008D
:10D0400002003700828171000A0178002200070087
:10D050000CF0A70001F0A000180037006420E100E8
:10D0600002003A00838F6C00180033000801BE00F4
:10D070000200BE00110037000004BE003C000700A3
:10D080000003BE000405BE000200BE003800070019
:10D09000844F7500000006000200BE006450E100ED
:10D0A000050036006420E100020036000968A30094
:10D0B00001003A000800BE000160A0004F067800A1
:10D0C0004F05BE004F04BE0000000600F0FF2F0019
:10D0D000F1FF2700F9FF3700810020006180550033
:10D0E0000B003D000B00200061FE2F000100E1005D
:10D0F0001D00340082817100610164008904D10047
:10D100000884D3000000E800FAFF3A007100200014
:10D11000610064000300700002006000090032003A
:10D1200061044400E0844C000988A5000500320039
:10D130008B05E8006808E10002003A008904D1008C
:10D140000884D300F20F20000258E10005003D00E2
:10D15000C75DDD00F907B20089807500080078001E
:10D16000000006000BF827008B0078000000050087
:10D17000C70ADE00F107B200F50FB2000800320066
:10D18000E1CF4200020032000170A000240005003F
:10D19000810F700001003200040805004400050002
:10D1A000810F700002003A00140005008502E900BA
:10D1B0000000400081C04800FCFF3B000170A0005F
:10D1C000240005000080FA00000006000000FA00BC
:10D1D00002000700186A040000000000889FBE00DB
:10D1E0008A9FBE008C1F78003E0007004500330078
:10D1F00003866C006450E1002E0032006420E100E0
:10D20000330032006150E1002F0032006120E10064
:10D210003100320085855500EB07B0000900200081
:10D2200008042000050037000804440089844C00ED
:10D230000A0031000603430087834B0000015300BE
:10D2400081815B00F8FF33000203BE000800A000EC
:10D250000804440089844C00F6FF3900C639DD001B
:10D260008301730001003200130020008904D10003
:10D270000884D3000998A300050032000800A70025
:10D280000300A0008904D1000884D3008B05E800C6
:10D290008904D1000884D3000001EB000281D20090
:10D2A0002800070001F0A1000CF0A70001F0A00089
:10D2B0001D0037006420E1001F0032000801BE009D
:10D2C0000200BE00F7FF37006120E1001A003200C3
:10D2D0006000B800F3FF37000000200001F82700CD
:10D2E000F0FF37000004BE003C0007000003BE0052
:10D2F0000405BE000200BE0038000700844F750020
:10D30000000006000200BE006450E1000500360087
:10D310006420E100020036000968A30001003A0021
:10D320000800BE000160A0004F0678004F05BE0057
:10D330004F04BE0000000600F0FF2F00F1FF2700A1
:10D34000F9FF370081002000618055000B003D008F
:10D350000B00200061FE2F000100E1001D003400E1
:10D3600082817100610164008904D1000884D300C6
:10D370000000E800FAFF3A0071002000610064003C
:10D3800003007000020060000900320061044400E4
:10D39000E0844C000988A500050032008B05E800F8
:10D3A0006808E10002003A008904D1000884D30033
:10D3B000F20F20000258E10005003D00C75DDD00CE
:10D3C000F907B200898075000800780000000600A7
:10D3D0000BF827008B00780000000500C70ADE006C
:10D3E000F107B200F50FB20008003200E1CF4200B1
:10D3F000020032000170A00024000500810F7000BF
:10D40000010032000408050044000500810F70008F
:10D4100002003A00140005008502E9000000400007
:10D4200081C04800FCFF3B000170A0002400050003
:10D430000080FA00000006000000FA00020AB800AE
:10D44000800278000200B80081004200032AB80080
:10D45000810042000080FA00000006000F802000DA
:10D46000E0BF2000000188004440A8000000200028
:10D47000A001880060F7200061F62F000700090076
:10D48000315878008A00FA006000470051F02F0000
:10D490000E000900315878006F00470041F12F005D
:10D4A0002C00090031587800C0032000000047001C
:10D4B00011F42F00180009003158780050052000A1
:10D4C00000004700A1F52F00030009003158780043
:10D4D0009005200000004700E1F52F00070009003B
:10D4E000315878000000200010379800000020001C
:10D4F0004037980000772000400E88000000200090
:10D50000C0168800E4FF2F00A02D20001008620044
:10D51000E0E02000801F780010002000801F7800CD
:10D52000FBFC07004F00B10014002000A02D2000DC
:10D5300010087200002C210001002000801F7800DC
:10D54000811F7800DECC07004F00B10004402000AE
:10D55000C02020001008720000102E0001002000E2
:10D56000801F7800811F78006ECD07004F00B1004A
:10D5700004002800602120001008720060F72000DD
:10D5800000608800C1CD0700D5CD07000000200055
:10D59000CF80DE007078880081788800000020004D
:10D5A0000100200050788800617888000000200089
:10D5B00001002000307888004178880000002000B9
:10D5C00001002000107888002178880060EA20009F
:10D5D000CF80DE00F06888000169880060EA2000E2
:10D5E00001002000D0688800E168880060EA20001F
:10D5F00001002000706888008168880060EA2000CF
:10D6000001002000B0688800C16888001000200078
:10D61000707588000000200001002000507688000E
:10D62000617688000000200001002000606B880007
:10D63000716B8800000020000100200080728800CB
:10D64000917288000000200001002000B072880064
:10D65000C17288000000200001002000806B88005B
:10D66000916B88000000200001002000D07088002D
:10D67000E17088000000200001002000106B88008D
:10D68000216B88000000200001002000F06A880063
:10D69000016B88000000200001002000A06A8800C3
:10D6A000B16A88000000200001002000D06A8800D4
:10D6B000E16A88000000200001002000303F98004F
:10D6C000413F98000000200001002000103F98001A
:10D6D000213F98000000200001002000B070880069
:10D6E000C17088000000200001002000F070880058
:10D6F0000171880000002000010020009070880067
:10D70000A17088000000200001002000A06F8800A8
:10D71000B16F88000000200001002000606F8800C9
:10D72000716F88000000200001002000806F8800D9
:10D73000916F8800000020004070880000002000E9
:10D740003070880000002000207088000000200059
:10D75000806A880000002000906A88000000200095
:10D760000100200070379800013F98000000200061
:10D7700001002000606A8800716A880000002000B3
:10D7800001002000D0768800E176880000002000AB
:10D79000010020006BFC0700A071880090718800D8
:10D7A000A072880070728800CF80DE000081EB00DC
:10D7B000A0FC0700B0758800C17588003071880032
:10D7C0004171880050718800617188001071880073
:10D7D0002171880084D5200000022000004A7800D2
:10D7E00094D5200000022000004A780074D3200065
:10D7F00000022000004A780000002000CF80DE00F8
:10D8000090698800A1698800000020007069880084
:10D8100000002000206988000000200010698800B6
:10D820000000200000788800000020006037980089
:10D830000000200050379800000020008071880010
:10D8400000002000506B880000002000507088000D
:10D8500000002000A06B88000000200000778800F6
:10D8600000002000F0768800000020006069880039
:10D87000000020003037980000002000207788004A
:10D880000000200090688800A0C52F00F10720004C
:10D89000703F98000187980000002000CF80DE00D4
:10D8A00010879800218798000000200010758800DC
:10D8B00000002000007588000000200050758800DE
:10D8C00000002000307588000000200040758800AE
:10D8D00000002000207588000000200020608800E3
:10D8E000000020003060880010002000106F8800C9
:10D8F00010002000A068880064D3200040002000B1
:10D90000004A7800000020004068880000002000E5
:10D910005068880000002000606888000010200027
:10D92000801F780000002000801F78000000200089
:10D93000801F780000002000801F78000000200079
:10D94000801F780020002000801F78000000200049
:10D95000801F780000022000801F780086CD07001D
:10D960000F01B10000C02F00F1072000503F9800C8
:10D97000613F980020002000801F780060ED2000AB
:10D98000801F7800A007200000004700801F78005B
:10D99000B1CF07006F00B10020002000801F780089
:10D9A00000EB2000801F7800A00720000000470047
:10D9B000801F7800A8CF07006F00B1002000200072
:10D9C000801F7800E0E02000801F7800A007200082
:10D9D00000004700801F78009FCF07006F00B10054
:10D9E00010002000801F7800C0E02000801F780019
:10D9F000A007200000004700801F780096CF070096
:10DA00006F00B10020002000801F780020ED200072
:10DA1000801F7800A007200000004700801F7800CA
:10DA20008DCF07006F00B10020002000801F78001C
:10DA300020E42000801F7800A0072000000047009D
:10DA4000801F780084CF07006F00B1002000200005
:10DA5000801F780060EE2000801F7800A007200063
:10DA600000004700801F78007BCF07006F00B100E7
:10DA700020002000801F7800E0E32000801F780055
:10DA8000A007200000004700801F780072CF070029
:10DA90006F00B10020002000801F7800A0EE200061
:10DAA000801F7800A007200000004700801F78003A
:10DAB00069CF07006F00B10020002000801F7800B0
:10DAC000E0EE2000801F7800A00720000000470043
:10DAD000801F780060CF07006F00B1002000200099
:10DAE000801F7800A0E42000801F7800A00720009D
:10DAF00000004700801F780057CF07006F00B1007B
:10DB000020002000801F780060E42000801F780043
:10DB1000A007200000004700801F78004ECF0700BC
:10DB20006F00B10020002000801F780060E320001B
:10DB3000801F7800A007200000004700801F7800A9
:10DB400045CF07006F00B10020002000801F780043
:10DB500020EF2000801F7800A00720000000470071
:10DB6000801F78003CCF07006F00B100200020002C
:10DB7000801F7800A0E32000801F7800A00720000D
:10DB800000004700801F780033CF07006F00B1000E
:10DB900020002000801F7800E0EC2000801F78002B
:10DBA000A007200000004700801F78002ACF070050
:10DBB0006F00B10010002000801F7800C0E5200039
:10DBC000801F7800A007200000004700801F780019
:10DBD00021CF07006F00B10010002000801F7800E7
:10DBE00000E62000801F7800A0072000000047000A
:10DBF000801F780018CF07006F00B10010002000D0
:10DC0000801F7800E0EA2000801F7800A007200035
:10DC100000004700801F78000FCF07006F00B100A1
:10DC200010002000801F780000D32000801F7800A3
:10DC3000A007200000004700801F780006CF0700E3
:10DC40006F00B10010002000801F780040DE20002F
:10DC5000801F7800A007200000004700801F780088
:10DC6000FDCE07006F00B10010002000801F78007B
:10DC700060EF2000801F7800A00720000000470010
:10DC8000801F7800F4CE07006F00B1002000200054
:10DC9000801F780080EF2000801F7800A007200000
:10DCA00000004700801F7800EBCE07006F00B10036
:10DCB00020002000801F7800C0EF2000801F780027
:10DCC000A007200000004700801F7800E2CE070078
:10DCD0006F00B10010002000801F7800C0EA200013
:10DCE000801F7800A007200000004700801F7800F8
:10DCF000D9CE07006F00B100607580007071880098
:10DD000010002000801F780020EE2000801F780087
:10DD1000A007200000004700801F7800CECE07003B
:10DD20006F00B10010002000801F780040EB200041
:10DD3000801F7800A007200000004700801F7800A7
:10DD4000C5CE07006F00B100647080006000520013
:10DD50000C00350076092000C4E0200014001300F8
:10DD600008003C00A6D72000CFB3DE0064D120001D
:10DD70003400130024801B0002003500766F04007D
:10DD800000000000000020000124240050728800E0
:10DD9000617288000000200001222400F0718800D8
:10DDA00001728800000020000117240050778800CD
:10DDB00061778800000020000112240010728800A2
:10DDC0002172880000002000011024007077880074
:10DDD000817788000000200001F823003077880058
:10DDE0004177880000002000010A2400307288007A
:10DDF00041728800000020004123240090778800B1
:10DE0000A17788000000200001122400D071880052
:10DE1000E1718800B00420006070880000002400D8
:10DE2000C159240090768800A1768800606626009B
:10DE300061FA230070708800817088001000200053
:10DE4000E0728800100020000073880000002000AD
:10DE5000812C2400B0718800C17188000000280066
:10DE6000414D2400707688008176880090C225009C
:10DE7000F1D823008075880091758800000020008B
:10DE800061492400B0768800C17688001000200027
:10DE900070758800800720008069880010002000CD
:10DEA000206F880050002000B077880060712C003F
:10DEB000C1A52300C0778800D1778800B0D82F0093
:10DEC00051DA2300E0778800F17788000000200015
:10DED000707188000000200060758800000020003C
:10DEE0001077880000002000A07588000000200046
:10DEF000010E2400D0758800E17588000000200024
:10DF0000010E240010768800217688007070800051
:10DF100081708000306F8800416F880060708000E1
:10DF2000506F880064708000A0DE2000610842000D
:10DF30000000200010379800200620000000470055
:10DF4000100278006C00520016003D0026062000EA
:10DF500006034700160078004202DD0060D720006B
:10DF60000402400000002000000A7800060078004B
:10DF7000100078004202DD0060D72000040040005D
:10DF80006202400000002000000A78001400200017
:10DF90002006200000004700100842009C6F04008B
:10DFA0000000000000002000100E8800701A2600FB
:10DFB000200E880080002800000E880060EA200003
:10DFC000D00E8800D00E8000C00E8800C00E8000E9
:10DFD000B00E8800E06A2000801F7800700B2000DF
:10DFE000801F78004AFA07004F00B10041E40700A3
:10DFF000E40DF80090EE2F00801F780040E620002E
:10E00000801F7800D9F307006F00B10040E62000C0
:10E01000801F7800FAF307002F00B100600047006E
:10E02000801F7800F6F307002F00B100E0462000C3
:10E03000801F7800A0072000801F780034FA0700B6
:10E040004F00B10018F407006F004700801F7800F0
:10E05000EBF307002F00B100E01E2100801F7800C5
:10E06000801E2000801F780029FA07004F00B100B1
:10E0700020002000103798002006200000004700F4
:10E0800010027800600052001800340020062000C2
:10E090000000470010007800610050001037980021
:10E0A000801F780020EF2F00801F780060DA2000AA
:10E0B000801F7800ADF307006F00B10060DA200028
:10E0C000801F780018D107002F00B100E0CE220099
:10E0D000801F7800404C2000801F78000CFA070059
:10E0E0004F00B1003C7004000000000001E4070094
:10E0F00004402000E02020001008720004002800E6
:10E10000C02020001008720010082000801F780036
:10E11000B9CB07002F00B10000022000801F78005B
:10E12000B5CB07002F00B100A0002000801F7800B1
:10E13000B1CB07002F00B100F4DF2F004008200012
:10E1400010086200D4FF2F00E020200010086200B9
:10E15000C003200000004700801F7800F2D00700B5
:10E160002F00B100BECB0700600250000200350056
:10E17000B270040000000000D1CB07000004E000F2
:10E1800003003A000060FE00BC70040000000000C4
:10E19000E08E2000801F7800400F2000801F780054
:10E1A000DBF907004F00B100D2E30700E068200070
:10E1B000801F780060002000801F7800D4F90700DD
:10E1C0004F00B100B8F307005005200000004700E1
:10E1D000801F780087E607002F00B100E04620008E
:10E1E000801F7800A0072000801F7800C8F9070072
:10E1F0004F00B10010002000801F7800C6E6070025
:10E200002F00B100E0462000801F7800A00720000A
:10E21000801F7800BEF907004F00B1009005200074
:10E2200000004700801F780072E607002F00B10051
:10E2300010698000CF80DE000081EB00FDF907004F
:10E24000B2FA2C0053CD230055FA0700308798000E
:10E2500041879800B0758800C175880020698000EA
:10E26000CF80DE000081EB00F2F9070012362C00AF
:10E2700033CD23004AFA0700F07588000176880044
:10E280003E809000CE8090000002780081027800ED
:10E29000000020008110240004017800850178002E
:10E2A000CCFA07000000E00002003C000000200063
:10E2B00001003700100020000000E00006003200DE
:10E2C00000002000010E2400D0758800E175880050
:10E2D00074710400000000000000200001122400FE
:10E2E000D0758800E1758800F4758000057680009F
:10E2F00000002000811024000401780085017800CE
:10E30000B4FA07000000E00002003C00000020001A
:10E3100001003700100020000000E000060032007D
:10E3200000002000010E240010768800217688006D
:10E33000CC71040000000000F475800005768000B8
:10E34000D0CC2C00C1142400040178008501780091
:10E35000A0FA07000000E00002003C0000002000DE
:10E3600001003700100020000000E000060032002D
:10E370000000200001122400107688002176880019
:10E38000CC710400000000000000200001152400F2
:10E390001076880021768800000020001037980051
:10E3A0000000200040379800E20EF80082E60700E7
:10E3B0002F00B10042CB07000004E0008C013200C6
:10E3C0000060FE0026CB0700203798006002500056
:10E3D000850135003606200024062000040247008F
:10E3E00014001300060034000000200010379800CD
:10E3F0000000200040379800F47404000000000082
:10E40000D2740400000000000000200010379800C3
:10E410001000200040379800F47404000000000051
:10E4200020F12000260620000603470016024000C7
:10E4300000002000004A780010002000160B400069
:10E44000F47404000000000024F1200020062000E5
:10E45000000047001002420000002000004A78003F
:10E460008006200000004700100278006000520083
:10E4700039013200000020004037980020F12000D0
:10E48000801F780022CD07002F00B10060025000ED
:10E4900031013400846B8000956B8000A26F800096
:10E4A000B36F800004007800850078004EFA070002
:10E4B000D0708800E1708800E0062000000047006E
:10E4C00030027800A0027800606A8000716A8000E3
:10E4D000040178008501780081FA07000000E0005F
:10E4E00002003A0000002000010037001000200068
:10E4F0000000E0008E003200E0062000000047002F
:10E5000030027800A0027800606A8000716A8000A2
:10E51000040178008501780071FA07000000E0002E
:10E52000020035000000200001003700100020002C
:10E530000000E0000B003200E00620000000470071
:10E5400030027800A0027800020020000327240097
:10E55000040078008500780023FA070070379800DF
:10E56000013F980014002000A00620000000470092
:10E570001008420014002000C006200000004700E0
:10E5800010084200D6708000E77080002407200049
:10E590000402470034017800A401780006007800E6
:10E5A0008700780010FA0700807288009172880056
:10E5B000166B8000276B8000640720000402470070
:10E5C00034017800A4017800060078008700780004
:10E5D00005FA0700B0728800C17288000002780056
:10E5E00081027800000020004133240004017800FB
:10E5F000850178003AFA07000000E00002003500CB
:10E600000000200001003700100020000000E000A2
:10E610000B003200B4728000C5728000020020003E
:10E62000433B24000400780085007800EEF90700E1
:10E63000B0728800C17288004E73040000000000B0
:10E64000B4728000C57280000000200041332C00AD
:10E650000401780085017800DEF907000000E00081
:10E6600002003C00000020000100370010002000E4
:10E670000000E00009003200B4728000C572800022
:10E6800000002000413B240004017800850178004F
:10E6900018FA0700B0728800C1728800666A8000AC
:10E6A000776A8000E4062000040247003401780005
:10E6B000A40178000600780087007800CAF90700F6
:10E6C0003087980041879800000178008101780028
:10E6D000B0728000C1728000BCFA0700B07288007E
:10E6E000C17288003E819000CE81900080728000CF
:10E6F00091728000B5FA07008072880091728800DC
:10E70000606A8000716A800070379800013F98004D
:10E71000D0708000E1708000103F9800213F980089
:10E72000106B8000216B8000303F9800413F9800C3
:10E73000547080006000520003003A0091CF07003F
:10E74000AC7404000000000000002000801F78006E
:10E75000E5D307002F00B100A468800060005200DC
:10E760000C003A00946880006000520009003A00F2
:10E77000A006200000004700901F78001000200035
:10E78000801F780056D507004F00B100D8730400F1
:10E7900000000000A006200000004700901F780045
:10E7A00000002000801F78004DD507004F00B10009
:10E7B0000000200050379800B477800060005200BD
:10E7C00065003400C00620000000470010037800F8
:10E7D00064EF2000140053005F00350000002000AB
:10E7E00060379800F46A8000056B8000000020000C
:10E7F00001F023000401780085017800B8F90700D2
:10E800000000E0000200340000002000010037009A
:10E81000100020000000E00007003A006006200021
:10E820000000470010027800600052000200320031
:10E83000AC74040000000000E00720000000470066
:10E8400030037800A003780044FF2F00F507200074
:10E850000400530005805B003F003E0000242400BC
:10E86000F1002000826A8000CF91DE00F2FA0700FA
:10E8700066D6200036024000A68248003487980001
:10E880004587980000102E00515F2000926A80009A
:10E89000CF91DE00E8FA07003E829000CE82900021
:10E8A0000002420081824A00200820000000470048
:10E8B0001018420010904A00600620000000470037
:10E8C000100278006000520018003A00200020007A
:10E8D000CF80DE00E407200004024700141A100075
:10E8E0001492180010002000801F7800600620009D
:10E8F00000004700801F7800841F780083E5070030
:10E900006F00B10020002000801F78002008200048
:10E9100000004700801F7800E0072000000047004B
:10E92000801F780079E507006F00B10060062000C5
:10E930000000470010007800610040003037980068
:10E94000801F7800E007200000004700801F78004B
:10E9500093D607004F00B100F474040000000000DB
:10E96000800620000000470010027800600052007E
:10E970000A00320020F1200026062000060347008E
:10E9800016024000400620000000470010407800BA
:10E99000004A780010002000160B4000F4740400B8
:10E9A0000000000046022000440620000402470048
:10E9B0001400130094FE32004006200000004700BF
:10E9C000100278006D00520095FE320040062000D3
:10E9D00000004700100278006A0052009AFE3200E0
:10E9E000B074040000000000DA71040000000000B0
:10E9F00060D3200010427800644052009E0039002D
:10EA000064D3200000002000004A780010698000D4
:10EA1000CF80DE000081EB0006F80700B2FA2C0080
:10EA200053CD23005EF80700B4758000C5758000E3
:10EA300004017800850178002EF90700020020000B
:10EA400003002400E1F90700B0758800C175880053
:10EA500020698000CF80DE000081EB00F5F7070021
:10EA600012362C0033CD23004DF80700F4758000DA
:10EA70000576800004017800850178001DF9070003
:10EA80000200200003002400D0F90700F075880080
:10EA90000176880070698000CF80DE000081EB0085
:10EAA000E4F70700E2778000F37780003CF8070086
:10EAB0003076880041768800000278008102780074
:10EAC000D0768000E176800004017800850178002E
:10EAD00003F907000000E0000200350000002000FC
:10EAE00001003700100020000000E00004003200A8
:10EAF0003076800041768000D0768800E17688000C
:10EB000090698000A16980000001EB00C9F707004F
:10EB1000C2778000D377800021F807005076880004
:10EB20006176880006AF2000CFB3DE00A4D12000BC
:10EB30003400130024801B0014003D00507080003E
:10EB40000000E00011003200946880006100520073
:10EB500007003A00000020009068880010002000A4
:10EB6000A06B880063E10700C2750400000000008C
:10EB700000002000A068880010002000106F8800AE
:10EB8000EAD807003A7604000000000010002000D8
:10EB9000A0688800C63E2100CFB3DE00A4D12000CB
:10EBA0003400130024801B000400340060EA2000BD
:10EBB000CF80DE00D0688800E1688800C62521008B
:10EBC000CFB3DE00A4D120003400130024801B004A
:10EBD00008003400146F80006100520003003A0006
:10EBE00044E1070000002000106F88003A7604001E
:10EBF0000000000046192100CFB3DE00A4D12000A0
:10EC00003400130024801B000F003400146F8000B8
:10EC10006100520003003A0036E1070000002000C6
:10EC2000106F8800946880006000520003003A0072
:10EC30001000200090688800AEE307001FF1070075
:10EC40003A760400000000009468800061005200E1
:10EC500005003A00000020009068880025E10700C8
:10EC60003A7604000000000010002000106F8800B9
:10EC7000AED8070009F70700DA71040000000000B1
:10EC80000080FA00FFFF37003235FF00312CFF0013
:10EC90003131FF003532FF003030FF000000FF004F
:10ECA0000000FF000000FF000000FF000000FF0068
:10ECB0000000FF000000FF000000FF000000FF0058
:10ECC0000000FF00003CFF000A25FF003031FF007C
:10ECD000306CFF00750AFF000025FF00382EFF0092
:10ECE0003666FF002C25FF00382EFF003666FF0039
:10ECF0002C25FF00640AFF000047FF005052FF0070
:10ED00004D43FF000047FF005047FF004741FF0011
:10ED10000047FF005047FF005356FF000050FF0020
:10ED2000494EFF004700FF00504FFF004E47FF00D5
:10ED30000A00FF004745FF00544CFF004F47FF000B
:10ED4000003EFF000A00FF005365FF007474FF00DF
:10ED5000696EFF006720FF00484FFF004D45FF0030
:10ED60002025FF002D33FF006400FF00484FFF0007
:10ED70004D45FF00206EFF006F74FF002073FF0001
:10ED80006574FF0000FFFF000000FF000000FF00AF
:10ED9000C4FFFF007F3FFF0080EFFF00FFBEFF00CA
:10EDA00090E1FF00A93EFF00EC82FF0076BEFF006D
:10EDB00082ADFF002B3EFF000E3CFF00C3BDFF00F5
:10EDC00087D1FF00133DFF004178FF00D3BBFF0058
:10EDD0000000FF00803FFF001872FF00313FFF007E
:10EDE000F0FDFF00753EFF004758FF00633DFF0048
:10EDF0005895FF001D3CFF0082C4FF00AE3AFF00A3
:10EE0000A878FF002139FF00EF93FF008037FF0053
:10EE1000A092FF00A735FF004656FF001534FF0003
:10EE2000063CFF000442FF007D9FFF006A42FF0096
:10EE30005C90FF000142FF00604DFF00BB40FF00FF
:10EE400051ECFF00473EFF00DE8DFF001FBBFF00BF
:10EE5000063CFF000442FF00C059FF008B42FF0048
:10EE60007404FF004442FF00F99BFF004F41FF0084
:10EE70000000FF00803FFF001B5BFF003958FF00D0
:10EE8000001BFF005B37FF00396DFF004155FF009D
:10EE9000544FFF005049FF004C4FFF005400FF004B
:10EEA0001B5BFF00307AFF001B5BFF002564FF0047
:10EEB0003B25FF006478FF00001BFF005B34FF0070
:10EEC0007A1BFF005B25FF00643BFF002564FF0009
:10EED0007800FF00ECF3FF004A48FF003595FF0083
:10EEE00095C7FF0017C1FF00DC45FF00FDDBFF00F9
:10EEF0006DC3FF0072B3FF003340FF002B34FF00EF
:10EF00000148FF007F9DFF00B045FF00E7FFFF00C5
:10EF1000D942FF000000FF00803FFF001B5BFF00A5
:10EF2000302FFF007200FF001B5BFF002564FF0015
:10EF30003B25FF00642EFF007200FF001B5BFF00FB
:10EF40002564FF003B25FF00642DFF007200FF00D9
:10EF50001B5BFF002F72FF00001BFF005B25FF0003
:10EF6000643BFF002564FF002E72FF00001BFF00C2
:10EF70005B34FF003B30FF003B33FF003630FF00C7
:10EF80002972FF001B5BFF002F72FF00001BFF00B8
:10EF90005B30FF007A1BFF005B25FF00643BFF0036
:10EFA0002564FF004800FF002530FF003264FF00A9
:10EFB0003A25FF003032FF00641BFF005B34FF0086
:10EFC0007A25FF003032FF006420FF005554FF0017
:10EFD0004300FF002530FF003264FF003A25FF00A8
:10EFE0003032FF00641BFF005B34FF007A25FF0016
:10EFF0003032FF006400FF002523FF00362EFF00A3
:10F000003166FF001B5BFF00317AFF006B70FF0071
:10F010006800FF002523FF00362EFF003166FF0049
:10F020001B5BFF00317AFF006D70FF006800FF007E
:10F030002523FF00362EFF003166FF001B5BFF001B
:10F04000317AFF006D00FF002523FF00362EFF0000
:10F050003166FF001B5BFF00317AFF006674FF0022
:10F06000001BFF005B30FF007A25FF006325FF00D7
:10F070006300FF002523FF00352EFF003266FF00EE
:10F080001B5BFF00317AFF005600FF002523FF00C5
:10F09000352EFF003266FF001B5BFF00317AFF0058
:10F0A000561BFF005B36FF00396DFF001B5BFF0046
:10F0B000347AFF002045FF005854FF000025FF0070
:10F0C0002335FF002E31FF00661BFF005B31FF0080
:10F0D0007A41FF000025FF00352EFF003066FF005B
:10F0E0001B5BFF00317AFF006D41FF006800FF00ED
:10F0F0002534FF002E30FF00661BFF005B31FF0050
:10F100007A6DFF000025FF002334FF002E32FF0040
:10F11000661BFF005B31FF007A6DFF006C00FF0093
:10F120002534FF002E30FF00661BFF005B31FF001F
:10F130007A66FF007400FF002535FF002E30FF00C7
:10F14000661BFF005B31FF007A6DFF000025FF00AA
:10F150002335FF002E32FF00661BFF005B31FF00EE
:10F160007A6DFF006C00FF002535FF002E30FF0098
:10F17000661BFF005B31FF007A66FF007400FF0032
:10F180001B5BFF00347AFF005350FF004545FF0032
:10F190004420FF001B5BFF00307AFF002523FF00A7
:10F1A000362EFF003166FF001B5BFF00317AFF0047
:10F1B0006B70FF006800FF001B5BFF00347AFF00EC
:10F1C0002020FF00414CFF005420FF001B5BFF008C
:10F1D000307AFF002523FF00362EFF003166FF0046
:10F1E0001B5BFF00317AFF006D00FF001B5BFF001F
:10F1F000347AFF005241FF004E47FF004520FF00D8
:10F200001B5BFF00307AFF002536FF002E30FF0029
:10F21000661BFF005B31FF007A6DFF00001BFF00E3
:10F220005B34FF007A53FF005045FF004544FF0068
:10F23000201BFF005B30FF007A25FF002336FF0014
:10F240002E31FF00661BFF005B31FF007A6DFF006F
:10F250007068FF00001BFF005B34FF007A20FF0096
:10F260002041FF004C54FF00201BFF005B30FF00DB
:10F270007A25FF002336FF002E31FF00661BFF00BA
:10F280005B31FF007A66FF007400FF001B5BFF002C
:10F29000347AFF005241FF004E47FF004520FF0037
:10F2A0001B5BFF00307AFF002523FF00362EFF0096
:10F2B0003266FF001B5BFF00317AFF006D6CFF00C0
:10F2C000001BFF005B34FF007A20FF004355FF0066
:10F2D0005252FF00201BFF005B30FF007A25FF0029
:10F2E0002336FF002E31FF00661BFF005B31FF005D
:10F2F0007A41FF00001BFF005B36FF00356DFF0009
:10F300002532FF00641BFF005B36FF00396DFF00F4
:10F310001B5BFF00347AFF002053FF004154FF00C5
:10F320005300FF002532FF00641BFF005B34FF0029
:10F330007A20FF005341FF005453FF000025FF00D7
:10F340002331FF00302EFF003666FF001B5BFF00FD
:10F35000347AFF002563FF000025FF002331FF0002
:10F36000302EFF003666FF001B5BFF00347AFF0083
:10F370002563FF00001BFF005B34FF007A48FF009D
:10F38000444FFF005020FF001B5BFF00307AFF005E
:10F390002523FF002D36FF002E31FF006600FF0001
:10F3A0002530FF003364FF000020FF002573FF00BD
:10F3B0002000FF001B5BFF003734FF006D25FF00BE
:10F3C0003033FF002E30FF006600FF002530FF00C5
:10F3D000332EFF003066FF000020FF001B5BFF00A4
:10F3E0003731FF006D25FF00731BFF005B36FF0008
:10F3F000396DFF002000FF002025FF007320FF0073
:10F400000020FF002573FF002000FF00C425FF003F
:10F41000631BFF005B34FF007A20FF001B5BFF00D3
:10F42000307AFF0000C4FF002563FF001B5BFF0074
:10F43000347AFF00201BFF005B30FF007A00FF00E2
:10F440002530FF003264FF002000FF001B5BFF003F
:10F450003858FF00001BFF005B36FF005800FF001C
:10F460001B5BFF003758FF00001BFF005B37FF00EE
:10F470005800FF001B5BFF00347AFF004C4FFF0079
:10F480005320FF001B5BFF00307AFF000050FF009D
:10F490004541FF004B20FF005641FF004C55FF0047
:10F4A0004553FF00001BFF005B31FF003158FF0098
:10F4B000001BFF005B31FF003258FF00001BFF0004
:10F4C0005B31FF003258FF00001BFF005B31FF0083
:10F4D0003258FF00001BFF005B31FF003258FF0075
:10F4E000001BFF005B39FF005800FF001B5BFF00A3
:10F4F0003558FF00001BFF005B31FF003158FF0053
:10F50000001BFF005B31FF003158FF00001BFF00B4
:10F510005B39FF005800FF00C0A0FF0000C0FF00E3
:10F52000A000FF00C3BFFF0000C4FF008000FF0079
:10F53000C0A0FF0000C4FF008000FF00C3BFFF00A9
:10F5400000C0FF00A000FF001B5BFF00347AFF003B
:10F55000002DFF002D20FF00001BFF005B32FF008D
:10F560004A00FF001B5BFF00317AFF001B5BFF00BE
:10F570002564FF003B25FF006478FF000020FF00AA
:10F580004D41FF005852FF00414EFF004745FF002C
:10F590002020FF002020FF001B5BFF00307AFF00CF
:10F5A0002536FF002E30FF006620FF000020FF0000
:10F5B0004C4FFF005741FF004C54FF005241FF00E9
:10F5C0005449FF004F20FF001B5BFF00307AFF0013
:10F5D0002536FF002E32FF006620FF000020FF00CE
:10F5E0005641FF004C49FF004448FF00444FFF00D4
:10F5F0005020FF002020FF001B5BFF00307AFF003F
:10F600002536FF002E31FF006620FF000020FF009E
:10F610004D49FF004E56FF00414CFF004944FF009A
:10F620002020FF002020FF001B5BFF00307AFF003E
:10F630002536FF006420FF000020FF005348FF0034
:10F640004F57FF00484FFF004D45FF004C49FF005A
:10F650004D20FF001B5BFF00307AFF002536FF00C6
:10F660002E30FF006620FF000020FF00524FFF00F9
:10F67000434CFF00494DFF004954FF002020FF008C
:10F680002020FF001B5BFF00307AFF002536FF00C3
:10F690002E31FF006620FF000020FF00524FFF00C8
:10F6A0004353FF005445FF005047FF004149FF000E
:10F6B0004E20FF001B5BFF00307AFF002536FF0065
:10F6C0002E30FF006620FF000020FF004150FF00A9
:10F6D000524FFF004347FF004149FF004E20FF000B
:10F6E0002020FF001B5BFF00307AFF002536FF0063
:10F6F0002E31FF006620FF000020FF00524FFF0068
:10F70000544CFF00494DFF004954FF002020FF00EA
:10F710002020FF001B5BFF00307AFF002536FF0032
:10F720002E31FF006620FF000020FF00524FFF0037
:10F730005453FF005445FF005047FF004149FF006C
:10F740004E20FF001B5BFF00307AFF002536FF00D4
:10F750002E30FF006620FF000020FF004150FF0018
:10F76000524FFF005447FF004149FF004E20FF0069
:10F770002020FF001B5BFF00307AFF002536FF00D2
:10F780002E31FF006620FF000020FF005350FF00D5
:10F790004545FF00444CFF004F57FF004C49FF0018
:10F7A0004D20FF001B5BFF00307AFF002536FF0075
:10F7B0002E31FF006620FF000020FF004352FF00B3
:10F7C0005549FF005345FF00414CFF005420FF0006
:10F7D0002020FF001B5BFF00307AFF002536FF0072
:10F7E0002E30FF006620FF000020FF004D41FF008B
:10F7F0005841FF004C54FF004348FF004720FF00E2
:10F800002020FF001B5BFF00307AFF002536FF0041
:10F810002E30FF006620FF000020FF004D41FF005A
:10F820005848FF004447FF004348FF004720FF00BF
:10F830002020FF001B5BFF00307AFF002536FF0011
:10F840002E30FF006620FF000020FF004D41FF002A
:10F850004857FF004152FF004E49FF004E47FF004E
:10F860002020FF001B5BFF00307AFF002536FF00E1
:10F870002E30FF006620FF000020FF00454CFF00F7
:10F880004553FF004552FF00564FFF004449FF001B
:10F890005220FF001B5BFF00307AFF002536FF007F
:10F8A0007320FF000020FF005244FF005253FF006E
:10F8B0004552FF00564FFF004449FF005220FF0011
:10F8C0001B5BFF00307AFF002536FF007320FF002E
:10F8D0000020FF00554EFF004954FF005320FF0059
:10F8E0002020FF002020FF002020FF002025FF0017
:10F8F0003873FF002000FF002041FF004D50FF0043
:10F90000535AFF004552FF004F20FF002020FF0008
:10F91000201BFF005B30FF007A25FF003664FF00EC
:10F920002000FF002056FF004944FF00454FFF0024
:10F930004D4FFF004445FF002020FF002020FF0026
:10F940002538FF007320FF000020FF004C4FFF0010
:10F950004750FF004552FF00494FFF004420FF0081
:10F960002020FF001B5BFF00307AFF002536FF00E0
:10F970006420FF000020FF00484FFF004D45FF00BE
:10F980004C4FFF004320FF002020FF002020FF00FD
:10F990002025FF003873FF002000FF00204DFF00EE
:10F9A0004148FF004D55FF004C54FF002020FF0050
:10F9B0001B5BFF00307AFF002025FF00372EFF0081
:10F9C0003566FF002000FF002041FF004D50FF0082
:10F9D0004D55FF004C54FF002020FF002020FF0069
:10F9E000201BFF005B30FF007A25FF00362EFF0052
:10F9F0003366FF002000FF002053FF004146FF0058
:10FA0000455AFF004F4EFF004520FF002020FF0019
:10FA1000201BFF005B30FF007A25FF003664FF00EB
:10FA20002000FF002056FF004F4CFF005431FF0024
:10FA30004C4FFF005741FF00524EFF00201BFF00BC
:10FA40005B30FF007A25FF003673FF002000FF00C7
:10FA50002044FF005241FF005748FF004F52FF0073
:10FA6000495AFF004F4EFF00201BFF005B30FF0094
:10FA70007A25FF003673FF002000FF002053FF00AF
:10FA80004156FF004520FF00434FFF004E46FF0058
:10FA90004947FF00201BFF005B30FF007A25FF0075
:10FAA0003673FF002000FF004E4FFF005200FF00A2
:10FAB0005245FF005600FF004E4FFF005200FF006E
:10FAC0005245FF005600FF004D45FF005452FF0015
:10FAD0004943FF000049FF004D50FF004552FF0021
:10FAE0004941FF004C00FF005041FF004C00FF0067
:10FAF0004E54FF005343FF000053FF004554FF00E6
:10FB00000055FF004E53FF004554FF00004FFF001B
:10FB10004646FF000020FF004F4EFF00004FFF0051
:10FB20004E00FF00204FFF004646FF00002AFF0066
:10FB30000044FF004F4EFF004500FF002530FF004E
:10FB40003278FF000024FF00504DFF00544BFF00AF
:10FB50002573FF002A25FF00730DFF000A00FF0038
:10FB60003331FF00342CFF00302CFF00312CFF001C
:10FB7000302CFF00312CFF00302CFF000031FF0043
:10FB80000030FF00002CFF00302CFF00302CFF0065
:10FB9000302CFF00302CFF00302CFF00302CFF00F9
:10FBA000302CFF00302CFF00302CFF00302CFF00E9
:10FBB0003000FF000000FF00803FFF00CDCCFF00C1
:10FBC000CC3DFF000AD7FF00233CFF006F12FF006F
:10FBD000833AFF0017B7FF00D138FF00ACC5FF0024
:10FBE0002737FF00BD37FF008635FF0095BFFF00B8
:10FBF000D633FF0077CCFF002B32FF005F70FF0091
:10FC00008930FF00FFE6FF00DB2EFF0008E5FF0064
:10FC10003C1EFF006042FF00A20DFF000000FF003D
:10FC2000803FFF000000FF002041FF000000FF00B8
:10FC3000C842FF000000FF007A44FF000040FF00C0
:10FC40001C46FF000050FF00C347FF000024FF00D8
:10FC50007449FF008096FF00184BFF0020BCFF0096
:10FC6000BE4CFF00286BFF006E4EFF00F902FF0044
:10FC70001550FF00EC78FF00AD60FF00CAF2FF00F6
:10FC80004971FF000100FF000000FF000A00FF00B3
:10FC90000000FF006400FF000000FF00E803FF0019
:10FCA0000000FF001027FF000000FF00A086FF00FB
:10FCB0000100FF004042FF000F00FF008096FF00A0
:10FCC0009800FF0000E1FF00F505FF0000CAFF00FB
:10FCD0009A3BFF000100FF000000FF001000FF0042
:10FCE0000000FF000001FF000000FF000010FF0007
:10FCF0000000FF000000FF000100FF000000FF0007
:10FD00001000FF000000FF000001FF000000FF00E6
:10FD10000010FF000100FF000000FF000800FF00CE
:10FD20000000FF004000FF000000FF000002FF0095
:10FD30000000FF000010FF000000FF000080FF0037
:10FD40000000FF000000FF000400FF000000FF00B3
:10FD50002000FF000000FF000001FF000000FF0086
:10FD60000008FF000000FF000040FF000000FF004F
:10FD70000000FF003031FF003233FF003435FF0058
:10FD80003637FF003839FF004142FF004344FF008F
:10FD90004546FF000030FF003132FF003334FF00E2
:10FDA0003536FF003738FF003961FF006263FF001E
:10FDB0006465FF006600FF00286EFF00756CFF00A1
:10FDC0006C29FF00001BFF005B25FF00646DFF0036
:10FDD000001BFF005B31FF00363BFF002564FF0086
:10FDE0007600FF004750FF00532FFF004F53FF00E6
:10FDF0004420FF005354FF004152FF005455FF00C0
:10FE00005020FF002564FF00001BFF005B32FF0055
:10FE1000313BFF003076FF001B5BFF003332FF00F9
:10FE20003B31FF007600FF001B5BFF00317AFF00D3
:10FE30004472FF006167FF006F6EFF004F53FF00C9
:10FE40004420FF005634FF002E37FF006B20FF00D8
:10FE50003139FF002F34FF002F32FF003030FF0018
:10FE60003820FF002863FF002920FF004461FF00C5
:10FE70006E69FF00656CFF002057FF006565FF009D
:10FE80000057FF006169FF007469FF006E67FF00A3
:10FE90002066FF006F72FF002047FF005053FF00F5
:10FEA0002064FF006174FF006120FF002E2EFF0020
:10FEB0002E00FF003030FF003000FF003232FF0024
:10FEC000302CFF003230FF003000FF000000FF0048
:10FED0000000FF000000FF000000FF00FFFFFF0028
:0200000401F009
:10000000F6FF0000F4FF00007F7A0000FFFFFF0012
:0C001000FFFFFF00FFFF0000FFFF0000EB
:00000001FF
